******************************************************************************
               TMS320C6x Linker PC v8.2.4                      
******************************************************************************
>> Linked Wed Feb 27 10:57:48 2019

OUTPUT FILE NAME:   <spiInterrupt.out>
ENTRY POINT SYMBOL: "_c_int00"  address: c3118be0


MEMORY CONFIGURATION

         name            origin    length      used     unused   attr    fill
----------------------  --------  ---------  --------  --------  ----  --------
  IROM                  11700000   00100000  00064000  0009c000  R  X
  IRAM                  11800000   00040000  00000000  00040000  RW X
  L3_CBA_RAM            80000000   00020000  00000000  00020000  RW X
  DDR                   c3000000   01000000  0013972e  00ec68d2  RWIX


SEGMENT ALLOCATION MAP

run origin  load origin   length   init length attrs members
----------  ----------- ---------- ----------- ----- -------
11700000    11700000    00064000   00000000    rw-
  11700000    11700000    00064000   00000000    rw- systemHeap
c3000000    c3000000    00100c20   00000000    rw-
  c3000000    c3000000    00100c10   00000000    rw- .far
  c3100c10    c3100c10    00000010   00000000    rw- .fardata.1
c3100c20    c3100c20    0001c700   0001c700    r-x
  c3100c20    c3100c20    0001c700   0001c700    r-x .text
c311d320    c311d320    000177dc   00000000    rw-
  c311d320    c311d320    000177dc   00000000    rw- .fardata.2
c3134b00    c3134b00    00002ec6   00002ec6    r--
  c3134b00    c3134b00    00002ec6   00002ec6    r-- .const
c31379c8    c31379c8    00001120   00000000    rw-
  c31379c8    c31379c8    00001000   00000000    rw- .stack
  c31389c8    c31389c8    00000120   00000000    rw- .cio
c3138ae8    c3138ae8    000000e0   000000e0    r--
  c3138ae8    c3138ae8    000000e0   000000e0    r-- .switch
c3138bc8    c3138bc8    0000002c   00000000    rw-
  c3138bc8    c3138bc8    00000004   00000000    rw- .bss
  c3138bcc    c3138bcc    00000028   00000000    rw- .neardata
c3138c00    c3138c00    00000b40   00000b40    r-x
  c3138c00    c3138c00    00000200   00000200    r-x .vecs
  c3138e00    c3138e00    00000940   00000940    r-- .cinit


SECTION ALLOCATION MAP

 output                                  attributes/
section   page    origin      length       input sections
--------  ----  ----------  ----------   ----------------
.stack     0    c31379c8    00001000     UNINITIALIZED
                  c31379c8    00000008     boot.ae674 : boot.oe674 (.stack)
                  c31379d0    00000ff8     --HOLE--

.bss       0    c3138bc8    00000004     UNINITIALIZED
                  c3138bc8    00000004     (.common:dsp_num)

.neardata 
*          0    c3138bcc    00000028     UNINITIALIZED
                  c3138bcc    00000018     ti.osal.ae674 : Utils_tirtos.oe674 (.neardata)
                  c3138be4    00000008     ti.drv.spi.ae674 : SPI_drv.oe674 (.neardata)
                  c3138bec    00000004                      : SPI_v0.oe674 (.neardata)
                  c3138bf0    00000004     ti.drv.uart.ae674 : UART_drv.oe674 (.neardata)

.rodata    0    c3138bf4    00000000     UNINITIALIZED

.cinit     0    c3138e00    00000940     
                  c3138e00    000008bd     (.cinit..fardata.2.load) [load image, compression = rle]
                  c31396bd    00000012     (.cinit..neardata.load) [load image, compression = rle]
                  c31396cf    00000011     (.cinit..fardata.1.load) [load image, compression = rle]
                  c31396e0    0000000d     (.cinit..far.load) [load image, compression = rle]
                  c31396ed    0000000d     (.cinit.systemHeap.load) [load image, compression = rle]
                  c31396fa    00000009     (.cinit..bss.load) [load image, compression = rle]
                  c3139703    00000001     --HOLE-- [fill = 0]
                  c3139704    00000008     (__TI_handler_table)
                  c313970c    00000004     --HOLE-- [fill = 0]
                  c3139710    00000030     (__TI_cinit_table)

.init_array 
*          0    c3000000    00000000     UNINITIALIZED

.vecs      0    c3138c00    00000200     
                  c3138c00    00000200     spi_test_pe674.oe674 (.vecs)

xdc.meta   0    c3000000    000000e8     COPY SECTION
                  c3000000    000000e8     spi_test_pe674.oe674 (xdc.meta)

systemHeap 
*          0    11700000    00064000     UNINITIALIZED
                  11700000    00064000     spi_test_pe674.oe674 (systemHeap)

.far       0    c3000000    00100c10     UNINITIALIZED
                  c3000000    00100800     spi_test_pe674.oe674 (.far:taskStackSection)
                  c3100800    00000198     (.common:UartObjects)
                  c3100998    00000140     (.common:__TI_tmpnams)
                  c3100ad8    00000098     (.common:SpiObjects)
                  c3100b70    00000014     (.common:edma3_dma_ch_max_val)
                  c3100b84    00000004     --HOLE--
                  c3100b88    00000014     (.common:edma3_link_ch_max_val)
                  c3100b9c    00000004     --HOLE--
                  c3100ba0    00000014     (.common:edma3_link_ch_min_val)
                  c3100bb4    00000004     --HOLE--
                  c3100bb8    00000014     (.common:edma3_log_ch_max_val)
                  c3100bcc    00000004     --HOLE--
                  c3100bd0    00000014     (.common:edma3_qdma_ch_max_val)
                  c3100be4    00000004     --HOLE--
                  c3100be8    00000014     (.common:edma3_qdma_ch_min_val)
                  c3100bfc    00000004     --HOLE--
                  c3100c00    00000008     (.common:parmbuf)
                  c3100c08    00000008     (.common:uart_stdio)

.fardata.1 
*          0    c3100c10    00000010     UNINITIALIZED
                  c3100c10    0000000c     rts6740_elf.lib : exit.obj (.fardata)
                  c3100c1c    00000004                     : _lock.obj (.fardata:_lock)

.text      0    c3100c20    0001c700     
                  c3100c20    00001ce0     rts6740_elf.lib : _printfi.obj (.text:__TI_printfi)
                  c3102900    00000c40     edma3_lld_rm.ae674 : edma3resmgr.oe674 (.text:EDMA3_RM_allocResource)
                  c3103540    00000c20     edma3_lld_drv.ae674 : edma3_drv_basic.oe674 (.text:EDMA3_DRV_requestChannel)
                  c3104160    000008a0     ti.targets.rts6000.ae674 : System.oe674 (.text:xdc_runtime_System_doPrint__I)
                  c3104a00    00000820     ti.drv.spi.ae674 : SPI_v0.oe674 (.text:SPI_open_v0$0)
                  c3105220    00000780     sysbios.ae674 : BIOS.obj (.text:ti_sysbios_family_c64p_Exception_handler__I)
                  c31059a0    00000780                   : BIOS.obj (.text:ti_sysbios_knl_Semaphore_pend__E)
                  c3106120    000006e0                   : BIOS.obj (.text:ti_sysbios_timers_timer64_Timer_Module_startup__E)
                  c3106800    000006c0     ti.drv.uart.ae674 : UART_v0.oe674 (.text:UART_v0_hwiIntFxn$0)
                  c3106ec0    00000680     rts6740_elf.lib : _printfi.obj (.text:_pconv_a)
                  c3107540    00000640     ti.drv.uart.ae674 : UART_stdio.oe674 (.text:UART_printf)
                  c3107b80    00000640     sysbios.ae674 : BIOS.obj (.text:ti_sysbios_family_c64p_Cache_Module_startup__E)
                  c31081c0    00000640                   : BIOS.obj (.text:ti_sysbios_heaps_HeapMem_allocUnprotected__E)
                  c3108800    000005c0     rts6740_elf.lib : divd.obj (.text:__c6xabi_divd)
                  c3108dc0    000005a0     sysbios.ae674 : BIOS.obj (.text:ti_sysbios_heaps_HeapMem_freeUnprotected__E)
                  c3109360    00000560     ti.drv.spi.ae674 : SPI_v0.oe674 (.text:SPI_v0_hwiFxn$0)
                  c31098c0    00000500     rts6740_elf.lib : _printfi.obj (.text:_pconv_g)
                  c3109dc0    00000480     ti.drv.spi.ae674 : SPI_v0.oe674 (.text:SPI_transfer_v0$0)
                  c310a240    00000460     ti.board.ae674 : lcdkOMAPL138_pinmux.oe674 (.text:Board_pinmuxConfig)
                  c310a6a0    00000440     edma3_lld_rm.ae674 : edma3resmgr.oe674 (.text:EDMA3_RM_freeResource)
                  c310aae0    00000440     ti.drv.uart.ae674 : UART_v0.oe674 (.text:UART_open_v0$0)
                  c310af20    00000440     sysbios.ae674 : BIOS.obj (.text:ti_sysbios_knl_Task_sleep__E)
                  c310b360    00000420     ti.drv.uart.ae674 : UART_v0.oe674 (.text:UART_write2_v0$0)
                  c310b780    00000420     rts6740_elf.lib : _printfi.obj (.text:_pconv_e)
                  c310bba0    00000400     ti.drv.uart.ae674 : UART_v0.oe674 (.text:UART_read2_v0$0)
                  c310bfa0    000003e0     rts6740_elf.lib : fputs.obj (.text:fputs)
                  c310c380    00000340     sysbios.ae674 : BIOS.obj (.text:ti_sysbios_timers_timer64_Timer_deviceConfig__I)
                  c310c6c0    00000320     edma3_lld_drv.ae674 : edma3_drv_basic.oe674 (.text:EDMA3_DRV_freeChannel)
                  c310c9e0    00000320     sysbios.ae674 : BIOS.obj (.text:ti_sysbios_knl_Swi_runLoop__I)
                  c310cd00    000002e0     ti.board.ae674 : lcdkOMAPL138_pll.oe674 (.text:Board_CorePLLConfig)
                  c310cfe0    000002c0     edma3_lld_drv.ae674 : edma3_drv_basic.oe674 (.text:EDMA3_DRV_disableTransfer)
                  c310d2a0    000002c0     ti.drv.spi.ae674 : SPI_v0.oe674 (.text:SPI_DMA_primeTransfer_v0$0)
                  c310d560    000002c0     edma3_lld_drv.ae674 : edma3_drv_basic.oe674 (.text:edma3RemoveMapping)
                  c310d820    000002c0     sysbios.ae674 : BIOS.obj (.text:ti_sysbios_heaps_HeapMem_Instance_init__E)
                  c310dae0    000002c0                   : BIOS.obj (.text:ti_sysbios_knl_Task_Module_startup__E)
                  c310dda0    000002a0     ti.board.ae674 : lcdkOMAPL138_pll.oe674 (.text:Board_DDRPLLConfig)
                  c310e040    000002a0     rts6740_elf.lib : _printfi.obj (.text:_pconv_f)
                  c310e2e0    000002a0                     : _printfi.obj (.text:fcvt)
                  c310e580    000002a0     sysbios.ae674 : BIOS.obj (.text:ti_sysbios_knl_Clock_workFunc__E)
                  c310e820    00000280     edma3_lld_drv.ae674 : edma3_drv_basic.oe674 (.text:EDMA3_DRV_enableTransfer)
                  c310eaa0    00000280     sysbios.ae674 : BIOS.obj (.text:ti_sysbios_family_c64p_Hwi_reconfig__E)
                  c310ed20    00000280                   : BIOS.obj (.text:ti_sysbios_knl_Semaphore_post__E)
                  c310efa0    00000260     rts6740_elf.lib : imath64.obj (.text:__c6xabi_divull)
                  c310f200    00000260     sysbios.ae674 : BIOS.obj (.text:ti_sysbios_family_c64p_Cache_block__I)
                  c310f460    00000260                   : BIOS.obj (.text:ti_sysbios_family_c64p_Hwi_dispatchCore__I)
                  c310f6c0    00000260     ti.targets.rts6000.ae674 : Startup.oe674 (.text:xdc_runtime_Startup_startMods__I)
                  c310f920    00000240     ti.board.ae674 : lcdkOMAPL138_clock.oe674 (.text:Board_moduleClockEnable)
                  c310fb60    00000240     sysbios.ae674 : BIOS.obj (.text:ti_sysbios_family_c64p_EventCombiner_dispatch__E)
                  c310fda0    00000240                   : BIOS.obj (.text:ti_sysbios_family_c64p_Exception_internalHandler__I)
                  c310ffe0    00000240     ti.targets.rts6000.ae674 : Core-mem.oe674 (.text:xdc_runtime_Core_createObject__I)
                  c3110220    00000240     spi_test_pe674.oe674 (.text:xdc_runtime_System_printfExtend__I)
                  c3110460    00000220     rts6740_elf.lib : fputc.obj (.text:fputc)
                  c3110680    00000220     main_spi_loopback_example.obj (.text)
                  c31108a0    00000220     rts6740_elf.lib : setvbuf.obj (.text:setvbuf)
                  c3110ac0    00000220     sysbios.ae674 : BIOS.obj (.text:ti_sysbios_knl_Swi_run__I)
                  c3110ce0    00000220                   : BIOS.obj (.text:ti_sysbios_timers_timer64_Timer_setPeriodMicroSecs__E)
                  c3110f00    00000200     ti.osal.ae674 : SemaphoreP_tirtos.oe674 (.text:SemaphoreP_create)
                  c3111100    00000200     ti.drv.uart.ae674 : UART_v0.oe674 (.text:UART_readPolling_v0$0)
                  c3111300    00000200     rts6740_elf.lib : _printfi.obj (.text:_ltostr)
                  c3111500    00000200     sysbios.ae674 : c64p_Hwi_disp_always.obj (.text:_ti_sysbios_family_c64p_Hwi_dispatchAlways)
                  c3111700    00000200     ti.targets.rts6000.ae674 : Error.oe674 (.text:xdc_runtime_Error_policyDefault__E)
                  c3111900    000001e0     ti.board.ae674 : lcdkOMAPL138_clock.oe674 (.text:Board_moduleClockSyncReset)
                  c3111ae0    000001e0     ti.osal.ae674 : HwiP_tirtos.oe674 (.text:HwiP_create)
                  c3111cc0    000001e0     ti.drv.uart.ae674 : UART_stdio.oe674 (.text:UART_convertVal$0)
                  c3111ea0    000001e0     sysbios.ae674 : BIOS.obj (.text:ti_sysbios_gates_GateMutex_enter__E)
                  c3112080    000001e0     ti.targets.rts6000.ae674 : Text.oe674 (.text:xdc_runtime_Text_putSite__E)
                  c3112260    000001c0     edma3_lld_drv.ae674 : edma3_drv_adv.oe674 (.text:EDMA3_DRV_linkChannel)
                  c3112420    000001c0     rts6740_elf.lib : imath40.obj (.text:__c6xabi_divul)
                  c31125e0    000001c0                     : frexp.obj (.text:frexp)
                  c31127a0    000001c0     sysbios.ae674 : BIOS.obj (.text:ti_sysbios_family_c64p_EventCombiner_dispatchPlug__E)
                  c3112960    000001c0                   : BIOS.obj (.text:ti_sysbios_timers_timer64_Timer_getFreq__E)
                  c3112b20    000001a0     rts6740_elf.lib : hostrename.obj (.text:HOSTrename)
                  c3112cc0    000001a0     ti.drv.spi.ae674 : SPI_v0.oe674 (.text:SPI_control_v0$0)
                  c3112e60    000001a0     sysbios.ae674 : BIOS.obj (.text:ti_sysbios_family_c64p_EventCombiner_disableEvent__E)
                  c3113000    000001a0                   : BIOS.obj (.text:ti_sysbios_family_c64p_EventCombiner_enableEvent__E)
                  c31131a0    000001a0                   : BIOS.obj (.text:ti_sysbios_heaps_HeapBuf_Module_startup__E)
                  c3113340    000001a0                   : BIOS.obj (.text:ti_sysbios_timers_timer64_Timer_start__E)
                  c31134e0    000001a0     ti.targets.rts6000.ae674 : Core-smem.oe674 (.text:xdc_runtime_Core_constructObject__I)
                  c3113680    00000180     ti.board.ae674 : lcdkOMAPL138_ddr.oe674 (.text:Board_DDR3Init)
                  c3113800    00000180     edma3_lld_drv.ae674 : edma3_drv_adv.oe674 (.text:EDMA3_DRV_getPaRAM)
                  c3113980    00000180     edma3_lld_rm.ae674 : edma3resmgr.oe674 (.text:EDMA3_RM_registerTccCb)
                  c3113b00    00000180                        : edma3resmgr.oe674 (.text:EDMA3_RM_unregisterTccCb)
                  c3113c80    00000180     rts6740_elf.lib : ldexp.obj (.text:ldexp)
                  c3113e00    00000180     sysbios.ae674 : c64p_Exception_asm.obj (.text)
                  c3113f80    00000180                   : BIOS.obj (.text:ti_sysbios_knl_Task_exit__E)
                  c3114100    00000180                   : BIOS.obj (.text:ti_sysbios_knl_Task_schedule__I)
                  c3114280    00000180                   : BIOS.obj (.text:ti_sysbios_knl_Task_startCore__E)
                  c3114400    00000160     ti.board.ae674 : lcdkOMAPL138.oe674 (.text:Board_init)
                  c3114560    00000160     ti.osal.ae674 : RegisterIntr_tirtos.oe674 (.text:Osal_RegisterInterrupt)
                  c31146c0    00000160     sysbios.ae674 : BIOS.obj (.text:ti_sysbios_knl_Swi_post__E)
                  c3114820    00000160     ti.targets.rts6000.ae674 : Text.oe674 (.text:xdc_runtime_Text_putMod__E)
                  c3114980    00000140     edma3_lld_drv.ae674 : edma3_drv_adv.oe674 (.text:EDMA3_DRV_setPaRAM)
                  c3114ac0    00000140     rts6740_elf.lib : fclose.obj (.text:__TI_closefile)
                  c3114c00    00000140                     : fflush.obj (.text:fflush)
                  c3114d40    00000140                     : getdevice.obj (.text:getdevice)
                  c3114e80    00000140     sysbios.ae674 : BIOS.obj (.text:ti_sysbios_family_c64p_Hwi_Module_startup__E)
                  c3114fc0    00000140                   : BIOS.obj (.text:ti_sysbios_knl_Semaphore_Instance_init__E)
                  c3115100    00000140                   : BIOS.obj (.text:ti_sysbios_knl_Task_blockI__E)
                  c3115240    00000140     ti.targets.rts6000.ae674 : Core-mem.oe674 (.text:xdc_runtime_Core_deleteObject__I)
                  c3115380    00000140                              : Text.oe674 (.text:xdc_runtime_Text_putLab__E)
                  c31154c0    00000120     ti.board.ae674 : lcdkOMAPL138_pinmux.oe674 (.text:Board_configEmifPinMux)
                  c31155e0    00000120     ti.drv.spi.ae674 : SPI_v0.oe674 (.text:SPI_DMA_rxIsrHandler_v0$0)
                  c3115700    00000120                      : SPI_v0.oe674 (.text:SPI_DMA_txIsrHandler_v0$0)
                  c3115820    00000120     boot.ae674 : autoinit.oe674 (.text:_auto_init_elf)
                  c3115940    00000120     rts6740_elf.lib : fseek.obj (.text:fseek)
                  c3115a60    00000120     sysbios.ae674 : BIOS.obj (.text:ti_sysbios_family_c64p_Hwi_Instance_init__E)
                  c3115b80    00000120                   : BIOS.obj (.text:ti_sysbios_knl_Task_unblockI__E)
                  c3115ca0    00000100     ti.board.ae674 : lcdkOMAPL138_clock.oe674 (.text:Board_moduleClockInit)
                  c3115da0    00000100     edma3_lld_drv.ae674 : edma3_drv_basic.oe674 (.text:EDMA3_DRV_clearErrorBits)
                  c3115ea0    00000100     ti.osal.ae674 : EventCombinerP_tirtos.oe674 (.text:EventCombinerP_GroupRegisterInt)
                  c3115fa0    00000100     ti.drv.spi.ae674 : SPI_v0.oe674 (.text:SPI_close_v0$0)
                  c31160a0    00000100     ti.drv.uart.ae674 : UART_v0.oe674 (.text:UART_writePolling_v0$0)
                  c31161a0    00000100     rts6740_elf.lib : copy_decompress_rle.obj (.text:__TI_decompress_rle_core)
                  c31162a0    00000100                     : _io_perm.obj (.text:__TI_wrt_ok)
                  c31163a0    00000100                     : atoi.obj (.text:atoi)
                  c31164a0    00000100     sysbios.ae674 : BIOS.obj (.text:ti_sysbios_family_c64p_Hwi_Instance_finalize__E)
                  c31165a0    00000100                   : BIOS.obj (.text:ti_sysbios_knl_Swi_restoreHwi__E)
                  c31166a0    00000100                   : BIOS.obj (.text:ti_sysbios_timers_timer64_Timer_initDevice__I)
                  c31167a0    00000100     ti.targets.rts6000.ae674 : Error.oe674 (.text:xdc_runtime_Error_print__E)
                  c31168a0    00000100                              : Memory.oe674 (.text:xdc_runtime_Memory_alloc__E)
                  c31169a0    00000100                              : Startup.oe674 (.text:xdc_runtime_Startup_exec__E)
                  c3116aa0    000000e0     edma3_lld_drv.ae674 : edma3_drv_adv.oe674 (.text:EDMA3_DRV_getPaRAMPhyAddr)
                  c3116b80    000000e0                         : edma3_drv_adv.oe674 (.text:EDMA3_DRV_unlinkChannel)
                  c3116c60    000000e0     rts6740_elf.lib : hostlseek.obj (.text:HOSTlseek)
                  c3116d40    000000e0                     : hostopen.obj (.text:HOSTopen)
                  c3116e20    000000e0                     : hostwrite.obj (.text:HOSTwrite)
                  c3116f00    000000e0     ti.drv.spi.ae674 : SPI_drv.oe674 (.text:SPI_init)
                  c3116fe0    000000e0     ti.drv.uart.ae674 : UART_v0.oe674 (.text:UART_close_v0$0)
                  c31170c0    000000e0                       : UART_v0.oe674 (.text:UART_read_v0$0)
                  c31171a0    000000e0                       : UART_v0.oe674 (.text:UART_write_v0$0)
                  c3117280    000000e0     rts6740_elf.lib : close.obj (.text:close)
                  c3117360    000000e0                     : exit.obj (.text:exit)
                  c3117440    000000e0                     : ltoa.obj (.text:ltoa)
                  c3117520    000000e0                     : memset.obj (.text:memset)
                  c3117600    000000e0                     : printf.obj (.text:printf)
                  c31176e0    000000e0     sysbios.ae674 : BIOS.obj (.text:ti_sysbios_heaps_HeapMem_alloc__E)
                  c31177c0    000000e0                   : BIOS.obj (.text:ti_sysbios_timers_timer64_Timer_startup__E)
                  c31178a0    000000e0     ti.targets.rts6000.ae674 : Text.oe674 (.text:xdc_runtime_Text_visitRope2__I)
                  c3117980    000000c0     rts6740_elf.lib : hostread.obj (.text:HOSTread)
                  c3117a40    000000c0                     : hostunlink.obj (.text:HOSTunlink)
                  c3117b00    000000c0     ti.osal.ae674 : Utils_tirtos.oe674 (.text:Osal_delay)
                  c3117bc0    000000c0     ti.drv.spi.ae674 : SPI_drv.oe674 (.text:SPI_open)
                  c3117c80    000000c0     ti.drv.uart.ae674 : UART_v0.oe674 (.text:UART_charPut$0)
                  c3117d40    000000c0                       : UART_v0.oe674 (.text:UART_readCancelNoCB$0)
                  c3117e00    000000c0     rts6740_elf.lib : fflush.obj (.text:__TI_doflush)
                  c3117ec0    000000c0                     : divu.obj (.text:__divu)
                  c3117f80    000000c0                     : _printfi.obj (.text:_ecpy)
                  c3118040    000000c0     edma3_lld_rm.ae674 : edma3resmgr.oe674 (.text:edma3MemZero)
                  c3118100    000000c0     edma3_lld_drv_sample.ae674 : sample_cs.oe674 (.text:edma3OsProtectEntry)
                  c31181c0    000000c0     sysbios.ae674 : BIOS.obj (.text:ti_sysbios_heaps_HeapMem_getStats__E)
                  c3118280    000000c0                   : BIOS.obj (.text:ti_sysbios_knl_Clock_logTick__E)
                  c3118340    000000c0                   : BIOS.obj (.text:ti_sysbios_knl_Swi_schedule__I)
                  c3118400    000000c0     rts6740_elf.lib : tls.obj (.text:tls:init:__TI_tls_init)
                  c31184c0    000000c0     ti.targets.rts6000.ae674 : Assert.oe674 (.text:xdc_runtime_Assert_raise__I)
                  c3118580    000000c0                              : Error.oe674 (.text:xdc_runtime_Error_setX__E)
                  c3118640    000000a0     rts6740_elf.lib : hostclose.obj (.text:HOSTclose)
                  c31186e0    000000a0     ti.osal.ae674 : RegisterIntr_tirtos.oe674 (.text:Osal_DeleteInterrupt)
                  c3118780    000000a0     ti.drv.spi.ae674 : SPI_v0.oe674 (.text:SPI_DMA_localCompleteIOedmaCbk_v0$0)
                  c3118820    000000a0     ti.drv.uart.ae674 : UART_drv.oe674 (.text:UART_init)
                  c31188c0    000000a0                       : UART_stdio.oe674 (.text:UART_stdioInit)
                  c3118960    000000a0                       : UART_v0.oe674 (.text:UART_v0_callback$0)
                  c3118a00    000000a0                       : UART_v0.oe674 (.text:UART_writeCancelNoCB$0)
                  c3118aa0    000000a0     rts6740_elf.lib : fopen.obj (.text:__TI_cleanup)
                  c3118b40    000000a0                     : remu.obj (.text:__remu)
                  c3118be0    000000a0     boot.ae674 : boot.oe674 (.text:_c_int00)
                  c3118c80    000000a0     sysbios.ae674 : c64p_Hwi_asm.obj (.text:_ti_sysbios_family_c64p_Hwi_plug__E)
                  c3118d20    000000a0     rts6740_elf.lib : memcpy64.obj (.text:memcpy)
                  c3118dc0    000000a0     sysbios.ae674 : BIOS.obj (.text:ti_sysbios_family_c64p_Exception_Module_startup__E)
                  c3118e60    000000a0     spi_test_pe674.oe674 (.text:ti_sysbios_family_c64p_Hwi_construct)
                  c3118f00    000000a0     sysbios.ae674 : BIOS.obj (.text:ti_sysbios_family_c64p_Hwi_dispatchC__I)
                  c3118fa0    000000a0                   : BIOS.obj (.text:ti_sysbios_family_c64p_Hwi_getStackInfo__E)
                  c3119040    000000a0                   : BIOS.obj (.text:ti_sysbios_heaps_HeapMem_init__I)
                  c31190e0    000000a0                   : BIOS.obj (.text:ti_sysbios_knl_Task_allBlockedFunction__I)
                  c3119180    000000a0                   : BIOS.obj (.text:ti_sysbios_timers_timer64_Timer_stop__E)
                  c3119220    000000a0     ti.targets.rts6000.ae674 : Core-params.oe674 (.text:xdc_runtime_Core_assignParams__I)
                  c31192c0    000000a0                              : System.oe674 (.text:xdc_runtime_System_formatNum__I)
                  c3119360    000000a0                              : System.oe674 (.text:xdc_runtime_System_putchar__I)
                  c3119400    000000a0                              : Text.oe674 (.text:xdc_runtime_Text_printVisFxn__I)
                  c31194a0    000000a0                              : Text.oe674 (.text:xdc_runtime_Text_xprintf__I)
                  c3119540    00000080     ti.board.ae674 : lcdkOMAPL138_clock.oe674 (.text:CSL_PSC_setModuleNextState$0)
                  c31195c0    00000080     ti.osal.ae674 : EventCombinerP_tirtos.oe674 (.text:EventCombinerP_getHwi)
                  c3119640    00000080                   : EventCombinerP_tirtos.oe674 (.text:EventCombinerP_getIntNum)
                  c31196c0    00000080     ti.csl.ae674 : uart.oe674 (.text:UART_charPut_v0)
                  c3119740    00000080     rts6740_elf.lib : trgmsg.obj (.text:__TI_readmsg)
                  c31197c0    00000080                     : llshift.obj (.text:__c6xabi_llshl)
                  c3119840    00000080     sysbios.ae674 : c62_TaskSupport_asm.obj (.text:_ti_sysbios_family_c62_TaskSupport_swap__E)
                  c31198c0    00000080     edma3_lld_drv_sample.ae674 : sample_cs.oe674 (.text:edma3OsProtectExit)
                  c3119940    00000080     edma3_lld_rm.ae674 : edma3resmgr.oe674 (.text:edma3ParamCpy)
                  c31199c0    00000080     rts6740_elf.lib : getdevice.obj (.text:finddevice)
                  c3119a40    00000080     spi_test_pe674.oe674 (.text:ti_sysbios_BIOS_atExitFunc__I)
                  c3119ac0    00000080     spi_test_pe674.oe674 (.text:ti_sysbios_BIOS_registerRTSLock__I)
                  c3119b40    00000080     sysbios.ae674 : BIOS.obj (.text:ti_sysbios_family_c64p_Cache_invL1pAll__E)
                  c3119bc0    00000080     spi_test_pe674.oe674 (.text:ti_sysbios_gates_GateHwi_Object__create__S)
                  c3119c40    00000080     spi_test_pe674.oe674 (.text:ti_sysbios_gates_GateMutex_Object__create__S)
                  c3119cc0    00000080     sysbios.ae674 : BIOS.obj (.text:ti_sysbios_hal_Hwi_checkStack)
                  c3119d40    00000080                   : BIOS.obj (.text:ti_sysbios_hal_Hwi_initStack)
                  c3119dc0    00000080     spi_test_pe674.oe674 (.text:ti_sysbios_heaps_HeapMem_Object__create__S)
                  c3119e40    00000080     spi_test_pe674.oe674 (.text:ti_sysbios_knl_Clock_doTick__I)
                  c3119ec0    00000080     sysbios.ae674 : BIOS.obj (.text:ti_sysbios_knl_Idle_run__E)
                  c3119f40    00000080                   : BIOS.obj (.text:ti_sysbios_knl_Semaphore_pendTimeout__I)
                  c3119fc0    00000080                   : BIOS.obj (.text:ti_sysbios_knl_Swi_startup__E)
                  c311a040    00000080                   : BIOS.obj (.text:ti_sysbios_knl_Task_restore__E)
                  c311a0c0    00000080     spi_test_pe674.oe674 (.text:ti_sysbios_rts_MemAlloc_alloc)
                  c311a140    00000080     rts6740_elf.lib : unlink.obj (.text:unlink)
                  c311a1c0    00000080     ti.targets.rts6000.ae674 : Core-label.oe674 (.text:xdc_runtime_Core_assignLabel__I)
                  c311a240    00000080                              : SysStd.oe674 (.text:xdc_runtime_SysStd_abort__E)
                  c311a2c0    00000080                              : System.oe674 (.text:xdc_runtime_System_atexit__E)
                  c311a340    00000080                              : System.oe674 (.text:xdc_runtime_System_avprintf__E)
                  c311a3c0    00000080                              : System.oe674 (.text:xdc_runtime_System_processAtExit__E)
                  c311a440    00000080                              : System.oe674 (.text:xdc_runtime_System_vprintf__E)
                  c311a4c0    00000060     ti.osal.ae674 : HwiP_tirtos.oe674 (.text:HwiP_delete)
                  c311a520    00000060                   : RegisterIntr_tirtos.oe674 (.text:Osal_ClearInterrupt)
                  c311a580    00000060                   : Utils_tirtos.oe674 (.text:Osal_getHwAttrs)
                  c311a5e0    00000060                   : Utils_tirtos.oe674 (.text:Osal_getThreadType)
                  c311a640    00000060     ti.csl.ae674 : spi.oe674 (.text:SPIDataFormatSetup)
                  c311a6a0    00000060     ti.drv.spi.ae674 : SPI_drv.oe674 (.text:SPI_Params_init)
                  c311a700    00000060                      : SPI_drv.oe674 (.text:SPI_control)
                  c311a760    00000060                      : SPI_soc.oe674 (.text:SPI_socGetInitCfg)
                  c311a7c0    00000060                      : SPI_soc.oe674 (.text:SPI_socSetInitCfg)
                  c311a820    00000060                      : SPI_drv.oe674 (.text:SPI_transfer)
                  c311a880    00000060     ti.osal.ae674 : SemaphoreP_tirtos.oe674 (.text:SemaphoreP_delete)
                  c311a8e0    00000060                   : SemaphoreP_tirtos.oe674 (.text:SemaphoreP_pend)
                  c311a940    00000060     ti.csl.ae674 : uart.oe674 (.text:UART_divisorLatchWrite_v0)
                  c311a9a0    00000060                  : uart.oe674 (.text:UART_fifoWait_v0)
                  c311aa00    00000060                  : uart.oe674 (.text:UART_lineCharacConfig_v0)
                  c311aa60    00000060     ti.drv.uart.ae674 : UART_v0.oe674 (.text:UART_readCancel_v0$0)
                  c311aac0    00000060                       : UART_v0.oe674 (.text:UART_writeCancel_v0$0)
                  c311ab20    00000060     rts6740_elf.lib : trgmsg.obj (.text:__TI_writemsg)
                  c311ab80    00000060                     : llshift.obj (.text:__c6xabi_llshru)
                  c311abe0    00000060                     : imath64.obj (.text:_subcull)
                  c311ac40    00000060     sysbios.ae674 : c64p_Hwi_asm_switch.obj (.text:_ti_sysbios_family_c64p_Hwi_switchAndDispatch__I)
                  c311aca0    00000060                   : c64p_Hwi_asm_switch.obj (.text:_ti_sysbios_family_xxx_Hwi_switchAndRunFunc)
                  c311ad00    00000060     edma3_lld_drv_sample.ae674 : sample_cs.oe674 (.text:edma3OsSemTake)
                  c311ad60    00000060     rts6740_elf.lib : lseek.obj (.text:lseek)
                  c311adc0    00000060                     : memccpy.obj (.text:memccpy)
                  c311ae20    00000060     spi_test_pe674.oe674 (.text:ti_sysbios_BIOS_errorRaiseHook__I)
                  c311ae80    00000060     spi_test_pe674.oe674 (.text:ti_sysbios_BIOS_removeRTSLock__I)
                  c311aee0    00000060     spi_test_pe674.oe674 (.text:ti_sysbios_BIOS_startFunc__I)
                  c311af40    00000060     sysbios.ae674 : BIOS.obj (.text:ti_sysbios_family_c62_TaskSupport_start__E)
                  c311afa0    00000060                   : BIOS.obj (.text:ti_sysbios_family_c64p_Cache_setMar__E)
                  c311b000    00000060                   : BIOS.obj (.text:ti_sysbios_family_c64p_EventCombiner_Module_startup__E)
                  c311b060    00000060                   : BIOS.obj (.text:ti_sysbios_family_c64p_EventCombiner_unused__E)
                  c311b0c0    00000060                   : BIOS.obj (.text:ti_sysbios_family_c64p_Hwi_getEventId__E)
                  c311b120    00000060     spi_test_pe674.oe674 (.text:ti_sysbios_gates_GateMutex_Object__delete__S)
                  c311b180    00000060     sysbios.ae674 : BIOS.obj (.text:ti_sysbios_heaps_HeapMem_free__E)
                  c311b1e0    00000060                   : BIOS.obj (.text:ti_sysbios_knl_Clock_Module_startup__E)
                  c311b240    00000060     spi_test_pe674.oe674 (.text:ti_sysbios_knl_Queue_construct)
                  c311b2a0    00000060     spi_test_pe674.oe674 (.text:ti_sysbios_knl_Semaphore_construct)
                  c311b300    00000060     sysbios.ae674 : BIOS.obj (.text:ti_sysbios_knl_Swi_Module_startup__E)
                  c311b360    00000060                   : BIOS.obj (.text:ti_sysbios_knl_Task_enter__I)
                  c311b3c0    00000060     ti.drv.uart.ae674 : UART_stdio.oe674 (.text:uart_console_putc$0)
                  c311b420    00000060     rts6740_elf.lib : write.obj (.text:write)
                  c311b480    00000060     ti.targets.rts6000.ae674 : Memory.oe674 (.text:xdc_runtime_Memory_valloc__E)
                  c311b4e0    00000060                              : Text.oe674 (.text:xdc_runtime_Text_cordText__E)
                  c311b540    00000040     ti.osal.ae674 : MuxIntcP_tirtos.oe674 (.text:MuxIntcP_create)
                  c311b580    00000040                   : RegisterIntr_tirtos.oe674 (.text:Osal_RegisterInterrupt_initParams)
                  c311b5c0    00000040     ti.csl.ae674 : spi.oe674 (.text:SPICSDisable)
                  c311b600    00000040                  : spi.oe674 (.text:SPICSEnable)
                  c311b640    00000040                  : spi.oe674 (.text:SPIClockModeSetup)
                  c311b680    00000040                  : spi.oe674 (.text:SPIDataFormatSetupSlave)
                  c311b6c0    00000040                  : spi.oe674 (.text:SPIDelaySetup)
                  c311b700    00000040                  : spi.oe674 (.text:SPIIntInit2)
                  c311b740    00000040                  : spi.oe674 (.text:SPIPinControlSetup)
                  c311b780    00000040                  : spi.oe674 (.text:SPISetShiftDir)
                  c311b7c0    00000040                  : spi.oe674 (.text:SPITransmitData)
                  c311b800    00000040     ti.osal.ae674 : SemaphoreP_tirtos.oe674 (.text:SemaphoreP_Params_init)
                  c311b840    00000040                   : SemaphoreP_tirtos.oe674 (.text:SemaphoreP_post)
                  c311b880    00000040     ti.csl.ae674 : uart.oe674 (.text:UART_breakCtl_v0)
                  c311b8c0    00000040                  : uart.oe674 (.text:UART_charGetNonBlocking_v0)
                  c311b900    00000040                  : uart.oe674 (.text:UART_divisorValCompute_v0)
                  c311b940    00000040                  : uart.oe674 (.text:UART_fIFOConfig_v0)
                  c311b980    00000040                  : uart.oe674 (.text:UART_fIFORegisterWrite_v0)
                  c311b9c0    00000040                  : uart.oe674 (.text:UART_intDisable_v0)
                  c311ba00    00000040                  : uart.oe674 (.text:UART_intEnable_v0)
                  c311ba40    00000040                  : uart.oe674 (.text:UART_intIdentityGet_v0)
                  c311ba80    00000040                  : uart.oe674 (.text:UART_loopbackModeControl_v0)
                  c311bac0    00000040     ti.drv.uart.ae674 : UART_drv.oe674 (.text:UART_open)
                  c311bb00    00000040     ti.csl.ae674 : uart.oe674 (.text:UART_readLineStatus_v0)
                  c311bb40    00000040     ti.osal.ae674 : Utils_tirtos.oe674 (.text:_DebugP_assert)
                  c311bb80    00000040     rts6740_elf.lib : frcmpyd_div.obj (.text:__TI_frcmpyd_div)
                  c311bbc0    00000040                     : assert.obj (.text:__c6xabi_abort_msg)
                  c311bc00    00000040                     : isinf.obj (.text:__c6xabi_isinf)
                  c311bc40    00000040                     : _printfi.obj (.text:__c6xabi_isnan)
                  c311bc80    00000040                     : strasg.obj (.text:__strasgi_64plus)
                  c311bcc0    00000040                     : args_main.obj (.text:_args_main)
                  c311bd00    00000040     sysbios.ae674 : c62_TaskSupport_asm.obj (.text:_ti_sysbios_family_c62_TaskSupport_buildTaskStack)
                  c311bd40    00000040     edma3_lld_drv_sample.ae674 : sample_cs.oe674 (.text:edma3OsSemGive)
                  c311bd80    00000040     spi_test_pe674.oe674 (.text:free)
                  c311bdc0    00000040     spi_test_pe674.oe674 (.text:ti_sysbios_BIOS_exitFunc__I)
                  c311be00    00000040     spi_test_pe674.oe674 (.text:ti_sysbios_BIOS_rtsLock__I)
                  c311be40    00000040     spi_test_pe674.oe674 (.text:ti_sysbios_BIOS_rtsUnlock__I)
                  c311be80    00000040     spi_test_pe674.oe674 (.text:ti_sysbios_family_c64p_Hwi_destruct)
                  c311bec0    00000040     sysbios.ae674 : BIOS.obj (.text:ti_sysbios_family_c64p_Hwi_disableInterrupt__E)
                  c311bf00    00000040                   : BIOS.obj (.text:ti_sysbios_family_c64p_Hwi_enableInterrupt__E)
                  c311bf40    00000040                   : BIOS.obj (.text:ti_sysbios_family_c64p_primus_TimerSupport_enable__E)
                  c311bf80    00000040     spi_test_pe674.oe674 (.text:ti_sysbios_gates_GateHwi_Handle__label__S)
                  c311bfc0    00000040     spi_test_pe674.oe674 (.text:ti_sysbios_gates_GateHwi_Object__delete__S)
                  c311c000    00000040     spi_test_pe674.oe674 (.text:ti_sysbios_gates_GateMutex_Handle__label__S)
                  c311c040    00000040     sysbios.ae674 : BIOS.obj (.text:ti_sysbios_gates_GateMutex_Instance_init__E)
                  c311c080    00000040                   : BIOS.obj (.text:ti_sysbios_gates_GateMutex_leave__E)
                  c311c0c0    00000040     spi_test_pe674.oe674 (.text:ti_sysbios_heaps_HeapMem_Handle__label__S)
                  c311c100    00000040     spi_test_pe674.oe674 (.text:ti_sysbios_heaps_HeapMem_Object__delete__S)
                  c311c140    00000040     spi_test_pe674.oe674 (.text:ti_sysbios_heaps_HeapMem_Object__get__S)
                  c311c180    00000040     spi_test_pe674.oe674 (.text:ti_sysbios_knl_Semaphore_destruct)
                  c311c1c0    00000040     spi_test_pe674.oe674 (.text:ti_sysbios_knl_Swi_Object__get__S)
                  c311c200    00000040     spi_test_pe674.oe674 (.text:ti_sysbios_knl_Task_Object__get__S)
                  c311c240    00000040     sysbios.ae674 : BIOS.obj (.text:ti_sysbios_knl_Task_sleepTimeout__I)
                  c311c280    00000040     ti.targets.rts6000.ae674 : Error.oe674 (.text:xdc_runtime_Error_check__E)
                  c311c2c0    00000040                              : Error.oe674 (.text:xdc_runtime_Error_init__E)
                  c311c300    00000040                              : Registry.oe674 (.text:xdc_runtime_Registry_findById__E)
                  c311c340    00000040                              : System.oe674 (.text:xdc_runtime_System_abort__E)
                  c311c380    00000040     spi_test_pe674.oe674 (.text:xdc_runtime_System_aprintf__E)
                  c311c3c0    00000040     ti.targets.rts6000.ae674 : System.oe674 (.text:xdc_runtime_System_exit__E)
                  c311c400    00000040     spi_test_pe674.oe674 (.text:xdc_runtime_System_printf__E)
                  c311c440    00000020     ti.board.ae674 : lcdkOMAPL138_pll.oe674 (.text:Board_PLLInit)
                  c311c460    00000020                    : lcdkOMAPL138_lld_init.oe674 (.text:Board_uartStdioInit)
                  c311c480    00000020     ti.osal.ae674 : EventCombinerP_tirtos.oe674 (.text:EventCombinerP_disableEvent)
                  c311c4a0    00000020                   : EventCombinerP_tirtos.oe674 (.text:EventCombinerP_dispatchPlug)
                  c311c4c0    00000020                   : EventCombinerP_tirtos.oe674 (.text:EventCombinerP_enableEvent)
                  c311c4e0    00000020                   : HwiP_tirtos.oe674 (.text:HwiP_clearInterrupt)
                  c311c500    00000020                   : HwiP_tirtos.oe674 (.text:HwiP_disable)
                  c311c520    00000020                   : HwiP_tirtos.oe674 (.text:HwiP_restore)
                  c311c540    00000020                   : MuxIntcP_tirtos.oe674 (.text:MuxIntcP_clearInEvent)
                  c311c560    00000020                   : MuxIntcP_tirtos.oe674 (.text:MuxIntcP_disableOutEvent)
                  c311c580    00000020                   : MuxIntcP_tirtos.oe674 (.text:MuxIntcP_enableOutEvent)
                  c311c5a0    00000020     ti.csl.ae674 : spi.oe674 (.text:SPIData1Setup)
                  c311c5c0    00000020                  : spi.oe674 (.text:SPIGlobalControlSetup)
                  c311c5e0    00000020                  : spi.oe674 (.text:SPIIntDisable)
                  c311c600    00000020                  : spi.oe674 (.text:SPIIntEnable)
                  c311c620    00000020                  : spi.oe674 (.text:SPIIntStatusClear)
                  c311c640    00000020                  : spi.oe674 (.text:SPIIntStatusGet)
                  c311c660    00000020                  : spi.oe674 (.text:SPILoopbackDisable)
                  c311c680    00000020                  : spi.oe674 (.text:SPILoopbackEnable)
                  c311c6a0    00000020                  : spi.oe674 (.text:SPIPwrDownDisable)
                  c311c6c0    00000020                  : spi.oe674 (.text:SPIPwrDownEnable)
                  c311c6e0    00000020                  : spi.oe674 (.text:SPIReceiveData)
                  c311c700    00000020                  : spi.oe674 (.text:SPIReset)
                  c311c720    00000020                  : spi.oe674 (.text:SPIRxFull)
                  c311c740    00000020                  : spi.oe674 (.text:SPITxEmpty)
                  c311c760    00000020                  : spi.oe674 (.text:SPIXferDisable)
                  c311c780    00000020                  : spi.oe674 (.text:SPIXferEnable)
                  c311c7a0    00000020     ti.drv.spi.ae674 : SPI_v0.oe674 (.text:SPI_DMA_doNothing_v0$0)
                  c311c7c0    00000020                      : SPI_v0.oe674 (.text:SPI_init_v0$0)
                  c311c7e0    00000020                      : SPI_v0.oe674 (.text:SPI_transferCallback_v0$0)
                  c311c800    00000020                      : SPI_v0.oe674 (.text:SPI_transferCancel_v0$0)
                  c311c820    00000020     ti.drv.uart.ae674 : UART_drv.oe674 (.text:UART_Params_init)
                  c311c840    00000020                       : UART_v0.oe674 (.text:UART_control_v0$0)
                  c311c860    00000020     ti.csl.ae674 : uart.oe674 (.text:UART_divisorLatchDisable_v0)
                  c311c880    00000020                  : uart.oe674 (.text:UART_fIFOCharPut_v0)
                  c311c8a0    00000020                  : uart.oe674 (.text:UART_fifoEmpty_v0)
                  c311c8c0    00000020     ti.drv.uart.ae674 : UART_v0.oe674 (.text:UART_init_v0$0)
                  c311c8e0    00000020     ti.csl.ae674 : uart.oe674 (.text:UART_operatingModeSelect_v0)
                  c311c900    00000020                  : uart.oe674 (.text:UART_pwremuConfig_v0)
                  c311c920    00000020     ti.drv.uart.ae674 : UART_drv.oe674 (.text:UART_write)
                  c311c940    00000020                       : UART_drv.oe674 (.text:UART_writePolling)
                  c311c960    00000020     rts6740_elf.lib : errno.obj (.text:__c6xabi_errno_addr)
                  c311c980    00000020                     : _lock.obj (.text:_nop)
                  c311c9a0    00000020                     : printf.obj (.text:_outc)
                  c311c9c0    00000020                     : printf.obj (.text:_outs)
                  c311c9e0    00000020                     : _lock.obj (.text:_register_lock)
                  c311ca00    00000020                     : _lock.obj (.text:_register_unlock)
                  c311ca20    00000020     sysbios.ae674 : c62_TaskSupport_asm.obj (.text:_ti_sysbios_family_c62_TaskSupport_glue)
                  c311ca40    00000020     rts6740_elf.lib : exit.obj (.text:abort)
                  c311ca60    00000020                     : copy_decompress_none.obj (.text:decompress:none:__TI_decompress_none)
                  c311ca80    00000020                     : copy_decompress_rle.obj (.text:decompress:rle24:__TI_decompress_rle24)
                  c311caa0    00000020     edma3_lld_drv_sample.ae674 : sample_omapl138_int_reg.oe674 (.text:disableErrorInterrupt)
                  c311cac0    00000020                                : sample_omapl138_int_reg.oe674 (.text:disableXferCompInterrupt)
                  c311cae0    00000020                                : sample_omapl138_int_reg.oe674 (.text:enableErrorInterrupt)
                  c311cb00    00000020                                : sample_omapl138_int_reg.oe674 (.text:enableXferCompInterrupt)
                  c311cb20    00000020     rts6740_elf.lib : fputc.obj (.text:putchar)
                  c311cb40    00000020     spi_test_pe674.oe674 (.text:ti_sysbios_BIOS_RtsGateProxy_enter__E)
                  c311cb60    00000020     spi_test_pe674.oe674 (.text:ti_sysbios_BIOS_RtsGateProxy_leave__E)
                  c311cb80    00000020     sysbios.ae674 : BIOS.obj (.text:ti_sysbios_BIOS_getThreadType__E)
                  c311cba0    00000020                   : BIOS.obj (.text:ti_sysbios_BIOS_linkedWithIncorrectBootLibrary__E)
                  c311cbc0    00000020     spi_test_pe674.oe674 (.text:ti_sysbios_BIOS_nullFunc__I)
                  c311cbe0    00000020     sysbios.ae674 : BIOS.obj (.text:ti_sysbios_BIOS_setThreadType__E)
                  c311cc00    00000020                   : BIOS.obj (.text:ti_sysbios_BIOS_start__E)
                  c311cc20    00000020     spi_test_pe674.oe674 (.text:ti_sysbios_family_c62_TaskSupport_Module__startupDone__S)
                  c311cc40    00000020     sysbios.ae674 : BIOS.obj (.text:ti_sysbios_family_c64p_Cache_wbInv__E)
                  c311cc60    00000020     spi_test_pe674.oe674 (.text:ti_sysbios_family_c64p_Hwi_Module__startupDone__F)
                  c311cc80    00000020     spi_test_pe674.oe674 (.text:ti_sysbios_family_c64p_Hwi_Params__init__S)
                  c311cca0    00000020     sysbios.ae674 : BIOS.obj (.text:ti_sysbios_family_c64p_Hwi_clearInterrupt__E)
                  c311ccc0    00000020                   : BIOS.obj (.text:ti_sysbios_family_c64p_Hwi_getFunc__E)
                  c311cce0    00000020                   : BIOS.obj (.text:ti_sysbios_family_c64p_Hwi_getHandle__E)
                  c311cd00    00000020                   : BIOS.obj (.text:ti_sysbios_family_c64p_Hwi_startup__E)
                  c311cd20    00000020                   : BIOS.obj (.text:ti_sysbios_family_c64p_Hwi_switchFromBootStack__E)
                  c311cd40    00000020                   : BIOS.obj (.text:ti_sysbios_family_c64p_Hwi_unPluggedInterrupt__I)
                  c311cd60    00000020                   : BIOS.obj (.text:ti_sysbios_gates_GateHwi_Instance_init__E)
                  c311cd80    00000020                   : BIOS.obj (.text:ti_sysbios_gates_GateHwi_enter__E)
                  c311cda0    00000020                   : BIOS.obj (.text:ti_sysbios_gates_GateHwi_leave__E)
                  c311cdc0    00000020                   : BIOS.obj (.text:ti_sysbios_gates_GateHwi_query__E)
                  c311cde0    00000020                   : BIOS.obj (.text:ti_sysbios_gates_GateMutex_Instance_finalize__E)
                  c311ce00    00000020                   : BIOS.obj (.text:ti_sysbios_gates_GateMutex_query__E)
                  c311ce20    00000020                   : BIOS.obj (.text:ti_sysbios_hal_Hwi_Module_startup__E)
                  c311ce40    00000020     spi_test_pe674.oe674 (.text:ti_sysbios_heaps_HeapBuf_Object__get__S)
                  c311ce60    00000020     spi_test_pe674.oe674 (.text:ti_sysbios_heaps_HeapMem_Module_GateProxy_enter__E)
                  c311ce80    00000020     spi_test_pe674.oe674 (.text:ti_sysbios_heaps_HeapMem_Module_GateProxy_leave__E)
                  c311cea0    00000020     sysbios.ae674 : BIOS.obj (.text:ti_sysbios_heaps_HeapMem_isBlocking__E)
                  c311cec0    00000020     spi_test_pe674.oe674 (.text:ti_sysbios_knl_Clock_TimerProxy_getMaxTicks__E)
                  c311cee0    00000020     sysbios.ae674 : BIOS.obj (.text:ti_sysbios_knl_Idle_loop__E)
                  c311cf00    00000020                   : BIOS.obj (.text:ti_sysbios_knl_Queue_Instance_init__E)
                  c311cf20    00000020     spi_test_pe674.oe674 (.text:ti_sysbios_knl_Queue_Object__get__S)
                  c311cf40    00000020     spi_test_pe674.oe674 (.text:ti_sysbios_knl_Queue_destruct)
                  c311cf60    00000020     sysbios.ae674 : BIOS.obj (.text:ti_sysbios_knl_Queue_empty__E)
                  c311cf80    00000020                   : BIOS.obj (.text:ti_sysbios_knl_Semaphore_Instance_finalize__E)
                  c311cfa0    00000020     spi_test_pe674.oe674 (.text:ti_sysbios_knl_Semaphore_Params__init__S)
                  c311cfc0    00000020     sysbios.ae674 : BIOS.obj (.text:ti_sysbios_knl_Swi_disable__E)
                  c311cfe0    00000020                   : BIOS.obj (.text:ti_sysbios_knl_Task_disable__E)
                  c311d000    00000020                   : BIOS.obj (.text:ti_sysbios_knl_Task_enable__E)
                  c311d020    00000020                   : BIOS.obj (.text:ti_sysbios_knl_Task_startup__E)
                  c311d040    00000020     spi_test_pe674.oe674 (.text:ti_sysbios_timers_timer64_Timer_Module__startupDone__F)
                  c311d060    00000020     sysbios.ae674 : BIOS.obj (.text:ti_sysbios_timers_timer64_Timer_getMaxTicks__E)
                  c311d080    00000020     ti.targets.rts6000.ae674 : Error.oe674 (.text:xdc_runtime_Error_getSite__E)
                  c311d0a0    00000020                              : Error.oe674 (.text:xdc_runtime_Error_raiseX__E)
                  c311d0c0    00000020                              : Gate.oe674 (.text:xdc_runtime_Gate_enterSystem__E)
                  c311d0e0    00000020                              : Gate.oe674 (.text:xdc_runtime_Gate_leaveSystem__E)
                  c311d100    00000020     spi_test_pe674.oe674 (.text:xdc_runtime_IHeap_alloc)
                  c311d120    00000020     spi_test_pe674.oe674 (.text:xdc_runtime_IHeap_free)
                  c311d140    00000020     ti.targets.rts6000.ae674 : Memory.oe674 (.text:xdc_runtime_Memory_calloc__E)
                  c311d160    00000020                              : Memory.oe674 (.text:xdc_runtime_Memory_free__E)
                  c311d180    00000020                              : Memory.oe674 (.text:xdc_runtime_Memory_getMaxDefaultTypeAlign__E)
                  c311d1a0    00000020     spi_test_pe674.oe674 (.text:xdc_runtime_Startup_exec__I)
                  c311d1c0    00000020     spi_test_pe674.oe674 (.text:xdc_runtime_Startup_reset__I)
                  c311d1e0    00000020     ti.targets.rts6000.ae674 : Startup.oe674 (.text:xdc_runtime_Startup_rtsDone__E)
                  c311d200    00000020                              : SysStd.oe674 (.text:xdc_runtime_SysStd_exit__E)
                  c311d220    00000020                              : SysStd.oe674 (.text:xdc_runtime_SysStd_putch__E)
                  c311d240    00000020                              : SysStd.oe674 (.text:xdc_runtime_SysStd_ready__E)
                  c311d260    00000020     spi_test_pe674.oe674 (.text:xdc_runtime_System_Module_GateProxy_enter__E)
                  c311d280    00000020     spi_test_pe674.oe674 (.text:xdc_runtime_System_Module_GateProxy_leave__E)
                  c311d2a0    00000020     ti.targets.rts6000.ae674 : System.oe674 (.text:xdc_runtime_System_Module_startup__E)
                  c311d2c0    00000020                              : System.oe674 (.text:xdc_runtime_System_vsnprintf__E)
                  c311d2e0    00000020                              : Text.oe674 (.text:xdc_runtime_Text_ropeText__E)
                  c311d300    00000020     spi_test_pe674.oe674 (.text:xdc_runtime_Text_visitRope__I)

.fardata.2 
*          0    c311d320    000177dc     UNINITIALIZED
                  c311d320    0000df38     edma3_lld_drv.ae674 : edma3_drv_init.oe674 (.fardata:.edma3Globals:uninit)
                  c312b258    00007998     edma3_lld_rm.ae674 : edma3resmgr.oe674 (.fardata:.edma3Globals:uninit)
                  c3132bf0    00000b40     ti.osal.ae674 : SemaphoreP_tirtos.oe674 (.fardata:gOsalSemPTiRtosPool$0)
                  c3133730    00000500                   : HwiP_tirtos.oe674 (.fardata:gOsalHwiPTiRtosPool$0)
                  c3133c30    00000400     spi_test_pe674.oe674 (.fardata:ti_sysbios_family_c64p_EventCombiner_Module__state__V)
                  c3134030    000001e0     rts6740_elf.lib : defs.obj (.fardata:_ftable)
                  c3134210    000000f0     ti.drv.uart.ae674 : UART_soc.oe674 (.fardata:uartInitCfg)
                  c3134300    000000b8     spi_test_pe674.oe674 (.fardata:ti_sysbios_knl_Task_Object__table__V)
                  c31343b8    000000a0     rts6740_elf.lib : write.obj (.fardata:_stream)
                  c3134458    000000a0     ti.drv.spi.ae674 : SPI_soc.oe674 (.fardata:spiInitCfg)
                  c31344f8    00000080     spi_test_pe674.oe674 (.fardata:ti_sysbios_knl_Swi_Module_State_0_readyQ__A)
                  c3134578    00000078     rts6740_elf.lib : write.obj (.fardata:_device)
                  c31345f0    0000006c     spi_test_pe674.oe674 (.fardata:ti_sysbios_family_c64p_Hwi_Module__state__V)
                  c313465c    00000004     rts6740_elf.lib : _lock.obj (.fardata:_unlock)
                  c3134660    00000062     edma3_lld_rm.ae674 : edma3resmgr.oe674 (.fardata:.edma3Globals:init)
                  c31346c2    00000002     spi_test_pe674.oe674 (.fardata:xdc_runtime_Error_Module__state__V)
                  c31346c4    00000004     rts6740_elf.lib : defs.obj (.fardata)
                  c31346c8    00000060     spi_test_pe674.oe674 (.fardata:ti_sysbios_timers_timer64_Timer_Module_State_0_device__A)
                  c3134728    00000050     spi_test_pe674.oe674 (.fardata:ti_sysbios_timers_timer64_Timer_Object__table__V)
                  c3134778    00000048     spi_test_pe674.oe674 (.fardata:ti_sysbios_knl_Task_Module__state__V)
                  c31347c0    00000040     edma3_lld_drv_sample.ae674 : sample_omapl138_cfg.oe674 (.fardata:ccXferCompInt)
                  c3134800    00000040                                : sample_omapl138_cfg.oe674 (.fardata:tcErrorInt)
                  c3134840    00000040     spi_test_pe674.oe674 (.fardata:ti_sysbios_gates_GateMutex_Object__table__V)
                  c3134880    00000030     spi_test_pe674.oe674 (.fardata:ti_sysbios_family_c64p_Exception_Module__state__V)
                  c31348b0    00000030     spi_test_pe674.oe674 (.fardata:ti_sysbios_knl_Swi_Object__table__V)
                  c31348e0    0000002c     ti.osal.ae674 : Utils_tirtos.oe674 (.fardata:gOsal_HwAttrs)
                  c313490c    0000002c     spi_test_pe674.oe674 (.fardata:ti_sysbios_knl_Clock_Module__state__V)
                  c3134938    00000024     spi_test_pe674.oe674 (.fardata:ti_sysbios_BIOS_Module__state__V)
                  c313495c    00000004     rts6740_elf.lib : errno.obj (.fardata)
                  c3134960    00000020     spi_test_pe674.oe674 (.fardata:ti_sysbios_knl_Task_Module_State_0_readyQ__A)
                  c3134980    00000020     spi_test_pe674.oe674 (.fardata:ti_sysbios_timers_timer64_Timer_Module_State_0_gctrl__A)
                  c31349a0    00000020     spi_test_pe674.oe674 (.fardata:ti_sysbios_timers_timer64_Timer_Module_State_0_handles__A)
                  c31349c0    00000020     spi_test_pe674.oe674 (.fardata:ti_sysbios_timers_timer64_Timer_Module_State_0_intFreqs__A)
                  c31349e0    00000020     spi_test_pe674.oe674 (.fardata:xdc_runtime_Error_IgnoreBlock)
                  c3134a00    00000020     spi_test_pe674.oe674 (.fardata:xdc_runtime_System_Module_State_0_atexitHandlers__A)
                  c3134a20    0000001c     spi_test_pe674.oe674 (.fardata:ti_sysbios_knl_Swi_Module__state__V)
                  c3134a3c    00000004     spi_test_pe674.oe674 (.fardata:ti_sysbios_family_c64p_Cache_Module__state__V)
                  c3134a40    00000018     spi_test_pe674.oe674 (.fardata:ti_sysbios_family_c64p_Hwi_Object__table__V)
                  c3134a58    00000018     spi_test_pe674.oe674 (.fardata:ti_sysbios_heaps_HeapMem_Object__table__V)
                  c3134a70    00000018     spi_test_pe674.oe674 (.fardata:ti_sysbios_timers_timer64_Timer_Module__state__V)
                  c3134a88    00000008     edma3_lld_drv_sample.ae674 : sample_omapl138_cfg.oe674 (.fardata:ccErrorInt)
                  c3134a90    00000008     spi_test_pe674.oe674 (.fardata:ti_sysbios_family_c64p_Hwi_Module__root__V)
                  c3134a98    00000008     spi_test_pe674.oe674 (.fardata:ti_sysbios_family_c64p_primus_TimerSupport_Module_State_0_suspSrc__A)
                  c3134aa0    00000008     spi_test_pe674.oe674 (.fardata:ti_sysbios_gates_GateHwi_Module__root__V)
                  c3134aa8    00000008     spi_test_pe674.oe674 (.fardata:ti_sysbios_gates_GateMutex_Module__root__V)
                  c3134ab0    00000008     spi_test_pe674.oe674 (.fardata:ti_sysbios_hal_Hwi_Object__table__V)
                  c3134ab8    00000008     spi_test_pe674.oe674 (.fardata:ti_sysbios_heaps_HeapMem_Module__root__V)
                  c3134ac0    00000008     spi_test_pe674.oe674 (.fardata:ti_sysbios_knl_Queue_Module__root__V)
                  c3134ac8    00000008     spi_test_pe674.oe674 (.fardata:ti_sysbios_knl_Semaphore_Module__root__V)
                  c3134ad0    00000008     spi_test_pe674.oe674 (.fardata:xdc_runtime_Registry_Module__state__V)
                  c3134ad8    00000008     spi_test_pe674.oe674 (.fardata:xdc_runtime_Startup_Module__state__V)
                  c3134ae0    00000008     spi_test_pe674.oe674 (.fardata:xdc_runtime_System_Module__state__V)
                  c3134ae8    00000004     spi_test_pe674.oe674 (.fardata:ti_sysbios_family_c64p_primus_TimerSupport_Module__state__V)
                  c3134aec    00000004     spi_test_pe674.oe674 (.fardata:ti_sysbios_heaps_HeapBuf_Module__state__V)
                  c3134af0    00000004     spi_test_pe674.oe674 (.fardata:ti_sysbios_gates_GateHwi_Object__table__V)
                  c3134af4    00000004     spi_test_pe674.oe674 (.fardata:xdc_runtime_Memory_Module__state__V)
                  c3134af8    00000004     spi_test_pe674.oe674 (.fardata:ti_sysbios_knl_Task_Module_State_0_idleTask__A)

.const     0    c3134b00    00002ec6     
                  c3134b00    00001954     spi_test_pe674.oe674 (.const:xdc_runtime_Text_charTab__A)
                  c3136454    00000518     sysbios.ae674 : BIOS.obj (.const:.string)
                  c313696c    0000046c     edma3_lld_rm.ae674 : edma3resmgr.oe674 (.const:.string)
                  c3136dd8    00000101     rts6740_elf.lib : ctype.obj (.const:.string:_ctypes_)
                  c3136ed9    00000001     spi_test_pe674.oe674 (.const:ti_sysbios_timers_timer64_Timer_localTimerBaseId__C)
                  c3136eda    00000002     spi_test_pe674.oe674 (.const:ti_sysbios_family_c64p_Cache_Module__id__C)
                  c3136edc    00000004     ti.targets.rts6000.ae674 : Assert.oe674 (.const:.string)
                  c3136ee0    000000f0     spi_test_pe674.oe674 (.const:xdc_runtime_Text_nodeTab__A)
                  c3136fd0    000000b0     edma3_lld_drv.ae674 : edma3_drv_basic.oe674 (.const:.string)
                  c3137080    0000008c     spi_test_pe674.oe674 (.const:.string)
                  c313710c    00000058     ti.targets.rts6000.ae674 : Error.oe674 (.const:.string)
                  c3137164    00000004     spi_test_pe674.oe674 (.const:ti_sysbios_family_c64p_Cache_EMIFA_BASE__C)
                  c3137168    00000054     ti.drv.spi.ae674 : SPI_soc.oe674 (.const:SPI_config)
                  c31371bc    00000050     main_spi_loopback_example.obj (.const:.string)
                  c313720c    00000040     ti.targets.rts6000.ae674 : Text.oe674 (.const:.string)
                  c313724c    00000040     ti.drv.uart.ae674 : UART_drv.oe674 (.const:UART_defaultParams)
                  c313728c    00000030                       : UART_v0.oe674 (.const:UART_FxnTable_v0)
                  c31372bc    00000004     spi_test_pe674.oe674 (.const:ti_sysbios_family_c64p_Cache_EMIFA_CFG__C)
                  c31372c0    00000030     ti.drv.uart.ae674 : UART_soc.oe674 (.const:UART_config)
                  c31372f0    00000030     spi_test_pe674.oe674 (.const:ti_sysbios_family_c64p_Hwi_Object__PARAMS__C)
                  c3137320    0000002c     ti.targets.rts6000.ae674 : Startup.oe674 (.const:.string)
                  c313734c    00000004     spi_test_pe674.oe674 (.const:ti_sysbios_family_c64p_Cache_EMIFA_LENGTH__C)
                  c3137350    0000002c     spi_test_pe674.oe674 (.const:xdc_runtime_Startup_sfxnTab__A)
                  c313737c    00000028     spi_test_pe674.oe674 (.const:ti_sysbios_heaps_HeapMem_Module__FXNS__C)
                  c31373a4    00000024     rts6740_elf.lib : _printfi.obj (.const:.string)
                  c31373c8    00000024     ti.drv.uart.ae674 : UART_stdio.oe674 (.const:.string)
                  c31373ec    00000024     spi_test_pe674.oe674 (.const:ti_sysbios_gates_GateHwi_Module__FXNS__C)
                  c3137410    00000024     spi_test_pe674.oe674 (.const:ti_sysbios_gates_GateMutex_Module__FXNS__C)
                  c3137434    00000024     spi_test_pe674.oe674 (.const:ti_sysbios_heaps_HeapMem_Object__PARAMS__C)
                  c3137458    00000024     spi_test_pe674.oe674 (.const:ti_sysbios_knl_Semaphore_Object__PARAMS__C)
                  c313747c    00000020     ti.drv.spi.ae674 : SPI_v0.oe674 (.const:$P$T0$1$0)
                  c313749c    00000020                      : SPI_v0.oe674 (.const:$P$T1$2$0)
                  c31374bc    00000020                      : SPI_v0.oe674 (.const:$P$T2$3$0)
                  c31374dc    00000020                      : SPI_v0.oe674 (.const:$P$T3$5$0)
                  c31374fc    00000020                      : SPI_v0.oe674 (.const:$P$T4$6$0)
                  c313751c    00000020     ti.osal.ae674 : SemaphoreP_tirtos.oe674 (.const:.string)
                  c313753c    00000020     ti.drv.spi.ae674 : SPI_drv.oe674 (.const:SPI_defaultParams)
                  c313755c    00000020     spi_test_pe674.oe674 (.const:ti_sysbios_family_c64p_Hwi_Object__DESC__C)
                  c313757c    00000020     spi_test_pe674.oe674 (.const:ti_sysbios_gates_GateHwi_Object__DESC__C)
                  c313759c    00000020     spi_test_pe674.oe674 (.const:ti_sysbios_gates_GateMutex_Object__DESC__C)
                  c31375bc    00000020     spi_test_pe674.oe674 (.const:ti_sysbios_heaps_HeapMem_Object__DESC__C)
                  c31375dc    00000020     spi_test_pe674.oe674 (.const:ti_sysbios_knl_Queue_Object__DESC__C)
                  c31375fc    00000020     spi_test_pe674.oe674 (.const:ti_sysbios_knl_Semaphore_Object__DESC__C)
                  c313761c    0000001c     ti.drv.uart.ae674 : UART_v0.oe674 (.const:.string)
                  c3137638    0000001c     ti.osal.ae674 : HwiP_tirtos.oe674 (.const:.string)
                  c3137654    0000001c     ti.drv.spi.ae674 : SPI_v0.oe674 (.const:SPI_FxnTable_v0)
                  c3137670    00000018     ti.targets.rts6000.ae674 : System.oe674 (.const:.string)
                  c3137688    00000018     spi_test_pe674.oe674 (.const:ti_sysbios_gates_GateHwi_Object__PARAMS__C)
                  c31376a0    00000018     spi_test_pe674.oe674 (.const:ti_sysbios_gates_GateMutex_Object__PARAMS__C)
                  c31376b8    00000018     spi_test_pe674.oe674 (.const:ti_sysbios_knl_Queue_Object__PARAMS__C)
                  c31376d0    00000016     spi_test_pe674.oe674 (.const:xdc_runtime_Startup_sfxnRts__A)
                  c31376e6    00000002     spi_test_pe674.oe674 (.const:ti_sysbios_family_c64p_EventCombiner_Module__id__C)
                  c31376e8    00000010     ti.drv.spi.ae674 : SPI_drv.oe674 (.const:.string)
                  c31376f8    00000010     spi_test_pe674.oe674 (.const:ti_sysbios_family_c64p_EventCombiner_EVTMASK__C)
                  c3137708    00000008     spi_test_pe674.oe674 (.const:ti_sysbios_knl_Idle_funcList__C)
                  c3137710    00000008     spi_test_pe674.oe674 (.const:xdc_runtime_Startup_firstFxns__A)
                  c3137718    00000008     spi_test_pe674.oe674 (.const:xdc_runtime_Startup_firstFxns__C)
                  c3137720    00000008     spi_test_pe674.oe674 (.const:xdc_runtime_Startup_lastFxns__C)
                  c3137728    00000004     spi_test_pe674.oe674 (.const:ti_sysbios_family_c64p_Cache_EMIFB_BASE__C)
                  c313772c    00000004     spi_test_pe674.oe674 (.const:ti_sysbios_family_c64p_Cache_EMIFB_CFG__C)
                  c3137730    00000004     spi_test_pe674.oe674 (.const:ti_sysbios_family_c64p_Cache_EMIFB_LENGTH__C)
                  c3137734    00000004     spi_test_pe674.oe674 (.const:ti_sysbios_family_c64p_Cache_EMIFC_BASE__C)
                  c3137738    00000004     spi_test_pe674.oe674 (.const:ti_sysbios_family_c64p_Cache_EMIFC_CFG__C)
                  c313773c    00000004     spi_test_pe674.oe674 (.const:ti_sysbios_family_c64p_Cache_EMIFC_LENGTH__C)
                  c3137740    00000004     spi_test_pe674.oe674 (.const:ti_sysbios_family_c64p_Cache_E_invalidL1CacheSize__C)
                  c3137744    00000004     spi_test_pe674.oe674 (.const:ti_sysbios_family_c64p_Cache_E_invalidL2CacheSize__C)
                  c3137748    00000004     spi_test_pe674.oe674 (.const:ti_sysbios_family_c64p_Cache_MAR0_31__C)
                  c313774c    00000004     spi_test_pe674.oe674 (.const:ti_sysbios_family_c64p_Cache_MAR128_159__C)
                  c3137750    00000004     spi_test_pe674.oe674 (.const:ti_sysbios_family_c64p_Cache_MAR160_191__C)
                  c3137754    00000004     spi_test_pe674.oe674 (.const:ti_sysbios_family_c64p_Cache_MAR192_223__C)
                  c3137758    00000004     spi_test_pe674.oe674 (.const:ti_sysbios_family_c64p_Cache_MAR224_255__C)
                  c313775c    00000004     spi_test_pe674.oe674 (.const:ti_sysbios_family_c64p_Cache_MAR32_63__C)
                  c3137760    00000004     spi_test_pe674.oe674 (.const:ti_sysbios_family_c64p_Cache_MAR64_95__C)
                  c3137764    00000004     spi_test_pe674.oe674 (.const:ti_sysbios_family_c64p_Cache_MAR96_127__C)
                  c3137768    00000004     spi_test_pe674.oe674 (.const:ti_sysbios_family_c64p_EventCombiner_A_invalidEventId__C)
                  c313776c    00000004     spi_test_pe674.oe674 (.const:ti_sysbios_family_c64p_EventCombiner_EVTRegs__C)
                  c3137770    00000004     spi_test_pe674.oe674 (.const:ti_sysbios_family_c64p_EventCombiner_E_unpluggedEvent__C)
                  c3137774    00000004     spi_test_pe674.oe674 (.const:ti_sysbios_family_c64p_EventCombiner_Module__diagsEnabled__C)
                  c3137778    00000004     spi_test_pe674.oe674 (.const:ti_sysbios_family_c64p_EventCombiner_Module__diagsIncluded__C)
                  c313777c    00000004     spi_test_pe674.oe674 (.const:ti_sysbios_family_c64p_EventCombiner_Module__diagsMask__C)
                  c3137780    00000004     spi_test_pe674.oe674 (.const:ti_sysbios_family_c64p_Exception_E_exceptionMax__C)
                  c3137784    00000004     spi_test_pe674.oe674 (.const:ti_sysbios_family_c64p_Exception_exceptionHook__C)
                  c3137788    00000004     spi_test_pe674.oe674 (.const:ti_sysbios_family_c64p_Exception_externalHook__C)
                  c313778c    00000004     spi_test_pe674.oe674 (.const:ti_sysbios_family_c64p_Exception_internalHook__C)
                  c3137790    00000004     spi_test_pe674.oe674 (.const:ti_sysbios_family_c64p_Exception_nmiHook__C)
                  c3137794    00000004     spi_test_pe674.oe674 (.const:ti_sysbios_family_c64p_Hwi_E_alreadyDefined__C)
                  c3137798    00000004     spi_test_pe674.oe674 (.const:ti_sysbios_family_c64p_Hwi_E_handleNotFound__C)
                  c313779c    00000004     spi_test_pe674.oe674 (.const:ti_sysbios_family_c64p_Hwi_E_invalidIntNum__C)
                  c31377a0    00000004     spi_test_pe674.oe674 (.const:ti_sysbios_family_c64p_Hwi_INTRMUX1Address__C)
                  c31377a4    00000004     spi_test_pe674.oe674 (.const:ti_sysbios_family_c64p_Hwi_LD_end__C)
                  c31377a8    00000004     spi_test_pe674.oe674 (.const:ti_sysbios_family_c64p_Hwi_LM_begin__C)
                  c31377ac    00000004     spi_test_pe674.oe674 (.const:ti_sysbios_family_c64p_Hwi_Module__diagsEnabled__C)
                  c31377b0    00000004     spi_test_pe674.oe674 (.const:ti_sysbios_family_c64p_Hwi_Module__diagsIncluded__C)
                  c31377b4    00000004     spi_test_pe674.oe674 (.const:ti_sysbios_family_c64p_Hwi_Module__diagsMask__C)
                  c31377b8    00000004     spi_test_pe674.oe674 (.const:ti_sysbios_family_c64p_Hwi_Module__loggerFxn1__C)
                  c31377bc    00000004     spi_test_pe674.oe674 (.const:ti_sysbios_family_c64p_Hwi_Module__loggerFxn8__C)
                  c31377c0    00000004     spi_test_pe674.oe674 (.const:ti_sysbios_family_c64p_Hwi_Module__loggerObj__C)
                  c31377c4    00000004     spi_test_pe674.oe674 (.const:ti_sysbios_gates_GateMutex_A_badContext__C)
                  c31377c8    00000004     spi_test_pe674.oe674 (.const:ti_sysbios_gates_GateMutex_Instance_State_sem__O)
                  c31377cc    00000004     spi_test_pe674.oe674 (.const:ti_sysbios_gates_GateMutex_Module__diagsEnabled__C)
                  c31377d0    00000004     spi_test_pe674.oe674 (.const:ti_sysbios_gates_GateMutex_Module__diagsIncluded__C)
                  c31377d4    00000004     spi_test_pe674.oe674 (.const:ti_sysbios_gates_GateMutex_Module__diagsMask__C)
                  c31377d8    00000004     spi_test_pe674.oe674 (.const:ti_sysbios_hal_Hwi_E_stackOverflow__C)
                  c31377dc    00000004     spi_test_pe674.oe674 (.const:ti_sysbios_heaps_HeapBuf_Instance_State_freeList__O)
                  c31377e0    00000004     spi_test_pe674.oe674 (.const:ti_sysbios_heaps_HeapBuf_Object__count__C)
                  c31377e4    00000004     spi_test_pe674.oe674 (.const:ti_sysbios_heaps_HeapBuf_numConstructedHeaps__C)
                  c31377e8    00000004     spi_test_pe674.oe674 (.const:ti_sysbios_heaps_HeapMem_A_align__C)
                  c31377ec    00000004     spi_test_pe674.oe674 (.const:ti_sysbios_heaps_HeapMem_A_heapSize__C)
                  c31377f0    00000004     spi_test_pe674.oe674 (.const:ti_sysbios_heaps_HeapMem_A_invalidFree__C)
                  c31377f4    00000004     spi_test_pe674.oe674 (.const:ti_sysbios_heaps_HeapMem_A_zeroBlock__C)
                  c31377f8    00000004     spi_test_pe674.oe674 (.const:ti_sysbios_heaps_HeapMem_E_memory__C)
                  c31377fc    00000004     spi_test_pe674.oe674 (.const:ti_sysbios_heaps_HeapMem_Module__diagsEnabled__C)
                  c3137800    00000004     spi_test_pe674.oe674 (.const:ti_sysbios_heaps_HeapMem_Module__diagsIncluded__C)
                  c3137804    00000004     spi_test_pe674.oe674 (.const:ti_sysbios_heaps_HeapMem_Module__diagsMask__C)
                  c3137808    00000004     spi_test_pe674.oe674 (.const:ti_sysbios_heaps_HeapMem_Module__gateObj__C)
                  c313780c    00000004     spi_test_pe674.oe674 (.const:ti_sysbios_heaps_HeapMem_Object__count__C)
                  c3137810    00000004     spi_test_pe674.oe674 (.const:ti_sysbios_heaps_HeapMem_reqAlign__C)
                  c3137814    00000004     spi_test_pe674.oe674 (.const:ti_sysbios_knl_Clock_LM_begin__C)
                  c3137818    00000004     spi_test_pe674.oe674 (.const:ti_sysbios_knl_Clock_LM_tick__C)
                  c313781c    00000004     spi_test_pe674.oe674 (.const:ti_sysbios_knl_Clock_LW_delayed__C)
                  c3137820    00000004     spi_test_pe674.oe674 (.const:ti_sysbios_knl_Clock_Module_State_clockQ__O)
                  c3137824    00000004     spi_test_pe674.oe674 (.const:ti_sysbios_knl_Clock_Module__diagsEnabled__C)
                  c3137828    00000004     spi_test_pe674.oe674 (.const:ti_sysbios_knl_Clock_Module__diagsIncluded__C)
                  c313782c    00000004     spi_test_pe674.oe674 (.const:ti_sysbios_knl_Clock_Module__diagsMask__C)
                  c3137830    00000004     spi_test_pe674.oe674 (.const:ti_sysbios_knl_Clock_Module__loggerFxn1__C)
                  c3137834    00000004     spi_test_pe674.oe674 (.const:ti_sysbios_knl_Clock_Module__loggerFxn2__C)
                  c3137838    00000004     spi_test_pe674.oe674 (.const:ti_sysbios_knl_Clock_Module__loggerObj__C)
                  c313783c    00000004     spi_test_pe674.oe674 (.const:ti_sysbios_knl_Semaphore_A_badContext__C)
                  c3137840    00000004     spi_test_pe674.oe674 (.const:ti_sysbios_knl_Idle_funcList__A)
                  c3137844    00000004     spi_test_pe674.oe674 (.const:ti_sysbios_knl_Semaphore_A_noEvents__C)
                  c3137848    00000004     spi_test_pe674.oe674 (.const:ti_sysbios_knl_Semaphore_A_overflow__C)
                  c313784c    00000004     spi_test_pe674.oe674 (.const:ti_sysbios_knl_Semaphore_A_pendTaskDisabled__C)
                  c3137850    00000004     spi_test_pe674.oe674 (.const:ti_sysbios_knl_Semaphore_Instance_State_pendQ__O)
                  c3137854    00000004     spi_test_pe674.oe674 (.const:ti_sysbios_knl_Semaphore_LM_pend__C)
                  c3137858    00000004     spi_test_pe674.oe674 (.const:ti_sysbios_knl_Semaphore_LM_post__C)
                  c313785c    00000004     spi_test_pe674.oe674 (.const:ti_sysbios_knl_Semaphore_Module__diagsEnabled__C)
                  c3137860    00000004     spi_test_pe674.oe674 (.const:ti_sysbios_knl_Semaphore_Module__diagsIncluded__C)
                  c3137864    00000004     spi_test_pe674.oe674 (.const:ti_sysbios_knl_Semaphore_Module__diagsMask__C)
                  c3137868    00000004     spi_test_pe674.oe674 (.const:ti_sysbios_knl_Semaphore_Module__loggerFxn2__C)
                  c313786c    00000004     spi_test_pe674.oe674 (.const:ti_sysbios_knl_Semaphore_Module__loggerFxn4__C)
                  c3137870    00000004     spi_test_pe674.oe674 (.const:ti_sysbios_knl_Semaphore_Module__loggerObj__C)
                  c3137874    00000004     spi_test_pe674.oe674 (.const:ti_sysbios_knl_Swi_LD_end__C)
                  c3137878    00000004     spi_test_pe674.oe674 (.const:ti_sysbios_knl_Swi_LM_begin__C)
                  c313787c    00000004     spi_test_pe674.oe674 (.const:ti_sysbios_knl_Swi_LM_post__C)
                  c3137880    00000004     spi_test_pe674.oe674 (.const:ti_sysbios_knl_Swi_Module__diagsEnabled__C)
                  c3137884    00000004     spi_test_pe674.oe674 (.const:ti_sysbios_knl_Swi_Module__diagsIncluded__C)
                  c3137888    00000004     spi_test_pe674.oe674 (.const:ti_sysbios_knl_Swi_Module__diagsMask__C)
                  c313788c    00000004     spi_test_pe674.oe674 (.const:ti_sysbios_knl_Swi_Module__loggerFxn1__C)
                  c3137890    00000004     spi_test_pe674.oe674 (.const:ti_sysbios_knl_Swi_Module__loggerFxn4__C)
                  c3137894    00000004     spi_test_pe674.oe674 (.const:ti_sysbios_knl_Swi_Module__loggerObj__C)
                  c3137898    00000004     spi_test_pe674.oe674 (.const:ti_sysbios_knl_Swi_Object__count__C)
                  c313789c    00000004     spi_test_pe674.oe674 (.const:ti_sysbios_knl_Task_A_badTimeout__C)
                  c31378a0    00000004     spi_test_pe674.oe674 (.const:ti_sysbios_knl_Task_A_sleepTaskDisabled__C)
                  c31378a4    00000004     spi_test_pe674.oe674 (.const:ti_sysbios_knl_Task_LD_block__C)
                  c31378a8    00000004     spi_test_pe674.oe674 (.const:ti_sysbios_knl_Task_LD_exit__C)
                  c31378ac    00000004     spi_test_pe674.oe674 (.const:ti_sysbios_knl_Task_LD_ready__C)
                  c31378b0    00000004     spi_test_pe674.oe674 (.const:ti_sysbios_knl_Task_LM_sleep__C)
                  c31378b4    00000004     spi_test_pe674.oe674 (.const:ti_sysbios_knl_Task_LM_switch__C)
                  c31378b8    00000004     spi_test_pe674.oe674 (.const:ti_sysbios_knl_Task_Module_State_inactiveQ__O)
                  c31378bc    00000004     spi_test_pe674.oe674 (.const:ti_sysbios_knl_Task_Module__diagsEnabled__C)
                  c31378c0    00000004     spi_test_pe674.oe674 (.const:ti_sysbios_knl_Task_Module__diagsIncluded__C)
                  c31378c4    00000004     spi_test_pe674.oe674 (.const:ti_sysbios_knl_Task_Module__diagsMask__C)
                  c31378c8    00000004     spi_test_pe674.oe674 (.const:ti_sysbios_knl_Task_Module__loggerFxn2__C)
                  c31378cc    00000004     spi_test_pe674.oe674 (.const:ti_sysbios_knl_Task_Module__loggerFxn4__C)
                  c31378d0    00000004     spi_test_pe674.oe674 (.const:ti_sysbios_knl_Task_Module__loggerObj__C)
                  c31378d4    00000004     spi_test_pe674.oe674 (.const:ti_sysbios_knl_Task_Object__count__C)
                  c31378d8    00000004     spi_test_pe674.oe674 (.const:ti_sysbios_knl_Task_allBlockedFunc__C)
                  c31378dc    00000004     spi_test_pe674.oe674 (.const:ti_sysbios_knl_Task_numConstructedTasks__C)
                  c31378e0    00000004     spi_test_pe674.oe674 (.const:ti_sysbios_timers_timer64_Timer_A_notAvailable__C)
                  c31378e4    00000004     spi_test_pe674.oe674 (.const:ti_sysbios_timers_timer64_Timer_E_cannotSupport__C)
                  c31378e8    00000004     spi_test_pe674.oe674 (.const:ti_sysbios_timers_timer64_Timer_Module__diagsEnabled__C)
                  c31378ec    00000004     spi_test_pe674.oe674 (.const:ti_sysbios_timers_timer64_Timer_Module__diagsIncluded__C)
                  c31378f0    00000004     spi_test_pe674.oe674 (.const:ti_sysbios_timers_timer64_Timer_Module__diagsMask__C)
                  c31378f4    00000004     spi_test_pe674.oe674 (.const:ti_sysbios_timers_timer64_Timer_anyMaskHigh__C)
                  c31378f8    00000004     spi_test_pe674.oe674 (.const:ti_sysbios_timers_timer64_Timer_anyMask__C)
                  c31378fc    00000004     spi_test_pe674.oe674 (.const:ti_sysbios_timers_timer64_Timer_freqDivisor__C)
                  c3137900    00000004     spi_test_pe674.oe674 (.const:ti_sysbios_timers_timer64_Timer_numLocalTimers__C)
                  c3137904    00000004     spi_test_pe674.oe674 (.const:ti_sysbios_timers_timer64_Timer_numTimerDevices__C)
                  c3137908    00000004     spi_test_pe674.oe674 (.const:xdc_runtime_Assert_E_assertFailed__C)
                  c313790c    00000004     spi_test_pe674.oe674 (.const:xdc_runtime_Core_A_initializedParams__C)
                  c3137910    00000004     spi_test_pe674.oe674 (.const:xdc_runtime_Core_Module__diagsEnabled__C)
                  c3137914    00000004     spi_test_pe674.oe674 (.const:xdc_runtime_Core_Module__diagsIncluded__C)
                  c3137918    00000004     spi_test_pe674.oe674 (.const:xdc_runtime_Core_Module__diagsMask__C)
                  c313791c    00000004     spi_test_pe674.oe674 (.const:xdc_runtime_Error_E_memory__C)
                  c3137920    00000004     spi_test_pe674.oe674 (.const:xdc_runtime_Error_Module__diagsEnabled__C)
                  c3137924    00000004     spi_test_pe674.oe674 (.const:xdc_runtime_Error_Module__diagsIncluded__C)
                  c3137928    00000004     spi_test_pe674.oe674 (.const:xdc_runtime_Error_Module__diagsMask__C)
                  c313792c    00000004     spi_test_pe674.oe674 (.const:xdc_runtime_Error_Module__loggerFxn8__C)
                  c3137930    00000004     spi_test_pe674.oe674 (.const:xdc_runtime_Error_Module__loggerObj__C)
                  c3137934    00000004     spi_test_pe674.oe674 (.const:xdc_runtime_Error_policyFxn__C)
                  c3137938    00000004     spi_test_pe674.oe674 (.const:xdc_runtime_Error_policy__C)
                  c313793c    00000004     spi_test_pe674.oe674 (.const:xdc_runtime_Error_raiseHook__C)
                  c3137940    00000004     spi_test_pe674.oe674 (.const:xdc_runtime_IGateProvider_Interface__BASE__C)
                  c3137944    00000004     spi_test_pe674.oe674 (.const:xdc_runtime_IHeap_Interface__BASE__C)
                  c3137948    00000004     spi_test_pe674.oe674 (.const:xdc_runtime_IModule_Interface__BASE__C)
                  c313794c    00000004     spi_test_pe674.oe674 (.const:xdc_runtime_Log_L_error__C)
                  c3137950    00000004     spi_test_pe674.oe674 (.const:xdc_runtime_Memory_defaultHeapInstance__C)
                  c3137954    00000004     spi_test_pe674.oe674 (.const:xdc_runtime_Startup_execImpl__C)
                  c3137958    00000004     spi_test_pe674.oe674 (.const:xdc_runtime_Startup_maxPasses__C)
                  c313795c    00000004     spi_test_pe674.oe674 (.const:xdc_runtime_Startup_sfxnRts__C)
                  c3137960    00000004     spi_test_pe674.oe674 (.const:xdc_runtime_Startup_sfxnTab__C)
                  c3137964    00000004     spi_test_pe674.oe674 (.const:xdc_runtime_System_Module__gateObj__C)
                  c3137968    00000004     spi_test_pe674.oe674 (.const:xdc_runtime_System_abortFxn__C)
                  c313796c    00000004     spi_test_pe674.oe674 (.const:xdc_runtime_System_exitFxn__C)
                  c3137970    00000004     spi_test_pe674.oe674 (.const:xdc_runtime_System_extendFxn__C)
                  c3137974    00000004     spi_test_pe674.oe674 (.const:xdc_runtime_System_maxAtexitHandlers__C)
                  c3137978    00000004     spi_test_pe674.oe674 (.const:xdc_runtime_Text_charTab__C)
                  c313797c    00000004     spi_test_pe674.oe674 (.const:xdc_runtime_Text_nameEmpty__C)
                  c3137980    00000004     spi_test_pe674.oe674 (.const:xdc_runtime_Text_nameStatic__C)
                  c3137984    00000004     spi_test_pe674.oe674 (.const:xdc_runtime_Text_nameUnknown__C)
                  c3137988    00000004     spi_test_pe674.oe674 (.const:xdc_runtime_Text_nodeTab__C)
                  c313798c    00000004     spi_test_pe674.oe674 (.const:xdc_runtime_Text_visitRopeFxn__C)
                  c3137990    00000002     spi_test_pe674.oe674 (.const:ti_sysbios_family_c64p_Exception_Module__id__C)
                  c3137992    00000002     spi_test_pe674.oe674 (.const:ti_sysbios_family_c64p_Exception_useInternalBuffer__C)
                  c3137994    00000002     spi_test_pe674.oe674 (.const:ti_sysbios_family_c64p_Hwi_Module__id__C)
                  c3137996    00000002     spi_test_pe674.oe674 (.const:ti_sysbios_family_c64p_Hwi_Module__loggerDefined__C)
                  c3137998    00000002     spi_test_pe674.oe674 (.const:ti_sysbios_gates_GateMutex_Module__id__C)
                  c313799a    00000002     spi_test_pe674.oe674 (.const:ti_sysbios_hal_Hwi_Module__id__C)
                  c313799c    00000002     spi_test_pe674.oe674 (.const:ti_sysbios_heaps_HeapMem_Module__id__C)
                  c313799e    00000002     spi_test_pe674.oe674 (.const:ti_sysbios_knl_Clock_Module__id__C)
                  c31379a0    00000002     spi_test_pe674.oe674 (.const:ti_sysbios_knl_Clock_Module__loggerDefined__C)
                  c31379a2    00000002     spi_test_pe674.oe674 (.const:ti_sysbios_knl_Semaphore_Module__id__C)
                  c31379a4    00000002     spi_test_pe674.oe674 (.const:ti_sysbios_knl_Semaphore_Module__loggerDefined__C)
                  c31379a6    00000002     spi_test_pe674.oe674 (.const:ti_sysbios_knl_Swi_Module__id__C)
                  c31379a8    00000002     spi_test_pe674.oe674 (.const:ti_sysbios_knl_Swi_Module__loggerDefined__C)
                  c31379aa    00000002     spi_test_pe674.oe674 (.const:ti_sysbios_knl_Task_Module__id__C)
                  c31379ac    00000002     spi_test_pe674.oe674 (.const:ti_sysbios_knl_Task_Module__loggerDefined__C)
                  c31379ae    00000002     spi_test_pe674.oe674 (.const:ti_sysbios_timers_timer64_Timer_Module__id__C)
                  c31379b0    00000002     spi_test_pe674.oe674 (.const:ti_sysbios_timers_timer64_Timer_startupNeeded__C)
                  c31379b2    00000002     spi_test_pe674.oe674 (.const:ti_sysbios_timers_timer64_Timer_useTimer64pRegMap__C)
                  c31379b4    00000002     spi_test_pe674.oe674 (.const:xdc_runtime_Core_Module__id__C)
                  c31379b6    00000002     spi_test_pe674.oe674 (.const:xdc_runtime_Error_Module__loggerDefined__C)
                  c31379b8    00000002     spi_test_pe674.oe674 (.const:xdc_runtime_Error_maxDepth__C)
                  c31379ba    00000002     spi_test_pe674.oe674 (.const:xdc_runtime_Main_Module__id__C)
                  c31379bc    00000002     spi_test_pe674.oe674 (.const:xdc_runtime_Memory_Module__id__C)
                  c31379be    00000002     spi_test_pe674.oe674 (.const:xdc_runtime_Text_charCnt__C)
                  c31379c0    00000002     spi_test_pe674.oe674 (.const:xdc_runtime_Text_isLoaded__C)
                  c31379c2    00000002     spi_test_pe674.oe674 (.const:xdc_runtime_Text_registryModsLastId__C)
                  c31379c4    00000002     spi_test_pe674.oe674 (.const:xdc_runtime_Text_unnamedModsLastId__C)

.cio       0    c31389c8    00000120     UNINITIALIZED
                  c31389c8    00000120     rts6740_elf.lib : trgmsg.obj (.cio)

.switch    0    c3138ae8    000000e0     
                  c3138ae8    00000038     rts6740_elf.lib : _printfi.obj (.switch:__TI_printfi)
                  c3138b20    00000024     ti.drv.uart.ae674 : UART_stdio.oe674 (.switch:UART_printf)
                  c3138b44    00000018     ti.drv.spi.ae674 : SPI_v0.oe674 (.switch:SPI_control_v0$0)
                  c3138b5c    00000014     ti.drv.uart.ae674 : UART_v0.oe674 (.switch:UART_open_v0$0)
                  c3138b70    00000014     edma3_lld_drv_sample.ae674 : sample_cs.oe674 (.switch:edma3OsProtectEntry)
                  c3138b84    00000014                                : sample_cs.oe674 (.switch:edma3OsProtectExit)
                  c3138b98    00000010     edma3_lld_rm.ae674 : edma3resmgr.oe674 (.switch:EDMA3_RM_allocResource)
                  c3138ba8    00000010                        : edma3resmgr.oe674 (.switch:EDMA3_RM_freeResource)
                  c3138bb8    00000010     ti.drv.spi.ae674 : SPI_v0.oe674 (.switch:SPI_open_v0$0)

MODULE SUMMARY

       Module                          code     ro data   rw data
       ------                          ----     -------   -------
    .\
       main_spi_loopback_example.obj   544      80        0      
    +--+-------------------------------+--------+---------+---------+
       Total:                          544      80        0      
                                                                 
    D:\Bhargavi_TVWS\spiInterrupt\Debug\configPkg\package\cfg\
       spi_test_pe674.oe674            4416     8161      1462562
    +--+-------------------------------+--------+---------+---------+
       Total:                          4416     8161      1462562
                                                                 
    C:\ti\bios_6_73_00_12\packages\ti\targets\rts6000\lib\boot.ae674
       autoinit.oe674                  288      0         0      
       boot.oe674                      160      0         0      
    +--+-------------------------------+--------+---------+---------+
       Total:                          448      0         0      
                                                                 
    C:\ti\bios_6_73_00_12\packages\ti\targets\rts6000\lib\ti.targets.rts6000.ae674
       System.oe674                    3232     24        0      
       Text.oe674                      1824     64        0      
       Error.oe674                     1152     88        0      
       Startup.oe674                   896      44        0      
       Core-mem.oe674                  896      0         0      
       Memory.oe674                    448      0         0      
       Core-smem.oe674                 416      0         0      
       SysStd.oe674                    224      0         0      
       Assert.oe674                    192      4         0      
       Core-params.oe674               160      0         0      
       Core-label.oe674                128      0         0      
       Gate.oe674                      64       0         0      
       Registry.oe674                  64       0         0      
    +--+-------------------------------+--------+---------+---------+
       Total:                          9696     224       0      
                                                                 
    C:\ti\edma3_lld_2_12_05_30C\packages\ti\sdo\edma3\drv\lib\674\release\edma3_lld_drv.ae674
       edma3_drv_init.oe674            0        0         57144  
       edma3_drv_basic.oe674           6208     176       0      
       edma3_drv_adv.oe674             1600     0         0      
    +--+-------------------------------+--------+---------+---------+
       Total:                          7808     176       57144  
                                                                 
    C:\ti\edma3_lld_2_12_05_30C\packages\ti\sdo\edma3\drv\sample\lib\omapl138-evm\674\release\edma3_lld_drv_sample.ae674
       sample_cs.oe674                 480      40        0      
       sample_omapl138_cfg.oe674       0        0         136    
       sample_omapl138_int_reg.oe674   128      0         0      
       sample_init.oe674               0        0         4      
    +--+-------------------------------+--------+---------+---------+
       Total:                          608      40        140    
                                                                 
    C:\ti\edma3_lld_2_12_05_30C\packages\ti\sdo\edma3\rm\lib\omapl138-evm\674\release\edma3_lld_rm.ae674
       edma3resmgr.oe674               5312     1164      31346  
    +--+-------------------------------+--------+---------+---------+
       Total:                          5312     1164      31346  
                                                                 
    C:\ti_old_pdk\ccv8\ccsv8\tools\compiler\ti-cgt-c6000_8.2.4\lib\rts6740_elf.lib
       _printfi.obj                    13504    92        0      
       divd.obj                        1472     0         0      
       fputs.obj                       992      0         0      
       defs.obj                        0        0         804    
       imath64.obj                     704      0         0      
       fputc.obj                       576      0         0      
       setvbuf.obj                     544      0         0      
       fflush.obj                      512      0         0      
       trgmsg.obj                      224      0         288    
       frexp.obj                       448      0         0      
       getdevice.obj                   448      0         0      
       imath40.obj                     448      0         0      
       hostrename.obj                  416      0         0      
       ldexp.obj                       384      0         0      
       write.obj                       96       0         280    
       fclose.obj                      320      0         0      
       copy_decompress_rle.obj         288      0         0      
       fseek.obj                       288      0         0      
       printf.obj                      288      0         0      
       exit.obj                        256      0         12     
       ctype.obj                       0        257       0      
       _io_perm.obj                    256      0         0      
       atoi.obj                        256      0         0      
       hostopen.obj                    224      0         8      
       close.obj                       224      0         0      
       hostlseek.obj                   224      0         0      
       hostwrite.obj                   224      0         0      
       llshift.obj                     224      0         0      
       ltoa.obj                        224      0         0      
       memset.obj                      224      0         0      
       divu.obj                        192      0         0      
       hostread.obj                    192      0         0      
       hostunlink.obj                  192      0         0      
       tls.obj                         192      0         0      
       fopen.obj                       160      0         0      
       hostclose.obj                   160      0         0      
       memcpy64.obj                    160      0         0      
       remu.obj                        160      0         0      
       unlink.obj                      128      0         0      
       _lock.obj                       96       0         8      
       lseek.obj                       96       0         0      
       memccpy.obj                     96       0         0      
       args_main.obj                   64       0         0      
       assert.obj                      64       0         0      
       frcmpyd_div.obj                 64       0         0      
       isinf.obj                       64       0         0      
       strasg.obj                      64       0         0      
       errno.obj                       32       0         4      
       copy_decompress_none.obj        32       0         0      
    +--+-------------------------------+--------+---------+---------+
       Total:                          26496    349       1404   
                                                                 
    C:\ti_old_pdk\pdk_omapl138_1_0_5\packages\ti\board\lib\lcdkOMAPL138\c674\release\ti.board.ae674
       lcdkOMAPL138_clock.oe674        1440     0         0      
       lcdkOMAPL138_pll.oe674          1440     0         0      
       lcdkOMAPL138_pinmux.oe674       1408     0         0      
       lcdkOMAPL138_ddr.oe674          384      0         0      
       lcdkOMAPL138.oe674              352      0         0      
       lcdkOMAPL138_lld_init.oe674     32       0         0      
    +--+-------------------------------+--------+---------+---------+
       Total:                          5056     0         0      
                                                                 
    C:\ti_old_pdk\pdk_omapl138_1_0_5\packages\ti\csl\lib\omapl138\c674\release\ti.csl.ae674
       uart.oe674                      1216     0         0      
       spi.oe674                       1184     0         0      
    +--+-------------------------------+--------+---------+---------+
       Total:                          2400     0         0      
                                                                 
    C:\ti_old_pdk\pdk_omapl138_1_0_5\packages\ti\drv\spi\lib\omapl138\c674\release\ti.drv.spi.ae674
       SPI_v0.oe674                    6848     228       4      
       SPI_drv.oe674                   704      48        8      
       SPI_soc.oe674                   192      84        312    
    +--+-------------------------------+--------+---------+---------+
       Total:                          7744     360       324    
                                                                 
    C:\ti_old_pdk\pdk_omapl138_1_0_5\packages\ti\drv\uart\lib\omapl138\c674\release\ti.drv.uart.ae674
       UART_v0.oe674                   7296     96        0      
       UART_stdio.oe674                2336     72        8      
       UART_soc.oe674                  0        48        648    
       UART_drv.oe674                  320      64        4      
    +--+-------------------------------+--------+---------+---------+
       Total:                          9952     280       660    
                                                                 
    C:\ti_old_pdk\pdk_omapl138_1_0_5\packages\ti\osal\lib\tirtos\omapl138\c674\release\ti.osal.ae674
       SemaphoreP_tirtos.oe674         832      32        2880   
       HwiP_tirtos.oe674               672      28        1280   
       RegisterIntr_tirtos.oe674       672      0         0      
       EventCombinerP_tirtos.oe674     608      0         0      
       Utils_tirtos.oe674              448      0         68     
       MuxIntcP_tirtos.oe674           160      0         0      
    +--+-------------------------------+--------+---------+---------+
       Total:                          3392     60        4228   
                                                                 
    D:\Bhargavi_TVWS\spiInterrupt\src\sysbios\sysbios.ae674
       BIOS.obj                        31648    1304      0      
       c64p_Hwi_disp_always.obj        512      0         0      
       c64p_Exception_asm.obj          384      0         0      
       c62_TaskSupport_asm.obj         224      0         0      
       c64p_Hwi_asm_switch.obj         192      0         0      
       c64p_Hwi_asm.obj                160      0         0      
    +--+-------------------------------+--------+---------+---------+
       Total:                          33120    1304      0      
                                                                 
       Stack:                          0        0         4096   
       Linker Generated:               0        2363      0      
    +--+-------------------------------+--------+---------+---------+
       Grand Total:                    116992   14561     1561904


LINKER GENERATED COPY TABLES

__TI_cinit_table @ c3139710 records: 6, size/record: 8, table size: 48
	.fardata.2: load addr=c3138e00, load size=000008bd bytes, run addr=c311d320, run size=000177dc bytes, compression=rle
	.neardata: load addr=c31396bd, load size=00000012 bytes, run addr=c3138bcc, run size=00000028 bytes, compression=rle
	.fardata.1: load addr=c31396cf, load size=00000011 bytes, run addr=c3100c10, run size=00000010 bytes, compression=rle
	.far: load addr=c31396e0, load size=0000000d bytes, run addr=c3000000, run size=00100c10 bytes, compression=rle
	systemHeap: load addr=c31396ed, load size=0000000d bytes, run addr=11700000, run size=00064000 bytes, compression=rle
	.bss: load addr=c31396fa, load size=00000009 bytes, run addr=c3138bc8, run size=00000004 bytes, compression=rle


LINKER GENERATED HANDLER TABLE

__TI_handler_table @ c3139704 records: 2, size/record: 4, table size: 8
	index: 0, handler: __TI_decompress_rle24
	index: 1, handler: __TI_decompress_none


GLOBAL SYMBOLS: SORTED ALPHABETICALLY BY Name 

address   name                                                                
-------   ----                                                                
c310cd00  Board_CorePLLConfig                                                 
c3113680  Board_DDR3Init                                                      
c310dda0  Board_DDRPLLConfig                                                  
c311c440  Board_PLLInit                                                       
c31154c0  Board_configEmifPinMux                                              
c3114400  Board_init                                                          
c3110680  Board_initSPI                                                       
c310f920  Board_moduleClockEnable                                             
c3115ca0  Board_moduleClockInit                                               
c3111900  Board_moduleClockSyncReset                                          
c310a240  Board_pinmuxConfig                                                  
c311c460  Board_uartStdioInit                                                 
c311ca40  C$$EXIT                                                             
c311ab78  C$$IO$$                                                             
c3115da0  EDMA3_DRV_clearErrorBits                                            
c310cfe0  EDMA3_DRV_disableTransfer                                           
c310e820  EDMA3_DRV_enableTransfer                                            
c310c6c0  EDMA3_DRV_freeChannel                                               
c3113800  EDMA3_DRV_getPaRAM                                                  
c3116aa0  EDMA3_DRV_getPaRAMPhyAddr                                           
c3112260  EDMA3_DRV_linkChannel                                               
c3103540  EDMA3_DRV_requestChannel                                            
c3114980  EDMA3_DRV_setPaRAM                                                  
c3116b80  EDMA3_DRV_unlinkChannel                                             
c3102900  EDMA3_RM_allocResource                                              
c310a6a0  EDMA3_RM_freeResource                                               
c3113980  EDMA3_RM_registerTccCb                                              
c3113b00  EDMA3_RM_unregisterTccCb                                            
c3115ea0  EventCombinerP_GroupRegisterInt                                     
c311c480  EventCombinerP_disableEvent                                         
c311c4a0  EventCombinerP_dispatchPlug                                         
c311c4c0  EventCombinerP_enableEvent                                          
c31195c0  EventCombinerP_getHwi                                               
c3119640  EventCombinerP_getIntNum                                            
c3118640  HOSTclose                                                           
c3116c60  HOSTlseek                                                           
c3116d40  HOSTopen                                                            
c3117980  HOSTread                                                            
c3112b20  HOSTrename                                                          
c3117a40  HOSTunlink                                                          
c3116e20  HOSTwrite                                                           
c311c4e0  HwiP_clearInterrupt                                                 
c3111ae0  HwiP_create                                                         
c311a4c0  HwiP_delete                                                         
c311c500  HwiP_disable                                                        
c311c520  HwiP_restore                                                        
c3116f00  MCSPI_init                                                          
c311c540  MuxIntcP_clearInEvent                                               
c311b540  MuxIntcP_create                                                     
c311c560  MuxIntcP_disableOutEvent                                            
c311c580  MuxIntcP_enableOutEvent                                             
c311a520  Osal_ClearInterrupt                                                 
c31186e0  Osal_DeleteInterrupt                                                
c3114560  Osal_RegisterInterrupt                                              
c311b580  Osal_RegisterInterrupt_initParams                                   
c3117b00  Osal_delay                                                          
c311a580  Osal_getHwAttrs                                                     
c311a5e0  Osal_getThreadType                                                  
c311b5c0  SPICSDisable                                                        
c311b600  SPICSEnable                                                         
c311b640  SPIClockModeSetup                                                   
c311c5a0  SPIData1Setup                                                       
c311a640  SPIDataFormatSetup                                                  
c311b680  SPIDataFormatSetupSlave                                             
c311b6c0  SPIDelaySetup                                                       
c311c5c0  SPIGlobalControlSetup                                               
c311c5e0  SPIIntDisable                                                       
c311c600  SPIIntEnable                                                        
c311b700  SPIIntInit2                                                         
c311c620  SPIIntStatusClear                                                   
c311c640  SPIIntStatusGet                                                     
c311c660  SPILoopbackDisable                                                  
c311c680  SPILoopbackEnable                                                   
c311b740  SPIPinControlSetup                                                  
c311c6a0  SPIPwrDownDisable                                                   
c311c6c0  SPIPwrDownEnable                                                    
c311c6e0  SPIReceiveData                                                      
c311c700  SPIReset                                                            
c311c720  SPIRxFull                                                           
c311b780  SPISetShiftDir                                                      
c311b7c0  SPITransmitData                                                     
c311c740  SPITxEmpty                                                          
c311c760  SPIXferDisable                                                      
c311c780  SPIXferEnable                                                       
c3137654  SPI_FxnTable_v0                                                     
c311a6a0  SPI_Params_init                                                     
c3137168  SPI_config                                                          
c311a700  SPI_control                                                         
c313753c  SPI_defaultParams                                                   
c3116f00  SPI_init                                                            
c3117bc0  SPI_open                                                            
c311a760  SPI_socGetInitCfg                                                   
c311a7c0  SPI_socSetInitCfg                                                   
c311a820  SPI_transfer                                                        
c311b800  SemaphoreP_Params_init                                              
c3110f00  SemaphoreP_create                                                   
c311a880  SemaphoreP_delete                                                   
c311a8e0  SemaphoreP_pend                                                     
c311b840  SemaphoreP_post                                                     
c311b840  SemaphoreP_postFromClock                                            
c311b840  SemaphoreP_postFromISR                                              
c3100ad8  SpiObjects                                                          
c313728c  UART_FxnTable_v0                                                    
c311c820  UART_Params_init                                                    
c311b880  UART_breakCtl_v0                                                    
c311b8c0  UART_charGetNonBlocking_v0                                          
c31196c0  UART_charPut_v0                                                     
c31372c0  UART_config                                                         
c313724c  UART_defaultParams                                                  
c311c860  UART_divisorLatchDisable_v0                                         
c311a940  UART_divisorLatchWrite_v0                                           
c311b900  UART_divisorValCompute_v0                                           
c311c880  UART_fIFOCharPut_v0                                                 
c311b940  UART_fIFOConfig_v0                                                  
c311b980  UART_fIFORegisterWrite_v0                                           
c311c8a0  UART_fifoEmpty_v0                                                   
c311a9a0  UART_fifoWait_v0                                                    
c3118820  UART_init                                                           
c311b9c0  UART_intDisable_v0                                                  
c311ba00  UART_intEnable_v0                                                   
c311ba40  UART_intIdentityGet_v0                                              
c311aa00  UART_lineCharacConfig_v0                                            
c311ba80  UART_loopbackModeControl_v0                                         
c311bac0  UART_open                                                           
c311c8e0  UART_operatingModeSelect_v0                                         
c3107540  UART_printf                                                         
c311b3c0  UART_putc                                                           
c311c900  UART_pwremuConfig_v0                                                
c311bb00  UART_readLineStatus_v0                                              
c31188c0  UART_stdioInit                                                      
c311c920  UART_write                                                          
c311c940  UART_writePolling                                                   
c3100800  UartObjects                                                         
c311bb40  _DebugP_assert                                                      
c3000000  __ASM__                                                             
c31389c8  __CIOBUF_                                                           
c3000058  __ISA__                                                             
c3000070  __PLAT__                                                            
c3000098  __TARG__                                                            
c3139710  __TI_CINIT_Base                                                     
c3139740  __TI_CINIT_Limit                                                    
c3139704  __TI_Handler_Table_Base                                             
c313970c  __TI_Handler_Table_Limit                                            
UNDEFED   __TI_INITARRAY_Base                                                 
UNDEFED   __TI_INITARRAY_Limit                                                
c31389c8  __TI_STACK_END                                                      
00001000  __TI_STACK_SIZE                                                     
c3138bc8  __TI_STATIC_BASE                                                    
UNDEFED   __TI_TLS_INIT_Base                                                  
UNDEFED   __TI_TLS_INIT_Limit                                                 
c3118aa0  __TI_cleanup                                                        
c3100c10  __TI_cleanup_ptr                                                    
c3114ac0  __TI_closefile                                                      
c311ca60  __TI_decompress_none                                                
c311ca80  __TI_decompress_rle24                                               
c3117e00  __TI_doflush                                                        
c3100c14  __TI_dtors_ptr                                                      
c3100c18  __TI_enable_exit_profile_output                                     
c311bb80  __TI_frcmpyd_div                                                    
c31346c4  __TI_ft_end                                                         
ffffffff  __TI_pprof_out_hndl                                                 
c3100c20  __TI_printfi                                                        
ffffffff  __TI_prof_data_size                                                 
ffffffff  __TI_prof_data_start                                                
c3119740  __TI_readmsg                                                        
c3118400  __TI_tls_init                                                       
c3100998  __TI_tmpnams                                                        
c311ab20  __TI_writemsg                                                       
c31162a0  __TI_wrt_ok                                                         
c30000c0  __TRDR__                                                            
ffffffff  __binit__                                                           
c311bbc0  __c6xabi_abort_msg                                                  
c3108800  __c6xabi_divd                                                       
c3117ec0  __c6xabi_divu                                                       
c3112420  __c6xabi_divul                                                      
c310efa0  __c6xabi_divull                                                     
c311c960  __c6xabi_errno_addr                                                 
c311bc00  __c6xabi_isinf                                                      
c31197c0  __c6xabi_llshl                                                      
c311ab80  __c6xabi_llshru                                                     
c3118b40  __c6xabi_remu                                                       
c311bc80  __c6xabi_strasgi_64plus                                             
ffffffff  __c_args__                                                          
c3117ec0  __divu                                                              
c313495c  __errno                                                             
c3118b40  __remu                                                              
c311bc80  __strasgi_64plus                                                    
c311bcc0  _args_main                                                          
00000000  _argsize                                                            
c3115820  _auto_init_elf                                                      
c3118be0  _c_int00                                                            
c3136dd8  _ctypes_                                                            
c3134578  _device                                                             
c3134030  _ftable                                                             
c3100c1c  _lock                                                               
c311c980  _nop                                                                
c311c9e0  _register_lock                                                      
c311ca00  _register_unlock                                                    
c31379c8  _stack                                                              
c31343b8  _stream                                                             
c311abe0  _subcull                                                            
c313465c  _unlock                                                             
c311ca40  abort                                                               
c31163a0  atoi                                                                
ffffffff  binit                                                               
c3134a88  ccErrorInt                                                          
c31347c0  ccXferCompInt                                                       
c3117280  close                                                               
c311caa0  disableErrorInterrupt                                               
c311cac0  disableXferCompInterrupt                                            
c311e198  drvInstance                                                         
c311d320  drvObj                                                              
c3138bc8  dsp_num                                                             
c3122978  edma3DrvChBoundRes                                                  
c3118040  edma3MemZero                                                        
c313467c  edma3NumPaRAMSets                                                   
c3118100  edma3OsProtectEntry                                                 
c31198c0  edma3OsProtectExit                                                  
c311bd40  edma3OsSemGive                                                      
c311ad00  edma3OsSemTake                                                      
c3119940  edma3ParamCpy                                                       
c3100b70  edma3_dma_ch_max_val                                                
c3100b88  edma3_link_ch_max_val                                               
c3100ba0  edma3_link_ch_min_val                                               
c3100bb8  edma3_log_ch_max_val                                                
c3100bd0  edma3_qdma_ch_max_val                                               
c3100be8  edma3_qdma_ch_min_val                                               
c311cae0  enableErrorInterrupt                                                
c311cb00  enableXferCompInterrupt                                             
c313495c  errno                                                               
c3117360  exit                                                                
c3114c00  fflush                                                              
c31199c0  finddevice                                                          
c3110460  fputc                                                               
c310bfa0  fputs                                                               
c311bd80  free                                                                
c31125e0  frexp                                                               
c31125e0  frexpl                                                              
c3115940  fseek                                                               
c3138bdc  gOsalHwiAllocCnt                                                    
c3138be0  gOsalHwiPeak                                                        
c3138bcc  gOsalSemAllocCnt                                                    
c3138bd0  gOsalSemPeak                                                        
c3138bd4  gOsalTimerAllocCnt                                                  
c3138bd8  gOsalTimerPeak                                                      
c31348e0  gOsal_HwAttrs                                                       
c3114d40  getdevice                                                           
c3113c80  ldexp                                                               
c3113c80  ldexpl                                                              
c311ad60  lseek                                                               
c3117440  ltoa                                                                
c3110888  main                                                                
c311a0c0  malloc                                                              
c311adc0  memccpy                                                             
c3118d20  memcpy                                                              
c3117520  memset                                                              
c3100c00  parmbuf                                                             
c3117600  printf                                                              
c3110460  putc                                                                
c311cb20  putchar                                                             
c311a140  remove                                                              
c312b258  resMgrObj                                                           
c31108a0  setvbuf                                                             
c3134458  spiInitCfg                                                          
c31106b0  spi_test                                                            
c3134800  tcErrorInt                                                          
c3134938  ti_sysbios_BIOS_Module__state__V                                    
c311c000  ti_sysbios_BIOS_RtsGateProxy_Handle__label__S                       
c311cb40  ti_sysbios_BIOS_RtsGateProxy_enter__E                               
c311cb60  ti_sysbios_BIOS_RtsGateProxy_leave__E                               
c311ce00  ti_sysbios_BIOS_RtsGateProxy_query__E                               
c3119a40  ti_sysbios_BIOS_atExitFunc__I                                       
c311ae20  ti_sysbios_BIOS_errorRaiseHook__I                                   
c311bdc0  ti_sysbios_BIOS_exitFunc__I                                         
c311cb80  ti_sysbios_BIOS_getThreadType__E                                    
c311cba0  ti_sysbios_BIOS_linkedWithIncorrectBootLibrary__E                   
c311cbc0  ti_sysbios_BIOS_nullFunc__I                                         
c3119ac0  ti_sysbios_BIOS_registerRTSLock__I                                  
c311ae80  ti_sysbios_BIOS_removeRTSLock__I                                    
c311be00  ti_sysbios_BIOS_rtsLock__I                                          
c311be40  ti_sysbios_BIOS_rtsUnlock__I                                        
c311cbe0  ti_sysbios_BIOS_setThreadType__E                                    
c311aee0  ti_sysbios_BIOS_startFunc__I                                        
c311cc00  ti_sysbios_BIOS_start__E                                            
c311cc20  ti_sysbios_family_c62_TaskSupport_Module__startupDone__S            
c311bd00  ti_sysbios_family_c62_TaskSupport_buildTaskStack                    
c311ca20  ti_sysbios_family_c62_TaskSupport_glue                              
c311af40  ti_sysbios_family_c62_TaskSupport_start__E                          
c3119840  ti_sysbios_family_c62_TaskSupport_swap__E                           
c3137164  ti_sysbios_family_c64p_Cache_EMIFA_BASE__C                          
c31372bc  ti_sysbios_family_c64p_Cache_EMIFA_CFG__C                           
c313734c  ti_sysbios_family_c64p_Cache_EMIFA_LENGTH__C                        
c3137728  ti_sysbios_family_c64p_Cache_EMIFB_BASE__C                          
c313772c  ti_sysbios_family_c64p_Cache_EMIFB_CFG__C                           
c3137730  ti_sysbios_family_c64p_Cache_EMIFB_LENGTH__C                        
c3137734  ti_sysbios_family_c64p_Cache_EMIFC_BASE__C                          
c3137738  ti_sysbios_family_c64p_Cache_EMIFC_CFG__C                           
c313773c  ti_sysbios_family_c64p_Cache_EMIFC_LENGTH__C                        
c3137740  ti_sysbios_family_c64p_Cache_E_invalidL1CacheSize__C                
c3137744  ti_sysbios_family_c64p_Cache_E_invalidL2CacheSize__C                
c3137748  ti_sysbios_family_c64p_Cache_MAR0_31__C                             
c313774c  ti_sysbios_family_c64p_Cache_MAR128_159__C                          
c3137750  ti_sysbios_family_c64p_Cache_MAR160_191__C                          
c3137754  ti_sysbios_family_c64p_Cache_MAR192_223__C                          
c3137758  ti_sysbios_family_c64p_Cache_MAR224_255__C                          
c313775c  ti_sysbios_family_c64p_Cache_MAR32_63__C                            
c3137760  ti_sysbios_family_c64p_Cache_MAR64_95__C                            
c3137764  ti_sysbios_family_c64p_Cache_MAR96_127__C                           
c3136eda  ti_sysbios_family_c64p_Cache_Module__id__C                          
c3134a3c  ti_sysbios_family_c64p_Cache_Module__state__V                       
c3107b80  ti_sysbios_family_c64p_Cache_Module_startup__E                      
c310f200  ti_sysbios_family_c64p_Cache_block__I                               
c3119b40  ti_sysbios_family_c64p_Cache_invL1pAll__E                           
00008000  ti_sysbios_family_c64p_Cache_l1dSize                                
00008000  ti_sysbios_family_c64p_Cache_l1pSize                                
00000000  ti_sysbios_family_c64p_Cache_l2Size                                 
c311afa0  ti_sysbios_family_c64p_Cache_setMar__E                              
c311cc40  ti_sysbios_family_c64p_Cache_wbInv__E                               
c3137768  ti_sysbios_family_c64p_EventCombiner_A_invalidEventId__C            
c31376f8  ti_sysbios_family_c64p_EventCombiner_EVTMASK__C                     
c313776c  ti_sysbios_family_c64p_EventCombiner_EVTRegs__C                     
c3137770  ti_sysbios_family_c64p_EventCombiner_E_unpluggedEvent__C            
c3137774  ti_sysbios_family_c64p_EventCombiner_Module__diagsEnabled__C        
c3137778  ti_sysbios_family_c64p_EventCombiner_Module__diagsIncluded__C       
c313777c  ti_sysbios_family_c64p_EventCombiner_Module__diagsMask__C           
c31376e6  ti_sysbios_family_c64p_EventCombiner_Module__id__C                  
c3133c30  ti_sysbios_family_c64p_EventCombiner_Module__state__V               
c311b000  ti_sysbios_family_c64p_EventCombiner_Module_startup__E              
c3112e60  ti_sysbios_family_c64p_EventCombiner_disableEvent__E                
c31127a0  ti_sysbios_family_c64p_EventCombiner_dispatchPlug__E                
c310fb60  ti_sysbios_family_c64p_EventCombiner_dispatch__E                    
c3113000  ti_sysbios_family_c64p_EventCombiner_enableEvent__E                 
c311b060  ti_sysbios_family_c64p_EventCombiner_unused__E                      
c3137780  ti_sysbios_family_c64p_Exception_E_exceptionMax__C                  
c3137990  ti_sysbios_family_c64p_Exception_Module__id__C                      
c3134880  ti_sysbios_family_c64p_Exception_Module__state__V                   
c3118dc0  ti_sysbios_family_c64p_Exception_Module_startup__E                  
c3113e00  ti_sysbios_family_c64p_Exception_dispatch__E                        
c3137784  ti_sysbios_family_c64p_Exception_exceptionHook__C                   
c3137788  ti_sysbios_family_c64p_Exception_externalHook__C                    
c3105220  ti_sysbios_family_c64p_Exception_handler__I                         
c310fda0  ti_sysbios_family_c64p_Exception_internalHandler__I                 
c313778c  ti_sysbios_family_c64p_Exception_internalHook__C                    
c3137790  ti_sysbios_family_c64p_Exception_nmiHook__C                         
c3137992  ti_sysbios_family_c64p_Exception_useInternalBuffer__C               
c3138c00  ti_sysbios_family_c64p_Hwi0                                         
c3137794  ti_sysbios_family_c64p_Hwi_E_alreadyDefined__C                      
c3137798  ti_sysbios_family_c64p_Hwi_E_handleNotFound__C                      
c313779c  ti_sysbios_family_c64p_Hwi_E_invalidIntNum__C                       
c31377a0  ti_sysbios_family_c64p_Hwi_INTRMUX1Address__C                       
c31164a0  ti_sysbios_family_c64p_Hwi_Instance_finalize__E                     
c3115a60  ti_sysbios_family_c64p_Hwi_Instance_init__E                         
c31377a4  ti_sysbios_family_c64p_Hwi_LD_end__C                                
c31377a8  ti_sysbios_family_c64p_Hwi_LM_begin__C                              
c31377ac  ti_sysbios_family_c64p_Hwi_Module__diagsEnabled__C                  
c31377b0  ti_sysbios_family_c64p_Hwi_Module__diagsIncluded__C                 
c31377b4  ti_sysbios_family_c64p_Hwi_Module__diagsMask__C                     
c3137994  ti_sysbios_family_c64p_Hwi_Module__id__C                            
c3137996  ti_sysbios_family_c64p_Hwi_Module__loggerDefined__C                 
c31377b8  ti_sysbios_family_c64p_Hwi_Module__loggerFxn1__C                    
c31377bc  ti_sysbios_family_c64p_Hwi_Module__loggerFxn8__C                    
c31377c0  ti_sysbios_family_c64p_Hwi_Module__loggerObj__C                     
c3134a90  ti_sysbios_family_c64p_Hwi_Module__root__V                          
c311cc60  ti_sysbios_family_c64p_Hwi_Module__startupDone__F                   
c311cc60  ti_sysbios_family_c64p_Hwi_Module__startupDone__S                   
c31345f0  ti_sysbios_family_c64p_Hwi_Module__state__V                         
c3114e80  ti_sysbios_family_c64p_Hwi_Module_startup__E                        
c313755c  ti_sysbios_family_c64p_Hwi_Object__DESC__C                          
c31372f0  ti_sysbios_family_c64p_Hwi_Object__PARAMS__C                        
c3134a40  ti_sysbios_family_c64p_Hwi_Object__table__V                         
c311cc80  ti_sysbios_family_c64p_Hwi_Params__init__S                          
c311cca0  ti_sysbios_family_c64p_Hwi_clearInterrupt__E                        
c3118e60  ti_sysbios_family_c64p_Hwi_construct                                
c311be80  ti_sysbios_family_c64p_Hwi_destruct                                 
c311bec0  ti_sysbios_family_c64p_Hwi_disableInterrupt__E                      
c3111500  ti_sysbios_family_c64p_Hwi_dispatchAlways                           
c3118f00  ti_sysbios_family_c64p_Hwi_dispatchC__I                             
c310f460  ti_sysbios_family_c64p_Hwi_dispatchCore__I                          
c311bf00  ti_sysbios_family_c64p_Hwi_enableInterrupt__E                       
c311b0c0  ti_sysbios_family_c64p_Hwi_getEventId__E                            
c311ccc0  ti_sysbios_family_c64p_Hwi_getFunc__E                               
c311cce0  ti_sysbios_family_c64p_Hwi_getHandle__E                             
c3118fa0  ti_sysbios_family_c64p_Hwi_getStackInfo__E                          
c3138c00  ti_sysbios_family_c64p_Hwi_int0                                     
c3138c20  ti_sysbios_family_c64p_Hwi_int1                                     
c3138d40  ti_sysbios_family_c64p_Hwi_int10                                    
c3138d60  ti_sysbios_family_c64p_Hwi_int11                                    
c3138d80  ti_sysbios_family_c64p_Hwi_int12                                    
c3138da0  ti_sysbios_family_c64p_Hwi_int13                                    
c3138dc0  ti_sysbios_family_c64p_Hwi_int14                                    
c3138de0  ti_sysbios_family_c64p_Hwi_int15                                    
c3138c40  ti_sysbios_family_c64p_Hwi_int2                                     
c3138c60  ti_sysbios_family_c64p_Hwi_int3                                     
c3138c80  ti_sysbios_family_c64p_Hwi_int4                                     
c3138ca0  ti_sysbios_family_c64p_Hwi_int5                                     
c3138cc0  ti_sysbios_family_c64p_Hwi_int6                                     
c3138ce0  ti_sysbios_family_c64p_Hwi_int7                                     
c3138d00  ti_sysbios_family_c64p_Hwi_int8                                     
c3138d20  ti_sysbios_family_c64p_Hwi_int9                                     
c3118c80  ti_sysbios_family_c64p_Hwi_plug__E                                  
c310eaa0  ti_sysbios_family_c64p_Hwi_reconfig__E                              
c311cd00  ti_sysbios_family_c64p_Hwi_startup__E                               
c311ac40  ti_sysbios_family_c64p_Hwi_switchAndDispatch__I                     
c311cd20  ti_sysbios_family_c64p_Hwi_switchFromBootStack__E                   
c311cd40  ti_sysbios_family_c64p_Hwi_unPluggedInterrupt__I                    
c3134a98  ti_sysbios_family_c64p_primus_TimerSupport_Module_State_0_suspSrc__A
c3134ae8  ti_sysbios_family_c64p_primus_TimerSupport_Module__state__V         
c311bf40  ti_sysbios_family_c64p_primus_TimerSupport_enable__E                
c311aca0  ti_sysbios_family_xxx_Hwi_switchAndRunFunc                          
c311bf80  ti_sysbios_gates_GateHwi_Handle__label__S                           
c311cd60  ti_sysbios_gates_GateHwi_Instance_init__E                           
c31373ec  ti_sysbios_gates_GateHwi_Module__FXNS__C                            
c3134aa0  ti_sysbios_gates_GateHwi_Module__root__V                            
c313757c  ti_sysbios_gates_GateHwi_Object__DESC__C                            
c3137688  ti_sysbios_gates_GateHwi_Object__PARAMS__C                          
c3119bc0  ti_sysbios_gates_GateHwi_Object__create__S                          
c311bfc0  ti_sysbios_gates_GateHwi_Object__delete__S                          
c3134af0  ti_sysbios_gates_GateHwi_Object__table__V                           
c311cd80  ti_sysbios_gates_GateHwi_enter__E                                   
c311cda0  ti_sysbios_gates_GateHwi_leave__E                                   
c311cdc0  ti_sysbios_gates_GateHwi_query__E                                   
c31377c4  ti_sysbios_gates_GateMutex_A_badContext__C                          
c311c000  ti_sysbios_gates_GateMutex_Handle__label__S                         
c31377c8  ti_sysbios_gates_GateMutex_Instance_State_sem__O                    
c311cde0  ti_sysbios_gates_GateMutex_Instance_finalize__E                     
c311c040  ti_sysbios_gates_GateMutex_Instance_init__E                         
c3137410  ti_sysbios_gates_GateMutex_Module__FXNS__C                          
c31377cc  ti_sysbios_gates_GateMutex_Module__diagsEnabled__C                  
c31377d0  ti_sysbios_gates_GateMutex_Module__diagsIncluded__C                 
c31377d4  ti_sysbios_gates_GateMutex_Module__diagsMask__C                     
c3137998  ti_sysbios_gates_GateMutex_Module__id__C                            
c3134aa8  ti_sysbios_gates_GateMutex_Module__root__V                          
c313759c  ti_sysbios_gates_GateMutex_Object__DESC__C                          
c31376a0  ti_sysbios_gates_GateMutex_Object__PARAMS__C                        
c3119c40  ti_sysbios_gates_GateMutex_Object__create__S                        
c311b120  ti_sysbios_gates_GateMutex_Object__delete__S                        
c3134840  ti_sysbios_gates_GateMutex_Object__table__V                         
c3111ea0  ti_sysbios_gates_GateMutex_enter__E                                 
c311c080  ti_sysbios_gates_GateMutex_leave__E                                 
c311ce00  ti_sysbios_gates_GateMutex_query__E                                 
c31377d8  ti_sysbios_hal_Hwi_E_stackOverflow__C                               
c311cc60  ti_sysbios_hal_Hwi_HwiProxy_Module__startupDone__S                  
c311cc80  ti_sysbios_hal_Hwi_HwiProxy_Params__init__S                         
c311cca0  ti_sysbios_hal_Hwi_HwiProxy_clearInterrupt__E                       
c311bec0  ti_sysbios_hal_Hwi_HwiProxy_disableInterrupt__E                     
c311bf00  ti_sysbios_hal_Hwi_HwiProxy_enableInterrupt__E                      
c3118fa0  ti_sysbios_hal_Hwi_HwiProxy_getStackInfo__E                         
c311cd00  ti_sysbios_hal_Hwi_HwiProxy_startup__E                              
c311cd20  ti_sysbios_hal_Hwi_HwiProxy_switchFromBootStack__E                  
c313799a  ti_sysbios_hal_Hwi_Module__id__C                                    
c311ce20  ti_sysbios_hal_Hwi_Module_startup__E                                
c3134ab0  ti_sysbios_hal_Hwi_Object__table__V                                 
c3119cc0  ti_sysbios_hal_Hwi_checkStack                                       
c311cca0  ti_sysbios_hal_Hwi_clearInterrupt__E                                
c311bec0  ti_sysbios_hal_Hwi_disableInterrupt__E                              
c311bf00  ti_sysbios_hal_Hwi_enableInterrupt__E                               
c3118fa0  ti_sysbios_hal_Hwi_getStackInfo__E                                  
c3119d40  ti_sysbios_hal_Hwi_initStack                                        
c311cd00  ti_sysbios_hal_Hwi_startup__E                                       
c311cd20  ti_sysbios_hal_Hwi_switchFromBootStack__E                           
c31377dc  ti_sysbios_heaps_HeapBuf_Instance_State_freeList__O                 
c3134aec  ti_sysbios_heaps_HeapBuf_Module__state__V                           
c31131a0  ti_sysbios_heaps_HeapBuf_Module_startup__E                          
c31377e0  ti_sysbios_heaps_HeapBuf_Object__count__C                           
c311ce40  ti_sysbios_heaps_HeapBuf_Object__get__S                             
c31377e4  ti_sysbios_heaps_HeapBuf_numConstructedHeaps__C                     
c31377e8  ti_sysbios_heaps_HeapMem_A_align__C                                 
c31377ec  ti_sysbios_heaps_HeapMem_A_heapSize__C                              
c31377f0  ti_sysbios_heaps_HeapMem_A_invalidFree__C                           
c31377f4  ti_sysbios_heaps_HeapMem_A_zeroBlock__C                             
c31377f8  ti_sysbios_heaps_HeapMem_E_memory__C                                
c311c0c0  ti_sysbios_heaps_HeapMem_Handle__label__S                           
11700000  ti_sysbios_heaps_HeapMem_Instance_State_0_buf__A                    
c310d820  ti_sysbios_heaps_HeapMem_Instance_init__E                           
c311c000  ti_sysbios_heaps_HeapMem_Module_GateProxy_Handle__label__S          
c311ce60  ti_sysbios_heaps_HeapMem_Module_GateProxy_enter__E                  
c311ce80  ti_sysbios_heaps_HeapMem_Module_GateProxy_leave__E                  
c311ce00  ti_sysbios_heaps_HeapMem_Module_GateProxy_query__E                  
c313737c  ti_sysbios_heaps_HeapMem_Module__FXNS__C                            
c31377fc  ti_sysbios_heaps_HeapMem_Module__diagsEnabled__C                    
c3137800  ti_sysbios_heaps_HeapMem_Module__diagsIncluded__C                   
c3137804  ti_sysbios_heaps_HeapMem_Module__diagsMask__C                       
c3137808  ti_sysbios_heaps_HeapMem_Module__gateObj__C                         
c313799c  ti_sysbios_heaps_HeapMem_Module__id__C                              
c3134ab8  ti_sysbios_heaps_HeapMem_Module__root__V                            
c31375bc  ti_sysbios_heaps_HeapMem_Object__DESC__C                            
c3137434  ti_sysbios_heaps_HeapMem_Object__PARAMS__C                          
c313780c  ti_sysbios_heaps_HeapMem_Object__count__C                           
c3119dc0  ti_sysbios_heaps_HeapMem_Object__create__S                          
c311c100  ti_sysbios_heaps_HeapMem_Object__delete__S                          
c311c140  ti_sysbios_heaps_HeapMem_Object__get__S                             
c3134a58  ti_sysbios_heaps_HeapMem_Object__table__V                           
c31081c0  ti_sysbios_heaps_HeapMem_allocUnprotected__E                        
c31176e0  ti_sysbios_heaps_HeapMem_alloc__E                                   
c3108dc0  ti_sysbios_heaps_HeapMem_freeUnprotected__E                         
c311b180  ti_sysbios_heaps_HeapMem_free__E                                    
c31181c0  ti_sysbios_heaps_HeapMem_getStats__E                                
c3119040  ti_sysbios_heaps_HeapMem_init__I                                    
c311cea0  ti_sysbios_heaps_HeapMem_isBlocking__E                              
c3137810  ti_sysbios_heaps_HeapMem_reqAlign__C                                
c3137814  ti_sysbios_knl_Clock_LM_begin__C                                    
c3137818  ti_sysbios_knl_Clock_LM_tick__C                                     
c313781c  ti_sysbios_knl_Clock_LW_delayed__C                                  
c3137820  ti_sysbios_knl_Clock_Module_State_clockQ__O                         
c3137824  ti_sysbios_knl_Clock_Module__diagsEnabled__C                        
c3137828  ti_sysbios_knl_Clock_Module__diagsIncluded__C                       
c313782c  ti_sysbios_knl_Clock_Module__diagsMask__C                           
c313799e  ti_sysbios_knl_Clock_Module__id__C                                  
c31379a0  ti_sysbios_knl_Clock_Module__loggerDefined__C                       
c3137830  ti_sysbios_knl_Clock_Module__loggerFxn1__C                          
c3137834  ti_sysbios_knl_Clock_Module__loggerFxn2__C                          
c3137838  ti_sysbios_knl_Clock_Module__loggerObj__C                           
c313490c  ti_sysbios_knl_Clock_Module__state__V                               
c311b1e0  ti_sysbios_knl_Clock_Module_startup__E                              
c311d040  ti_sysbios_knl_Clock_TimerProxy_Module__startupDone__S              
c311cec0  ti_sysbios_knl_Clock_TimerProxy_getMaxTicks__E                      
c31177c0  ti_sysbios_knl_Clock_TimerProxy_startup__E                          
c3119e40  ti_sysbios_knl_Clock_doTick__I                                      
c3118280  ti_sysbios_knl_Clock_logTick__E                                     
c310e580  ti_sysbios_knl_Clock_workFunc__E                                    
c3137840  ti_sysbios_knl_Idle_funcList__A                                     
c3137708  ti_sysbios_knl_Idle_funcList__C                                     
c311cee0  ti_sysbios_knl_Idle_loop__E                                         
c3119ec0  ti_sysbios_knl_Idle_run__E                                          
c311cf00  ti_sysbios_knl_Queue_Instance_init__E                               
c3134ac0  ti_sysbios_knl_Queue_Module__root__V                                
c31375dc  ti_sysbios_knl_Queue_Object__DESC__C                                
c31376b8  ti_sysbios_knl_Queue_Object__PARAMS__C                              
c311cf20  ti_sysbios_knl_Queue_Object__get__S                                 
c311b240  ti_sysbios_knl_Queue_construct                                      
c311cf40  ti_sysbios_knl_Queue_destruct                                       
c311cf60  ti_sysbios_knl_Queue_empty__E                                       
c313783c  ti_sysbios_knl_Semaphore_A_badContext__C                            
c3137844  ti_sysbios_knl_Semaphore_A_noEvents__C                              
c3137848  ti_sysbios_knl_Semaphore_A_overflow__C                              
c313784c  ti_sysbios_knl_Semaphore_A_pendTaskDisabled__C                      
c3137850  ti_sysbios_knl_Semaphore_Instance_State_pendQ__O                    
c311cf80  ti_sysbios_knl_Semaphore_Instance_finalize__E                       
c3114fc0  ti_sysbios_knl_Semaphore_Instance_init__E                           
c3137854  ti_sysbios_knl_Semaphore_LM_pend__C                                 
c3137858  ti_sysbios_knl_Semaphore_LM_post__C                                 
c313785c  ti_sysbios_knl_Semaphore_Module__diagsEnabled__C                    
c3137860  ti_sysbios_knl_Semaphore_Module__diagsIncluded__C                   
c3137864  ti_sysbios_knl_Semaphore_Module__diagsMask__C                       
c31379a2  ti_sysbios_knl_Semaphore_Module__id__C                              
c31379a4  ti_sysbios_knl_Semaphore_Module__loggerDefined__C                   
c3137868  ti_sysbios_knl_Semaphore_Module__loggerFxn2__C                      
c313786c  ti_sysbios_knl_Semaphore_Module__loggerFxn4__C                      
c3137870  ti_sysbios_knl_Semaphore_Module__loggerObj__C                       
c3134ac8  ti_sysbios_knl_Semaphore_Module__root__V                            
c31375fc  ti_sysbios_knl_Semaphore_Object__DESC__C                            
c3137458  ti_sysbios_knl_Semaphore_Object__PARAMS__C                          
c311cfa0  ti_sysbios_knl_Semaphore_Params__init__S                            
c311b2a0  ti_sysbios_knl_Semaphore_construct                                  
c311c180  ti_sysbios_knl_Semaphore_destruct                                   
c3119f40  ti_sysbios_knl_Semaphore_pendTimeout__I                             
c31059a0  ti_sysbios_knl_Semaphore_pend__E                                    
c310ed20  ti_sysbios_knl_Semaphore_post__E                                    
c3137874  ti_sysbios_knl_Swi_LD_end__C                                        
c3137878  ti_sysbios_knl_Swi_LM_begin__C                                      
c313787c  ti_sysbios_knl_Swi_LM_post__C                                       
c31344f8  ti_sysbios_knl_Swi_Module_State_0_readyQ__A                         
c3137880  ti_sysbios_knl_Swi_Module__diagsEnabled__C                          
c3137884  ti_sysbios_knl_Swi_Module__diagsIncluded__C                         
c3137888  ti_sysbios_knl_Swi_Module__diagsMask__C                             
c31379a6  ti_sysbios_knl_Swi_Module__id__C                                    
c31379a8  ti_sysbios_knl_Swi_Module__loggerDefined__C                         
c313788c  ti_sysbios_knl_Swi_Module__loggerFxn1__C                            
c3137890  ti_sysbios_knl_Swi_Module__loggerFxn4__C                            
c3137894  ti_sysbios_knl_Swi_Module__loggerObj__C                             
c3134a20  ti_sysbios_knl_Swi_Module__state__V                                 
c311b300  ti_sysbios_knl_Swi_Module_startup__E                                
c3137898  ti_sysbios_knl_Swi_Object__count__C                                 
c311c1c0  ti_sysbios_knl_Swi_Object__get__S                                   
c31348b0  ti_sysbios_knl_Swi_Object__table__V                                 
c311cfc0  ti_sysbios_knl_Swi_disable__E                                       
c31146c0  ti_sysbios_knl_Swi_post__E                                          
c31165a0  ti_sysbios_knl_Swi_restoreHwi__E                                    
c310c9e0  ti_sysbios_knl_Swi_runLoop__I                                       
c3110ac0  ti_sysbios_knl_Swi_run__I                                           
c3118340  ti_sysbios_knl_Swi_schedule__I                                      
c3119fc0  ti_sysbios_knl_Swi_startup__E                                       
c313789c  ti_sysbios_knl_Task_A_badTimeout__C                                 
c31378a0  ti_sysbios_knl_Task_A_sleepTaskDisabled__C                          
c3000000  ti_sysbios_knl_Task_Instance_State_0_stack__A                       
c3100000  ti_sysbios_knl_Task_Instance_State_1_stack__A                       
c31378a4  ti_sysbios_knl_Task_LD_block__C                                     
c31378a8  ti_sysbios_knl_Task_LD_exit__C                                      
c31378ac  ti_sysbios_knl_Task_LD_ready__C                                     
c31378b0  ti_sysbios_knl_Task_LM_sleep__C                                     
c31378b4  ti_sysbios_knl_Task_LM_switch__C                                    
c3134af8  ti_sysbios_knl_Task_Module_State_0_idleTask__A                      
c3134960  ti_sysbios_knl_Task_Module_State_0_readyQ__A                        
c31378b8  ti_sysbios_knl_Task_Module_State_inactiveQ__O                       
c31378bc  ti_sysbios_knl_Task_Module__diagsEnabled__C                         
c31378c0  ti_sysbios_knl_Task_Module__diagsIncluded__C                        
c31378c4  ti_sysbios_knl_Task_Module__diagsMask__C                            
c31379aa  ti_sysbios_knl_Task_Module__id__C                                   
c31379ac  ti_sysbios_knl_Task_Module__loggerDefined__C                        
c31378c8  ti_sysbios_knl_Task_Module__loggerFxn2__C                           
c31378cc  ti_sysbios_knl_Task_Module__loggerFxn4__C                           
c31378d0  ti_sysbios_knl_Task_Module__loggerObj__C                            
c3134778  ti_sysbios_knl_Task_Module__state__V                                
c310dae0  ti_sysbios_knl_Task_Module_startup__E                               
c31378d4  ti_sysbios_knl_Task_Object__count__C                                
c311c200  ti_sysbios_knl_Task_Object__get__S                                  
c3134300  ti_sysbios_knl_Task_Object__table__V                                
c311cc20  ti_sysbios_knl_Task_SupportProxy_Module__startupDone__S             
c311af40  ti_sysbios_knl_Task_SupportProxy_start__E                           
c3119840  ti_sysbios_knl_Task_SupportProxy_swap__E                            
c31378d8  ti_sysbios_knl_Task_allBlockedFunc__C                               
c31190e0  ti_sysbios_knl_Task_allBlockedFunction__I                           
c3115100  ti_sysbios_knl_Task_blockI__E                                       
c311cfe0  ti_sysbios_knl_Task_disable__E                                      
c311d000  ti_sysbios_knl_Task_enable__E                                       
c311b360  ti_sysbios_knl_Task_enter__I                                        
c3113f80  ti_sysbios_knl_Task_exit__E                                         
c31378dc  ti_sysbios_knl_Task_numConstructedTasks__C                          
c311a040  ti_sysbios_knl_Task_restore__E                                      
c3114100  ti_sysbios_knl_Task_schedule__I                                     
c311c240  ti_sysbios_knl_Task_sleepTimeout__I                                 
c310af20  ti_sysbios_knl_Task_sleep__E                                        
c3114280  ti_sysbios_knl_Task_startCore__E                                    
c311d020  ti_sysbios_knl_Task_startup__E                                      
c3115b80  ti_sysbios_knl_Task_unblockI__E                                     
c31378e0  ti_sysbios_timers_timer64_Timer_A_notAvailable__C                   
c31378e4  ti_sysbios_timers_timer64_Timer_E_cannotSupport__C                  
c31346c8  ti_sysbios_timers_timer64_Timer_Module_State_0_device__A            
c3134980  ti_sysbios_timers_timer64_Timer_Module_State_0_gctrl__A             
c31349a0  ti_sysbios_timers_timer64_Timer_Module_State_0_handles__A           
c31349c0  ti_sysbios_timers_timer64_Timer_Module_State_0_intFreqs__A          
c31378e8  ti_sysbios_timers_timer64_Timer_Module__diagsEnabled__C             
c31378ec  ti_sysbios_timers_timer64_Timer_Module__diagsIncluded__C            
c31378f0  ti_sysbios_timers_timer64_Timer_Module__diagsMask__C                
c31379ae  ti_sysbios_timers_timer64_Timer_Module__id__C                       
c311d040  ti_sysbios_timers_timer64_Timer_Module__startupDone__F              
c311d040  ti_sysbios_timers_timer64_Timer_Module__startupDone__S              
c3134a70  ti_sysbios_timers_timer64_Timer_Module__state__V                    
c3106120  ti_sysbios_timers_timer64_Timer_Module_startup__E                   
c3134728  ti_sysbios_timers_timer64_Timer_Object__table__V                    
c311bf40  ti_sysbios_timers_timer64_Timer_TimerSupportProxy_enable__E         
c31378f4  ti_sysbios_timers_timer64_Timer_anyMaskHigh__C                      
c31378f8  ti_sysbios_timers_timer64_Timer_anyMask__C                          
c310c380  ti_sysbios_timers_timer64_Timer_deviceConfig__I                     
c31378fc  ti_sysbios_timers_timer64_Timer_freqDivisor__C                      
c3112960  ti_sysbios_timers_timer64_Timer_getFreq__E                          
c311d060  ti_sysbios_timers_timer64_Timer_getMaxTicks__E                      
c31166a0  ti_sysbios_timers_timer64_Timer_initDevice__I                       
c3136ed9  ti_sysbios_timers_timer64_Timer_localTimerBaseId__C                 
c3137900  ti_sysbios_timers_timer64_Timer_numLocalTimers__C                   
c3137904  ti_sysbios_timers_timer64_Timer_numTimerDevices__C                  
c3110ce0  ti_sysbios_timers_timer64_Timer_setPeriodMicroSecs__E               
c3113340  ti_sysbios_timers_timer64_Timer_start__E                            
c31379b0  ti_sysbios_timers_timer64_Timer_startupNeeded__C                    
c31177c0  ti_sysbios_timers_timer64_Timer_startup__E                          
c3119180  ti_sysbios_timers_timer64_Timer_stop__E                             
c31379b2  ti_sysbios_timers_timer64_Timer_useTimer64pRegMap__C                
c3134210  uartInitCfg                                                         
c3100c08  uart_stdio                                                          
c311a140  unlink                                                              
c311b420  write                                                               
c3137908  xdc_runtime_Assert_E_assertFailed__C                                
c31184c0  xdc_runtime_Assert_raise__I                                         
c313790c  xdc_runtime_Core_A_initializedParams__C                             
c3137910  xdc_runtime_Core_Module__diagsEnabled__C                            
c3137914  xdc_runtime_Core_Module__diagsIncluded__C                           
c3137918  xdc_runtime_Core_Module__diagsMask__C                               
c31379b4  xdc_runtime_Core_Module__id__C                                      
c311a1c0  xdc_runtime_Core_assignLabel__I                                     
c3119220  xdc_runtime_Core_assignParams__I                                    
c31134e0  xdc_runtime_Core_constructObject__I                                 
c310ffe0  xdc_runtime_Core_createObject__I                                    
c3115240  xdc_runtime_Core_deleteObject__I                                    
c313791c  xdc_runtime_Error_E_memory__C                                       
c31349e0  xdc_runtime_Error_IgnoreBlock                                       
c3137920  xdc_runtime_Error_Module__diagsEnabled__C                           
c3137924  xdc_runtime_Error_Module__diagsIncluded__C                          
c3137928  xdc_runtime_Error_Module__diagsMask__C                              
c31379b6  xdc_runtime_Error_Module__loggerDefined__C                          
c313792c  xdc_runtime_Error_Module__loggerFxn8__C                             
c3137930  xdc_runtime_Error_Module__loggerObj__C                              
c31346c2  xdc_runtime_Error_Module__state__V                                  
c311c280  xdc_runtime_Error_check__E                                          
c311d080  xdc_runtime_Error_getSite__E                                        
c311c2c0  xdc_runtime_Error_init__E                                           
c31379b8  xdc_runtime_Error_maxDepth__C                                       
c3111700  xdc_runtime_Error_policyDefault__E                                  
c3137934  xdc_runtime_Error_policyFxn__C                                      
c3137938  xdc_runtime_Error_policy__C                                         
c31167a0  xdc_runtime_Error_print__E                                          
c313793c  xdc_runtime_Error_raiseHook__C                                      
c311d0a0  xdc_runtime_Error_raiseX__E                                         
c3118580  xdc_runtime_Error_setX__E                                           
c311d0c0  xdc_runtime_Gate_enterSystem__E                                     
c311d0e0  xdc_runtime_Gate_leaveSystem__E                                     
c3137940  xdc_runtime_IGateProvider_Interface__BASE__C                        
c3137944  xdc_runtime_IHeap_Interface__BASE__C                                
c3137948  xdc_runtime_IModule_Interface__BASE__C                              
c313794c  xdc_runtime_Log_L_error__C                                          
c311bf80  xdc_runtime_Main_Module_GateProxy_Handle__label__S                  
c311cdc0  xdc_runtime_Main_Module_GateProxy_query__E                          
c31379ba  xdc_runtime_Main_Module__id__C                                      
c311c0c0  xdc_runtime_Memory_HeapProxy_Handle__label__S                       
c311d100  xdc_runtime_Memory_HeapProxy_alloc__E                               
c311d120  xdc_runtime_Memory_HeapProxy_free__E                                
c31379bc  xdc_runtime_Memory_Module__id__C                                    
c3134af4  xdc_runtime_Memory_Module__state__V                                 
c31168a0  xdc_runtime_Memory_alloc__E                                         
c311d140  xdc_runtime_Memory_calloc__E                                        
c3137950  xdc_runtime_Memory_defaultHeapInstance__C                           
c311d160  xdc_runtime_Memory_free__E                                          
c311d180  xdc_runtime_Memory_getMaxDefaultTypeAlign__E                        
c311b480  xdc_runtime_Memory_valloc__E                                        
c3134ad0  xdc_runtime_Registry_Module__state__V                               
c311c300  xdc_runtime_Registry_findById__E                                    
c3134ad8  xdc_runtime_Startup_Module__state__V                                
00000001  xdc_runtime_Startup__EXECFXN__C                                     
00000001  xdc_runtime_Startup__RESETFXN__C                                    
c3137954  xdc_runtime_Startup_execImpl__C                                     
c31169a0  xdc_runtime_Startup_exec__E                                         
c311d1a0  xdc_runtime_Startup_exec__I                                         
c3137710  xdc_runtime_Startup_firstFxns__A                                    
c3137718  xdc_runtime_Startup_firstFxns__C                                    
c3137720  xdc_runtime_Startup_lastFxns__C                                     
c3137958  xdc_runtime_Startup_maxPasses__C                                    
c311d1c0  xdc_runtime_Startup_reset__I                                        
c311d1e0  xdc_runtime_Startup_rtsDone__E                                      
c31376d0  xdc_runtime_Startup_sfxnRts__A                                      
c313795c  xdc_runtime_Startup_sfxnRts__C                                      
c3137350  xdc_runtime_Startup_sfxnTab__A                                      
c3137960  xdc_runtime_Startup_sfxnTab__C                                      
c310f6c0  xdc_runtime_Startup_startMods__I                                    
c311a240  xdc_runtime_SysStd_abort__E                                         
c311d200  xdc_runtime_SysStd_exit__E                                          
c311d220  xdc_runtime_SysStd_putch__E                                         
c311d240  xdc_runtime_SysStd_ready__E                                         
c311bf80  xdc_runtime_System_Module_GateProxy_Handle__label__S                
c311d260  xdc_runtime_System_Module_GateProxy_enter__E                        
c311d280  xdc_runtime_System_Module_GateProxy_leave__E                        
c311cdc0  xdc_runtime_System_Module_GateProxy_query__E                        
c3134a00  xdc_runtime_System_Module_State_0_atexitHandlers__A                 
c3137964  xdc_runtime_System_Module__gateObj__C                               
c3134ae0  xdc_runtime_System_Module__state__V                                 
c311d2a0  xdc_runtime_System_Module_startup__E                                
c311a240  xdc_runtime_System_SupportProxy_abort__E                            
c311d200  xdc_runtime_System_SupportProxy_exit__E                             
c311d220  xdc_runtime_System_SupportProxy_putch__E                            
c311d240  xdc_runtime_System_SupportProxy_ready__E                            
c3137968  xdc_runtime_System_abortFxn__C                                      
c311ca40  xdc_runtime_System_abortStd__E                                      
c311c340  xdc_runtime_System_abort__E                                         
c311c380  xdc_runtime_System_aprintf__E                                       
c311a340  xdc_runtime_System_aprintf_va__E                                    
c311a340  xdc_runtime_System_aprintf_va__F                                    
c311a2c0  xdc_runtime_System_atexit__E                                        
c311a340  xdc_runtime_System_avprintf__E                                      
c3104160  xdc_runtime_System_doPrint__I                                       
c313796c  xdc_runtime_System_exitFxn__C                                       
c3117360  xdc_runtime_System_exitStd__E                                       
c311c3c0  xdc_runtime_System_exit__E                                          
c3137970  xdc_runtime_System_extendFxn__C                                     
c31192c0  xdc_runtime_System_formatNum__I                                     
c3137974  xdc_runtime_System_maxAtexitHandlers__C                             
c3110220  xdc_runtime_System_printfExtend__I                                  
c311c400  xdc_runtime_System_printf__E                                        
c311a440  xdc_runtime_System_printf_va__E                                     
c311a440  xdc_runtime_System_printf_va__F                                     
c311a3c0  xdc_runtime_System_processAtExit__E                                 
c3119360  xdc_runtime_System_putchar__I                                       
c311d2c0  xdc_runtime_System_snprintf_va__E                                   
c311d2c0  xdc_runtime_System_snprintf_va__F                                   
c311a440  xdc_runtime_System_vprintf__E                                       
c311d2c0  xdc_runtime_System_vsnprintf__E                                     
c31379be  xdc_runtime_Text_charCnt__C                                         
c3134b00  xdc_runtime_Text_charTab__A                                         
c3137978  xdc_runtime_Text_charTab__C                                         
c311b4e0  xdc_runtime_Text_cordText__E                                        
c31379c0  xdc_runtime_Text_isLoaded__C                                        
c313797c  xdc_runtime_Text_nameEmpty__C                                       
c3137980  xdc_runtime_Text_nameStatic__C                                      
c3137984  xdc_runtime_Text_nameUnknown__C                                     
c3136ee0  xdc_runtime_Text_nodeTab__A                                         
c3137988  xdc_runtime_Text_nodeTab__C                                         
c3119400  xdc_runtime_Text_printVisFxn__I                                     
c3115380  xdc_runtime_Text_putLab__E                                          
c3114820  xdc_runtime_Text_putMod__E                                          
c3112080  xdc_runtime_Text_putSite__E                                         
c31379c2  xdc_runtime_Text_registryModsLastId__C                              
c311d2e0  xdc_runtime_Text_ropeText__E                                        
c31379c4  xdc_runtime_Text_unnamedModsLastId__C                               
c31178a0  xdc_runtime_Text_visitRope2__I                                      
c313798c  xdc_runtime_Text_visitRopeFxn__C                                    
c311d300  xdc_runtime_Text_visitRope__I                                       
c31194a0  xdc_runtime_Text_xprintf__I                                         


GLOBAL SYMBOLS: SORTED BY Symbol Address 

address   name                                                                
-------   ----                                                                
00000000  _argsize                                                            
00000000  ti_sysbios_family_c64p_Cache_l2Size                                 
00000001  xdc_runtime_Startup__EXECFXN__C                                     
00000001  xdc_runtime_Startup__RESETFXN__C                                    
00001000  __TI_STACK_SIZE                                                     
00008000  ti_sysbios_family_c64p_Cache_l1dSize                                
00008000  ti_sysbios_family_c64p_Cache_l1pSize                                
11700000  ti_sysbios_heaps_HeapMem_Instance_State_0_buf__A                    
c3000000  __ASM__                                                             
c3000000  ti_sysbios_knl_Task_Instance_State_0_stack__A                       
c3000058  __ISA__                                                             
c3000070  __PLAT__                                                            
c3000098  __TARG__                                                            
c30000c0  __TRDR__                                                            
c3100000  ti_sysbios_knl_Task_Instance_State_1_stack__A                       
c3100800  UartObjects                                                         
c3100998  __TI_tmpnams                                                        
c3100ad8  SpiObjects                                                          
c3100b70  edma3_dma_ch_max_val                                                
c3100b88  edma3_link_ch_max_val                                               
c3100ba0  edma3_link_ch_min_val                                               
c3100bb8  edma3_log_ch_max_val                                                
c3100bd0  edma3_qdma_ch_max_val                                               
c3100be8  edma3_qdma_ch_min_val                                               
c3100c00  parmbuf                                                             
c3100c08  uart_stdio                                                          
c3100c10  __TI_cleanup_ptr                                                    
c3100c14  __TI_dtors_ptr                                                      
c3100c18  __TI_enable_exit_profile_output                                     
c3100c1c  _lock                                                               
c3100c20  __TI_printfi                                                        
c3102900  EDMA3_RM_allocResource                                              
c3103540  EDMA3_DRV_requestChannel                                            
c3104160  xdc_runtime_System_doPrint__I                                       
c3105220  ti_sysbios_family_c64p_Exception_handler__I                         
c31059a0  ti_sysbios_knl_Semaphore_pend__E                                    
c3106120  ti_sysbios_timers_timer64_Timer_Module_startup__E                   
c3107540  UART_printf                                                         
c3107b80  ti_sysbios_family_c64p_Cache_Module_startup__E                      
c31081c0  ti_sysbios_heaps_HeapMem_allocUnprotected__E                        
c3108800  __c6xabi_divd                                                       
c3108dc0  ti_sysbios_heaps_HeapMem_freeUnprotected__E                         
c310a240  Board_pinmuxConfig                                                  
c310a6a0  EDMA3_RM_freeResource                                               
c310af20  ti_sysbios_knl_Task_sleep__E                                        
c310bfa0  fputs                                                               
c310c380  ti_sysbios_timers_timer64_Timer_deviceConfig__I                     
c310c6c0  EDMA3_DRV_freeChannel                                               
c310c9e0  ti_sysbios_knl_Swi_runLoop__I                                       
c310cd00  Board_CorePLLConfig                                                 
c310cfe0  EDMA3_DRV_disableTransfer                                           
c310d820  ti_sysbios_heaps_HeapMem_Instance_init__E                           
c310dae0  ti_sysbios_knl_Task_Module_startup__E                               
c310dda0  Board_DDRPLLConfig                                                  
c310e580  ti_sysbios_knl_Clock_workFunc__E                                    
c310e820  EDMA3_DRV_enableTransfer                                            
c310eaa0  ti_sysbios_family_c64p_Hwi_reconfig__E                              
c310ed20  ti_sysbios_knl_Semaphore_post__E                                    
c310efa0  __c6xabi_divull                                                     
c310f200  ti_sysbios_family_c64p_Cache_block__I                               
c310f460  ti_sysbios_family_c64p_Hwi_dispatchCore__I                          
c310f6c0  xdc_runtime_Startup_startMods__I                                    
c310f920  Board_moduleClockEnable                                             
c310fb60  ti_sysbios_family_c64p_EventCombiner_dispatch__E                    
c310fda0  ti_sysbios_family_c64p_Exception_internalHandler__I                 
c310ffe0  xdc_runtime_Core_createObject__I                                    
c3110220  xdc_runtime_System_printfExtend__I                                  
c3110460  fputc                                                               
c3110460  putc                                                                
c3110680  Board_initSPI                                                       
c31106b0  spi_test                                                            
c3110888  main                                                                
c31108a0  setvbuf                                                             
c3110ac0  ti_sysbios_knl_Swi_run__I                                           
c3110ce0  ti_sysbios_timers_timer64_Timer_setPeriodMicroSecs__E               
c3110f00  SemaphoreP_create                                                   
c3111500  ti_sysbios_family_c64p_Hwi_dispatchAlways                           
c3111700  xdc_runtime_Error_policyDefault__E                                  
c3111900  Board_moduleClockSyncReset                                          
c3111ae0  HwiP_create                                                         
c3111ea0  ti_sysbios_gates_GateMutex_enter__E                                 
c3112080  xdc_runtime_Text_putSite__E                                         
c3112260  EDMA3_DRV_linkChannel                                               
c3112420  __c6xabi_divul                                                      
c31125e0  frexp                                                               
c31125e0  frexpl                                                              
c31127a0  ti_sysbios_family_c64p_EventCombiner_dispatchPlug__E                
c3112960  ti_sysbios_timers_timer64_Timer_getFreq__E                          
c3112b20  HOSTrename                                                          
c3112e60  ti_sysbios_family_c64p_EventCombiner_disableEvent__E                
c3113000  ti_sysbios_family_c64p_EventCombiner_enableEvent__E                 
c31131a0  ti_sysbios_heaps_HeapBuf_Module_startup__E                          
c3113340  ti_sysbios_timers_timer64_Timer_start__E                            
c31134e0  xdc_runtime_Core_constructObject__I                                 
c3113680  Board_DDR3Init                                                      
c3113800  EDMA3_DRV_getPaRAM                                                  
c3113980  EDMA3_RM_registerTccCb                                              
c3113b00  EDMA3_RM_unregisterTccCb                                            
c3113c80  ldexp                                                               
c3113c80  ldexpl                                                              
c3113e00  ti_sysbios_family_c64p_Exception_dispatch__E                        
c3113f80  ti_sysbios_knl_Task_exit__E                                         
c3114100  ti_sysbios_knl_Task_schedule__I                                     
c3114280  ti_sysbios_knl_Task_startCore__E                                    
c3114400  Board_init                                                          
c3114560  Osal_RegisterInterrupt                                              
c31146c0  ti_sysbios_knl_Swi_post__E                                          
c3114820  xdc_runtime_Text_putMod__E                                          
c3114980  EDMA3_DRV_setPaRAM                                                  
c3114ac0  __TI_closefile                                                      
c3114c00  fflush                                                              
c3114d40  getdevice                                                           
c3114e80  ti_sysbios_family_c64p_Hwi_Module_startup__E                        
c3114fc0  ti_sysbios_knl_Semaphore_Instance_init__E                           
c3115100  ti_sysbios_knl_Task_blockI__E                                       
c3115240  xdc_runtime_Core_deleteObject__I                                    
c3115380  xdc_runtime_Text_putLab__E                                          
c31154c0  Board_configEmifPinMux                                              
c3115820  _auto_init_elf                                                      
c3115940  fseek                                                               
c3115a60  ti_sysbios_family_c64p_Hwi_Instance_init__E                         
c3115b80  ti_sysbios_knl_Task_unblockI__E                                     
c3115ca0  Board_moduleClockInit                                               
c3115da0  EDMA3_DRV_clearErrorBits                                            
c3115ea0  EventCombinerP_GroupRegisterInt                                     
c31162a0  __TI_wrt_ok                                                         
c31163a0  atoi                                                                
c31164a0  ti_sysbios_family_c64p_Hwi_Instance_finalize__E                     
c31165a0  ti_sysbios_knl_Swi_restoreHwi__E                                    
c31166a0  ti_sysbios_timers_timer64_Timer_initDevice__I                       
c31167a0  xdc_runtime_Error_print__E                                          
c31168a0  xdc_runtime_Memory_alloc__E                                         
c31169a0  xdc_runtime_Startup_exec__E                                         
c3116aa0  EDMA3_DRV_getPaRAMPhyAddr                                           
c3116b80  EDMA3_DRV_unlinkChannel                                             
c3116c60  HOSTlseek                                                           
c3116d40  HOSTopen                                                            
c3116e20  HOSTwrite                                                           
c3116f00  MCSPI_init                                                          
c3116f00  SPI_init                                                            
c3117280  close                                                               
c3117360  exit                                                                
c3117360  xdc_runtime_System_exitStd__E                                       
c3117440  ltoa                                                                
c3117520  memset                                                              
c3117600  printf                                                              
c31176e0  ti_sysbios_heaps_HeapMem_alloc__E                                   
c31177c0  ti_sysbios_knl_Clock_TimerProxy_startup__E                          
c31177c0  ti_sysbios_timers_timer64_Timer_startup__E                          
c31178a0  xdc_runtime_Text_visitRope2__I                                      
c3117980  HOSTread                                                            
c3117a40  HOSTunlink                                                          
c3117b00  Osal_delay                                                          
c3117bc0  SPI_open                                                            
c3117e00  __TI_doflush                                                        
c3117ec0  __c6xabi_divu                                                       
c3117ec0  __divu                                                              
c3118040  edma3MemZero                                                        
c3118100  edma3OsProtectEntry                                                 
c31181c0  ti_sysbios_heaps_HeapMem_getStats__E                                
c3118280  ti_sysbios_knl_Clock_logTick__E                                     
c3118340  ti_sysbios_knl_Swi_schedule__I                                      
c3118400  __TI_tls_init                                                       
c31184c0  xdc_runtime_Assert_raise__I                                         
c3118580  xdc_runtime_Error_setX__E                                           
c3118640  HOSTclose                                                           
c31186e0  Osal_DeleteInterrupt                                                
c3118820  UART_init                                                           
c31188c0  UART_stdioInit                                                      
c3118aa0  __TI_cleanup                                                        
c3118b40  __c6xabi_remu                                                       
c3118b40  __remu                                                              
c3118be0  _c_int00                                                            
c3118c80  ti_sysbios_family_c64p_Hwi_plug__E                                  
c3118d20  memcpy                                                              
c3118dc0  ti_sysbios_family_c64p_Exception_Module_startup__E                  
c3118e60  ti_sysbios_family_c64p_Hwi_construct                                
c3118f00  ti_sysbios_family_c64p_Hwi_dispatchC__I                             
c3118fa0  ti_sysbios_family_c64p_Hwi_getStackInfo__E                          
c3118fa0  ti_sysbios_hal_Hwi_HwiProxy_getStackInfo__E                         
c3118fa0  ti_sysbios_hal_Hwi_getStackInfo__E                                  
c3119040  ti_sysbios_heaps_HeapMem_init__I                                    
c31190e0  ti_sysbios_knl_Task_allBlockedFunction__I                           
c3119180  ti_sysbios_timers_timer64_Timer_stop__E                             
c3119220  xdc_runtime_Core_assignParams__I                                    
c31192c0  xdc_runtime_System_formatNum__I                                     
c3119360  xdc_runtime_System_putchar__I                                       
c3119400  xdc_runtime_Text_printVisFxn__I                                     
c31194a0  xdc_runtime_Text_xprintf__I                                         
c31195c0  EventCombinerP_getHwi                                               
c3119640  EventCombinerP_getIntNum                                            
c31196c0  UART_charPut_v0                                                     
c3119740  __TI_readmsg                                                        
c31197c0  __c6xabi_llshl                                                      
c3119840  ti_sysbios_family_c62_TaskSupport_swap__E                           
c3119840  ti_sysbios_knl_Task_SupportProxy_swap__E                            
c31198c0  edma3OsProtectExit                                                  
c3119940  edma3ParamCpy                                                       
c31199c0  finddevice                                                          
c3119a40  ti_sysbios_BIOS_atExitFunc__I                                       
c3119ac0  ti_sysbios_BIOS_registerRTSLock__I                                  
c3119b40  ti_sysbios_family_c64p_Cache_invL1pAll__E                           
c3119bc0  ti_sysbios_gates_GateHwi_Object__create__S                          
c3119c40  ti_sysbios_gates_GateMutex_Object__create__S                        
c3119cc0  ti_sysbios_hal_Hwi_checkStack                                       
c3119d40  ti_sysbios_hal_Hwi_initStack                                        
c3119dc0  ti_sysbios_heaps_HeapMem_Object__create__S                          
c3119e40  ti_sysbios_knl_Clock_doTick__I                                      
c3119ec0  ti_sysbios_knl_Idle_run__E                                          
c3119f40  ti_sysbios_knl_Semaphore_pendTimeout__I                             
c3119fc0  ti_sysbios_knl_Swi_startup__E                                       
c311a040  ti_sysbios_knl_Task_restore__E                                      
c311a0c0  malloc                                                              
c311a140  remove                                                              
c311a140  unlink                                                              
c311a1c0  xdc_runtime_Core_assignLabel__I                                     
c311a240  xdc_runtime_SysStd_abort__E                                         
c311a240  xdc_runtime_System_SupportProxy_abort__E                            
c311a2c0  xdc_runtime_System_atexit__E                                        
c311a340  xdc_runtime_System_aprintf_va__E                                    
c311a340  xdc_runtime_System_aprintf_va__F                                    
c311a340  xdc_runtime_System_avprintf__E                                      
c311a3c0  xdc_runtime_System_processAtExit__E                                 
c311a440  xdc_runtime_System_printf_va__E                                     
c311a440  xdc_runtime_System_printf_va__F                                     
c311a440  xdc_runtime_System_vprintf__E                                       
c311a4c0  HwiP_delete                                                         
c311a520  Osal_ClearInterrupt                                                 
c311a580  Osal_getHwAttrs                                                     
c311a5e0  Osal_getThreadType                                                  
c311a640  SPIDataFormatSetup                                                  
c311a6a0  SPI_Params_init                                                     
c311a700  SPI_control                                                         
c311a760  SPI_socGetInitCfg                                                   
c311a7c0  SPI_socSetInitCfg                                                   
c311a820  SPI_transfer                                                        
c311a880  SemaphoreP_delete                                                   
c311a8e0  SemaphoreP_pend                                                     
c311a940  UART_divisorLatchWrite_v0                                           
c311a9a0  UART_fifoWait_v0                                                    
c311aa00  UART_lineCharacConfig_v0                                            
c311ab20  __TI_writemsg                                                       
c311ab78  C$$IO$$                                                             
c311ab80  __c6xabi_llshru                                                     
c311abe0  _subcull                                                            
c311ac40  ti_sysbios_family_c64p_Hwi_switchAndDispatch__I                     
c311aca0  ti_sysbios_family_xxx_Hwi_switchAndRunFunc                          
c311ad00  edma3OsSemTake                                                      
c311ad60  lseek                                                               
c311adc0  memccpy                                                             
c311ae20  ti_sysbios_BIOS_errorRaiseHook__I                                   
c311ae80  ti_sysbios_BIOS_removeRTSLock__I                                    
c311aee0  ti_sysbios_BIOS_startFunc__I                                        
c311af40  ti_sysbios_family_c62_TaskSupport_start__E                          
c311af40  ti_sysbios_knl_Task_SupportProxy_start__E                           
c311afa0  ti_sysbios_family_c64p_Cache_setMar__E                              
c311b000  ti_sysbios_family_c64p_EventCombiner_Module_startup__E              
c311b060  ti_sysbios_family_c64p_EventCombiner_unused__E                      
c311b0c0  ti_sysbios_family_c64p_Hwi_getEventId__E                            
c311b120  ti_sysbios_gates_GateMutex_Object__delete__S                        
c311b180  ti_sysbios_heaps_HeapMem_free__E                                    
c311b1e0  ti_sysbios_knl_Clock_Module_startup__E                              
c311b240  ti_sysbios_knl_Queue_construct                                      
c311b2a0  ti_sysbios_knl_Semaphore_construct                                  
c311b300  ti_sysbios_knl_Swi_Module_startup__E                                
c311b360  ti_sysbios_knl_Task_enter__I                                        
c311b3c0  UART_putc                                                           
c311b420  write                                                               
c311b480  xdc_runtime_Memory_valloc__E                                        
c311b4e0  xdc_runtime_Text_cordText__E                                        
c311b540  MuxIntcP_create                                                     
c311b580  Osal_RegisterInterrupt_initParams                                   
c311b5c0  SPICSDisable                                                        
c311b600  SPICSEnable                                                         
c311b640  SPIClockModeSetup                                                   
c311b680  SPIDataFormatSetupSlave                                             
c311b6c0  SPIDelaySetup                                                       
c311b700  SPIIntInit2                                                         
c311b740  SPIPinControlSetup                                                  
c311b780  SPISetShiftDir                                                      
c311b7c0  SPITransmitData                                                     
c311b800  SemaphoreP_Params_init                                              
c311b840  SemaphoreP_post                                                     
c311b840  SemaphoreP_postFromClock                                            
c311b840  SemaphoreP_postFromISR                                              
c311b880  UART_breakCtl_v0                                                    
c311b8c0  UART_charGetNonBlocking_v0                                          
c311b900  UART_divisorValCompute_v0                                           
c311b940  UART_fIFOConfig_v0                                                  
c311b980  UART_fIFORegisterWrite_v0                                           
c311b9c0  UART_intDisable_v0                                                  
c311ba00  UART_intEnable_v0                                                   
c311ba40  UART_intIdentityGet_v0                                              
c311ba80  UART_loopbackModeControl_v0                                         
c311bac0  UART_open                                                           
c311bb00  UART_readLineStatus_v0                                              
c311bb40  _DebugP_assert                                                      
c311bb80  __TI_frcmpyd_div                                                    
c311bbc0  __c6xabi_abort_msg                                                  
c311bc00  __c6xabi_isinf                                                      
c311bc80  __c6xabi_strasgi_64plus                                             
c311bc80  __strasgi_64plus                                                    
c311bcc0  _args_main                                                          
c311bd00  ti_sysbios_family_c62_TaskSupport_buildTaskStack                    
c311bd40  edma3OsSemGive                                                      
c311bd80  free                                                                
c311bdc0  ti_sysbios_BIOS_exitFunc__I                                         
c311be00  ti_sysbios_BIOS_rtsLock__I                                          
c311be40  ti_sysbios_BIOS_rtsUnlock__I                                        
c311be80  ti_sysbios_family_c64p_Hwi_destruct                                 
c311bec0  ti_sysbios_family_c64p_Hwi_disableInterrupt__E                      
c311bec0  ti_sysbios_hal_Hwi_HwiProxy_disableInterrupt__E                     
c311bec0  ti_sysbios_hal_Hwi_disableInterrupt__E                              
c311bf00  ti_sysbios_family_c64p_Hwi_enableInterrupt__E                       
c311bf00  ti_sysbios_hal_Hwi_HwiProxy_enableInterrupt__E                      
c311bf00  ti_sysbios_hal_Hwi_enableInterrupt__E                               
c311bf40  ti_sysbios_family_c64p_primus_TimerSupport_enable__E                
c311bf40  ti_sysbios_timers_timer64_Timer_TimerSupportProxy_enable__E         
c311bf80  ti_sysbios_gates_GateHwi_Handle__label__S                           
c311bf80  xdc_runtime_Main_Module_GateProxy_Handle__label__S                  
c311bf80  xdc_runtime_System_Module_GateProxy_Handle__label__S                
c311bfc0  ti_sysbios_gates_GateHwi_Object__delete__S                          
c311c000  ti_sysbios_BIOS_RtsGateProxy_Handle__label__S                       
c311c000  ti_sysbios_gates_GateMutex_Handle__label__S                         
c311c000  ti_sysbios_heaps_HeapMem_Module_GateProxy_Handle__label__S          
c311c040  ti_sysbios_gates_GateMutex_Instance_init__E                         
c311c080  ti_sysbios_gates_GateMutex_leave__E                                 
c311c0c0  ti_sysbios_heaps_HeapMem_Handle__label__S                           
c311c0c0  xdc_runtime_Memory_HeapProxy_Handle__label__S                       
c311c100  ti_sysbios_heaps_HeapMem_Object__delete__S                          
c311c140  ti_sysbios_heaps_HeapMem_Object__get__S                             
c311c180  ti_sysbios_knl_Semaphore_destruct                                   
c311c1c0  ti_sysbios_knl_Swi_Object__get__S                                   
c311c200  ti_sysbios_knl_Task_Object__get__S                                  
c311c240  ti_sysbios_knl_Task_sleepTimeout__I                                 
c311c280  xdc_runtime_Error_check__E                                          
c311c2c0  xdc_runtime_Error_init__E                                           
c311c300  xdc_runtime_Registry_findById__E                                    
c311c340  xdc_runtime_System_abort__E                                         
c311c380  xdc_runtime_System_aprintf__E                                       
c311c3c0  xdc_runtime_System_exit__E                                          
c311c400  xdc_runtime_System_printf__E                                        
c311c440  Board_PLLInit                                                       
c311c460  Board_uartStdioInit                                                 
c311c480  EventCombinerP_disableEvent                                         
c311c4a0  EventCombinerP_dispatchPlug                                         
c311c4c0  EventCombinerP_enableEvent                                          
c311c4e0  HwiP_clearInterrupt                                                 
c311c500  HwiP_disable                                                        
c311c520  HwiP_restore                                                        
c311c540  MuxIntcP_clearInEvent                                               
c311c560  MuxIntcP_disableOutEvent                                            
c311c580  MuxIntcP_enableOutEvent                                             
c311c5a0  SPIData1Setup                                                       
c311c5c0  SPIGlobalControlSetup                                               
c311c5e0  SPIIntDisable                                                       
c311c600  SPIIntEnable                                                        
c311c620  SPIIntStatusClear                                                   
c311c640  SPIIntStatusGet                                                     
c311c660  SPILoopbackDisable                                                  
c311c680  SPILoopbackEnable                                                   
c311c6a0  SPIPwrDownDisable                                                   
c311c6c0  SPIPwrDownEnable                                                    
c311c6e0  SPIReceiveData                                                      
c311c700  SPIReset                                                            
c311c720  SPIRxFull                                                           
c311c740  SPITxEmpty                                                          
c311c760  SPIXferDisable                                                      
c311c780  SPIXferEnable                                                       
c311c820  UART_Params_init                                                    
c311c860  UART_divisorLatchDisable_v0                                         
c311c880  UART_fIFOCharPut_v0                                                 
c311c8a0  UART_fifoEmpty_v0                                                   
c311c8e0  UART_operatingModeSelect_v0                                         
c311c900  UART_pwremuConfig_v0                                                
c311c920  UART_write                                                          
c311c940  UART_writePolling                                                   
c311c960  __c6xabi_errno_addr                                                 
c311c980  _nop                                                                
c311c9e0  _register_lock                                                      
c311ca00  _register_unlock                                                    
c311ca20  ti_sysbios_family_c62_TaskSupport_glue                              
c311ca40  C$$EXIT                                                             
c311ca40  abort                                                               
c311ca40  xdc_runtime_System_abortStd__E                                      
c311ca60  __TI_decompress_none                                                
c311ca80  __TI_decompress_rle24                                               
c311caa0  disableErrorInterrupt                                               
c311cac0  disableXferCompInterrupt                                            
c311cae0  enableErrorInterrupt                                                
c311cb00  enableXferCompInterrupt                                             
c311cb20  putchar                                                             
c311cb40  ti_sysbios_BIOS_RtsGateProxy_enter__E                               
c311cb60  ti_sysbios_BIOS_RtsGateProxy_leave__E                               
c311cb80  ti_sysbios_BIOS_getThreadType__E                                    
c311cba0  ti_sysbios_BIOS_linkedWithIncorrectBootLibrary__E                   
c311cbc0  ti_sysbios_BIOS_nullFunc__I                                         
c311cbe0  ti_sysbios_BIOS_setThreadType__E                                    
c311cc00  ti_sysbios_BIOS_start__E                                            
c311cc20  ti_sysbios_family_c62_TaskSupport_Module__startupDone__S            
c311cc20  ti_sysbios_knl_Task_SupportProxy_Module__startupDone__S             
c311cc40  ti_sysbios_family_c64p_Cache_wbInv__E                               
c311cc60  ti_sysbios_family_c64p_Hwi_Module__startupDone__F                   
c311cc60  ti_sysbios_family_c64p_Hwi_Module__startupDone__S                   
c311cc60  ti_sysbios_hal_Hwi_HwiProxy_Module__startupDone__S                  
c311cc80  ti_sysbios_family_c64p_Hwi_Params__init__S                          
c311cc80  ti_sysbios_hal_Hwi_HwiProxy_Params__init__S                         
c311cca0  ti_sysbios_family_c64p_Hwi_clearInterrupt__E                        
c311cca0  ti_sysbios_hal_Hwi_HwiProxy_clearInterrupt__E                       
c311cca0  ti_sysbios_hal_Hwi_clearInterrupt__E                                
c311ccc0  ti_sysbios_family_c64p_Hwi_getFunc__E                               
c311cce0  ti_sysbios_family_c64p_Hwi_getHandle__E                             
c311cd00  ti_sysbios_family_c64p_Hwi_startup__E                               
c311cd00  ti_sysbios_hal_Hwi_HwiProxy_startup__E                              
c311cd00  ti_sysbios_hal_Hwi_startup__E                                       
c311cd20  ti_sysbios_family_c64p_Hwi_switchFromBootStack__E                   
c311cd20  ti_sysbios_hal_Hwi_HwiProxy_switchFromBootStack__E                  
c311cd20  ti_sysbios_hal_Hwi_switchFromBootStack__E                           
c311cd40  ti_sysbios_family_c64p_Hwi_unPluggedInterrupt__I                    
c311cd60  ti_sysbios_gates_GateHwi_Instance_init__E                           
c311cd80  ti_sysbios_gates_GateHwi_enter__E                                   
c311cda0  ti_sysbios_gates_GateHwi_leave__E                                   
c311cdc0  ti_sysbios_gates_GateHwi_query__E                                   
c311cdc0  xdc_runtime_Main_Module_GateProxy_query__E                          
c311cdc0  xdc_runtime_System_Module_GateProxy_query__E                        
c311cde0  ti_sysbios_gates_GateMutex_Instance_finalize__E                     
c311ce00  ti_sysbios_BIOS_RtsGateProxy_query__E                               
c311ce00  ti_sysbios_gates_GateMutex_query__E                                 
c311ce00  ti_sysbios_heaps_HeapMem_Module_GateProxy_query__E                  
c311ce20  ti_sysbios_hal_Hwi_Module_startup__E                                
c311ce40  ti_sysbios_heaps_HeapBuf_Object__get__S                             
c311ce60  ti_sysbios_heaps_HeapMem_Module_GateProxy_enter__E                  
c311ce80  ti_sysbios_heaps_HeapMem_Module_GateProxy_leave__E                  
c311cea0  ti_sysbios_heaps_HeapMem_isBlocking__E                              
c311cec0  ti_sysbios_knl_Clock_TimerProxy_getMaxTicks__E                      
c311cee0  ti_sysbios_knl_Idle_loop__E                                         
c311cf00  ti_sysbios_knl_Queue_Instance_init__E                               
c311cf20  ti_sysbios_knl_Queue_Object__get__S                                 
c311cf40  ti_sysbios_knl_Queue_destruct                                       
c311cf60  ti_sysbios_knl_Queue_empty__E                                       
c311cf80  ti_sysbios_knl_Semaphore_Instance_finalize__E                       
c311cfa0  ti_sysbios_knl_Semaphore_Params__init__S                            
c311cfc0  ti_sysbios_knl_Swi_disable__E                                       
c311cfe0  ti_sysbios_knl_Task_disable__E                                      
c311d000  ti_sysbios_knl_Task_enable__E                                       
c311d020  ti_sysbios_knl_Task_startup__E                                      
c311d040  ti_sysbios_knl_Clock_TimerProxy_Module__startupDone__S              
c311d040  ti_sysbios_timers_timer64_Timer_Module__startupDone__F              
c311d040  ti_sysbios_timers_timer64_Timer_Module__startupDone__S              
c311d060  ti_sysbios_timers_timer64_Timer_getMaxTicks__E                      
c311d080  xdc_runtime_Error_getSite__E                                        
c311d0a0  xdc_runtime_Error_raiseX__E                                         
c311d0c0  xdc_runtime_Gate_enterSystem__E                                     
c311d0e0  xdc_runtime_Gate_leaveSystem__E                                     
c311d100  xdc_runtime_Memory_HeapProxy_alloc__E                               
c311d120  xdc_runtime_Memory_HeapProxy_free__E                                
c311d140  xdc_runtime_Memory_calloc__E                                        
c311d160  xdc_runtime_Memory_free__E                                          
c311d180  xdc_runtime_Memory_getMaxDefaultTypeAlign__E                        
c311d1a0  xdc_runtime_Startup_exec__I                                         
c311d1c0  xdc_runtime_Startup_reset__I                                        
c311d1e0  xdc_runtime_Startup_rtsDone__E                                      
c311d200  xdc_runtime_SysStd_exit__E                                          
c311d200  xdc_runtime_System_SupportProxy_exit__E                             
c311d220  xdc_runtime_SysStd_putch__E                                         
c311d220  xdc_runtime_System_SupportProxy_putch__E                            
c311d240  xdc_runtime_SysStd_ready__E                                         
c311d240  xdc_runtime_System_SupportProxy_ready__E                            
c311d260  xdc_runtime_System_Module_GateProxy_enter__E                        
c311d280  xdc_runtime_System_Module_GateProxy_leave__E                        
c311d2a0  xdc_runtime_System_Module_startup__E                                
c311d2c0  xdc_runtime_System_snprintf_va__E                                   
c311d2c0  xdc_runtime_System_snprintf_va__F                                   
c311d2c0  xdc_runtime_System_vsnprintf__E                                     
c311d2e0  xdc_runtime_Text_ropeText__E                                        
c311d300  xdc_runtime_Text_visitRope__I                                       
c311d320  drvObj                                                              
c311e198  drvInstance                                                         
c3122978  edma3DrvChBoundRes                                                  
c312b258  resMgrObj                                                           
c3133c30  ti_sysbios_family_c64p_EventCombiner_Module__state__V               
c3134030  _ftable                                                             
c3134210  uartInitCfg                                                         
c3134300  ti_sysbios_knl_Task_Object__table__V                                
c31343b8  _stream                                                             
c3134458  spiInitCfg                                                          
c31344f8  ti_sysbios_knl_Swi_Module_State_0_readyQ__A                         
c3134578  _device                                                             
c31345f0  ti_sysbios_family_c64p_Hwi_Module__state__V                         
c313465c  _unlock                                                             
c313467c  edma3NumPaRAMSets                                                   
c31346c2  xdc_runtime_Error_Module__state__V                                  
c31346c4  __TI_ft_end                                                         
c31346c8  ti_sysbios_timers_timer64_Timer_Module_State_0_device__A            
c3134728  ti_sysbios_timers_timer64_Timer_Object__table__V                    
c3134778  ti_sysbios_knl_Task_Module__state__V                                
c31347c0  ccXferCompInt                                                       
c3134800  tcErrorInt                                                          
c3134840  ti_sysbios_gates_GateMutex_Object__table__V                         
c3134880  ti_sysbios_family_c64p_Exception_Module__state__V                   
c31348b0  ti_sysbios_knl_Swi_Object__table__V                                 
c31348e0  gOsal_HwAttrs                                                       
c313490c  ti_sysbios_knl_Clock_Module__state__V                               
c3134938  ti_sysbios_BIOS_Module__state__V                                    
c313495c  __errno                                                             
c313495c  errno                                                               
c3134960  ti_sysbios_knl_Task_Module_State_0_readyQ__A                        
c3134980  ti_sysbios_timers_timer64_Timer_Module_State_0_gctrl__A             
c31349a0  ti_sysbios_timers_timer64_Timer_Module_State_0_handles__A           
c31349c0  ti_sysbios_timers_timer64_Timer_Module_State_0_intFreqs__A          
c31349e0  xdc_runtime_Error_IgnoreBlock                                       
c3134a00  xdc_runtime_System_Module_State_0_atexitHandlers__A                 
c3134a20  ti_sysbios_knl_Swi_Module__state__V                                 
c3134a3c  ti_sysbios_family_c64p_Cache_Module__state__V                       
c3134a40  ti_sysbios_family_c64p_Hwi_Object__table__V                         
c3134a58  ti_sysbios_heaps_HeapMem_Object__table__V                           
c3134a70  ti_sysbios_timers_timer64_Timer_Module__state__V                    
c3134a88  ccErrorInt                                                          
c3134a90  ti_sysbios_family_c64p_Hwi_Module__root__V                          
c3134a98  ti_sysbios_family_c64p_primus_TimerSupport_Module_State_0_suspSrc__A
c3134aa0  ti_sysbios_gates_GateHwi_Module__root__V                            
c3134aa8  ti_sysbios_gates_GateMutex_Module__root__V                          
c3134ab0  ti_sysbios_hal_Hwi_Object__table__V                                 
c3134ab8  ti_sysbios_heaps_HeapMem_Module__root__V                            
c3134ac0  ti_sysbios_knl_Queue_Module__root__V                                
c3134ac8  ti_sysbios_knl_Semaphore_Module__root__V                            
c3134ad0  xdc_runtime_Registry_Module__state__V                               
c3134ad8  xdc_runtime_Startup_Module__state__V                                
c3134ae0  xdc_runtime_System_Module__state__V                                 
c3134ae8  ti_sysbios_family_c64p_primus_TimerSupport_Module__state__V         
c3134aec  ti_sysbios_heaps_HeapBuf_Module__state__V                           
c3134af0  ti_sysbios_gates_GateHwi_Object__table__V                           
c3134af4  xdc_runtime_Memory_Module__state__V                                 
c3134af8  ti_sysbios_knl_Task_Module_State_0_idleTask__A                      
c3134b00  xdc_runtime_Text_charTab__A                                         
c3136dd8  _ctypes_                                                            
c3136ed9  ti_sysbios_timers_timer64_Timer_localTimerBaseId__C                 
c3136eda  ti_sysbios_family_c64p_Cache_Module__id__C                          
c3136ee0  xdc_runtime_Text_nodeTab__A                                         
c3137164  ti_sysbios_family_c64p_Cache_EMIFA_BASE__C                          
c3137168  SPI_config                                                          
c313724c  UART_defaultParams                                                  
c313728c  UART_FxnTable_v0                                                    
c31372bc  ti_sysbios_family_c64p_Cache_EMIFA_CFG__C                           
c31372c0  UART_config                                                         
c31372f0  ti_sysbios_family_c64p_Hwi_Object__PARAMS__C                        
c313734c  ti_sysbios_family_c64p_Cache_EMIFA_LENGTH__C                        
c3137350  xdc_runtime_Startup_sfxnTab__A                                      
c313737c  ti_sysbios_heaps_HeapMem_Module__FXNS__C                            
c31373ec  ti_sysbios_gates_GateHwi_Module__FXNS__C                            
c3137410  ti_sysbios_gates_GateMutex_Module__FXNS__C                          
c3137434  ti_sysbios_heaps_HeapMem_Object__PARAMS__C                          
c3137458  ti_sysbios_knl_Semaphore_Object__PARAMS__C                          
c313753c  SPI_defaultParams                                                   
c313755c  ti_sysbios_family_c64p_Hwi_Object__DESC__C                          
c313757c  ti_sysbios_gates_GateHwi_Object__DESC__C                            
c313759c  ti_sysbios_gates_GateMutex_Object__DESC__C                          
c31375bc  ti_sysbios_heaps_HeapMem_Object__DESC__C                            
c31375dc  ti_sysbios_knl_Queue_Object__DESC__C                                
c31375fc  ti_sysbios_knl_Semaphore_Object__DESC__C                            
c3137654  SPI_FxnTable_v0                                                     
c3137688  ti_sysbios_gates_GateHwi_Object__PARAMS__C                          
c31376a0  ti_sysbios_gates_GateMutex_Object__PARAMS__C                        
c31376b8  ti_sysbios_knl_Queue_Object__PARAMS__C                              
c31376d0  xdc_runtime_Startup_sfxnRts__A                                      
c31376e6  ti_sysbios_family_c64p_EventCombiner_Module__id__C                  
c31376f8  ti_sysbios_family_c64p_EventCombiner_EVTMASK__C                     
c3137708  ti_sysbios_knl_Idle_funcList__C                                     
c3137710  xdc_runtime_Startup_firstFxns__A                                    
c3137718  xdc_runtime_Startup_firstFxns__C                                    
c3137720  xdc_runtime_Startup_lastFxns__C                                     
c3137728  ti_sysbios_family_c64p_Cache_EMIFB_BASE__C                          
c313772c  ti_sysbios_family_c64p_Cache_EMIFB_CFG__C                           
c3137730  ti_sysbios_family_c64p_Cache_EMIFB_LENGTH__C                        
c3137734  ti_sysbios_family_c64p_Cache_EMIFC_BASE__C                          
c3137738  ti_sysbios_family_c64p_Cache_EMIFC_CFG__C                           
c313773c  ti_sysbios_family_c64p_Cache_EMIFC_LENGTH__C                        
c3137740  ti_sysbios_family_c64p_Cache_E_invalidL1CacheSize__C                
c3137744  ti_sysbios_family_c64p_Cache_E_invalidL2CacheSize__C                
c3137748  ti_sysbios_family_c64p_Cache_MAR0_31__C                             
c313774c  ti_sysbios_family_c64p_Cache_MAR128_159__C                          
c3137750  ti_sysbios_family_c64p_Cache_MAR160_191__C                          
c3137754  ti_sysbios_family_c64p_Cache_MAR192_223__C                          
c3137758  ti_sysbios_family_c64p_Cache_MAR224_255__C                          
c313775c  ti_sysbios_family_c64p_Cache_MAR32_63__C                            
c3137760  ti_sysbios_family_c64p_Cache_MAR64_95__C                            
c3137764  ti_sysbios_family_c64p_Cache_MAR96_127__C                           
c3137768  ti_sysbios_family_c64p_EventCombiner_A_invalidEventId__C            
c313776c  ti_sysbios_family_c64p_EventCombiner_EVTRegs__C                     
c3137770  ti_sysbios_family_c64p_EventCombiner_E_unpluggedEvent__C            
c3137774  ti_sysbios_family_c64p_EventCombiner_Module__diagsEnabled__C        
c3137778  ti_sysbios_family_c64p_EventCombiner_Module__diagsIncluded__C       
c313777c  ti_sysbios_family_c64p_EventCombiner_Module__diagsMask__C           
c3137780  ti_sysbios_family_c64p_Exception_E_exceptionMax__C                  
c3137784  ti_sysbios_family_c64p_Exception_exceptionHook__C                   
c3137788  ti_sysbios_family_c64p_Exception_externalHook__C                    
c313778c  ti_sysbios_family_c64p_Exception_internalHook__C                    
c3137790  ti_sysbios_family_c64p_Exception_nmiHook__C                         
c3137794  ti_sysbios_family_c64p_Hwi_E_alreadyDefined__C                      
c3137798  ti_sysbios_family_c64p_Hwi_E_handleNotFound__C                      
c313779c  ti_sysbios_family_c64p_Hwi_E_invalidIntNum__C                       
c31377a0  ti_sysbios_family_c64p_Hwi_INTRMUX1Address__C                       
c31377a4  ti_sysbios_family_c64p_Hwi_LD_end__C                                
c31377a8  ti_sysbios_family_c64p_Hwi_LM_begin__C                              
c31377ac  ti_sysbios_family_c64p_Hwi_Module__diagsEnabled__C                  
c31377b0  ti_sysbios_family_c64p_Hwi_Module__diagsIncluded__C                 
c31377b4  ti_sysbios_family_c64p_Hwi_Module__diagsMask__C                     
c31377b8  ti_sysbios_family_c64p_Hwi_Module__loggerFxn1__C                    
c31377bc  ti_sysbios_family_c64p_Hwi_Module__loggerFxn8__C                    
c31377c0  ti_sysbios_family_c64p_Hwi_Module__loggerObj__C                     
c31377c4  ti_sysbios_gates_GateMutex_A_badContext__C                          
c31377c8  ti_sysbios_gates_GateMutex_Instance_State_sem__O                    
c31377cc  ti_sysbios_gates_GateMutex_Module__diagsEnabled__C                  
c31377d0  ti_sysbios_gates_GateMutex_Module__diagsIncluded__C                 
c31377d4  ti_sysbios_gates_GateMutex_Module__diagsMask__C                     
c31377d8  ti_sysbios_hal_Hwi_E_stackOverflow__C                               
c31377dc  ti_sysbios_heaps_HeapBuf_Instance_State_freeList__O                 
c31377e0  ti_sysbios_heaps_HeapBuf_Object__count__C                           
c31377e4  ti_sysbios_heaps_HeapBuf_numConstructedHeaps__C                     
c31377e8  ti_sysbios_heaps_HeapMem_A_align__C                                 
c31377ec  ti_sysbios_heaps_HeapMem_A_heapSize__C                              
c31377f0  ti_sysbios_heaps_HeapMem_A_invalidFree__C                           
c31377f4  ti_sysbios_heaps_HeapMem_A_zeroBlock__C                             
c31377f8  ti_sysbios_heaps_HeapMem_E_memory__C                                
c31377fc  ti_sysbios_heaps_HeapMem_Module__diagsEnabled__C                    
c3137800  ti_sysbios_heaps_HeapMem_Module__diagsIncluded__C                   
c3137804  ti_sysbios_heaps_HeapMem_Module__diagsMask__C                       
c3137808  ti_sysbios_heaps_HeapMem_Module__gateObj__C                         
c313780c  ti_sysbios_heaps_HeapMem_Object__count__C                           
c3137810  ti_sysbios_heaps_HeapMem_reqAlign__C                                
c3137814  ti_sysbios_knl_Clock_LM_begin__C                                    
c3137818  ti_sysbios_knl_Clock_LM_tick__C                                     
c313781c  ti_sysbios_knl_Clock_LW_delayed__C                                  
c3137820  ti_sysbios_knl_Clock_Module_State_clockQ__O                         
c3137824  ti_sysbios_knl_Clock_Module__diagsEnabled__C                        
c3137828  ti_sysbios_knl_Clock_Module__diagsIncluded__C                       
c313782c  ti_sysbios_knl_Clock_Module__diagsMask__C                           
c3137830  ti_sysbios_knl_Clock_Module__loggerFxn1__C                          
c3137834  ti_sysbios_knl_Clock_Module__loggerFxn2__C                          
c3137838  ti_sysbios_knl_Clock_Module__loggerObj__C                           
c313783c  ti_sysbios_knl_Semaphore_A_badContext__C                            
c3137840  ti_sysbios_knl_Idle_funcList__A                                     
c3137844  ti_sysbios_knl_Semaphore_A_noEvents__C                              
c3137848  ti_sysbios_knl_Semaphore_A_overflow__C                              
c313784c  ti_sysbios_knl_Semaphore_A_pendTaskDisabled__C                      
c3137850  ti_sysbios_knl_Semaphore_Instance_State_pendQ__O                    
c3137854  ti_sysbios_knl_Semaphore_LM_pend__C                                 
c3137858  ti_sysbios_knl_Semaphore_LM_post__C                                 
c313785c  ti_sysbios_knl_Semaphore_Module__diagsEnabled__C                    
c3137860  ti_sysbios_knl_Semaphore_Module__diagsIncluded__C                   
c3137864  ti_sysbios_knl_Semaphore_Module__diagsMask__C                       
c3137868  ti_sysbios_knl_Semaphore_Module__loggerFxn2__C                      
c313786c  ti_sysbios_knl_Semaphore_Module__loggerFxn4__C                      
c3137870  ti_sysbios_knl_Semaphore_Module__loggerObj__C                       
c3137874  ti_sysbios_knl_Swi_LD_end__C                                        
c3137878  ti_sysbios_knl_Swi_LM_begin__C                                      
c313787c  ti_sysbios_knl_Swi_LM_post__C                                       
c3137880  ti_sysbios_knl_Swi_Module__diagsEnabled__C                          
c3137884  ti_sysbios_knl_Swi_Module__diagsIncluded__C                         
c3137888  ti_sysbios_knl_Swi_Module__diagsMask__C                             
c313788c  ti_sysbios_knl_Swi_Module__loggerFxn1__C                            
c3137890  ti_sysbios_knl_Swi_Module__loggerFxn4__C                            
c3137894  ti_sysbios_knl_Swi_Module__loggerObj__C                             
c3137898  ti_sysbios_knl_Swi_Object__count__C                                 
c313789c  ti_sysbios_knl_Task_A_badTimeout__C                                 
c31378a0  ti_sysbios_knl_Task_A_sleepTaskDisabled__C                          
c31378a4  ti_sysbios_knl_Task_LD_block__C                                     
c31378a8  ti_sysbios_knl_Task_LD_exit__C                                      
c31378ac  ti_sysbios_knl_Task_LD_ready__C                                     
c31378b0  ti_sysbios_knl_Task_LM_sleep__C                                     
c31378b4  ti_sysbios_knl_Task_LM_switch__C                                    
c31378b8  ti_sysbios_knl_Task_Module_State_inactiveQ__O                       
c31378bc  ti_sysbios_knl_Task_Module__diagsEnabled__C                         
c31378c0  ti_sysbios_knl_Task_Module__diagsIncluded__C                        
c31378c4  ti_sysbios_knl_Task_Module__diagsMask__C                            
c31378c8  ti_sysbios_knl_Task_Module__loggerFxn2__C                           
c31378cc  ti_sysbios_knl_Task_Module__loggerFxn4__C                           
c31378d0  ti_sysbios_knl_Task_Module__loggerObj__C                            
c31378d4  ti_sysbios_knl_Task_Object__count__C                                
c31378d8  ti_sysbios_knl_Task_allBlockedFunc__C                               
c31378dc  ti_sysbios_knl_Task_numConstructedTasks__C                          
c31378e0  ti_sysbios_timers_timer64_Timer_A_notAvailable__C                   
c31378e4  ti_sysbios_timers_timer64_Timer_E_cannotSupport__C                  
c31378e8  ti_sysbios_timers_timer64_Timer_Module__diagsEnabled__C             
c31378ec  ti_sysbios_timers_timer64_Timer_Module__diagsIncluded__C            
c31378f0  ti_sysbios_timers_timer64_Timer_Module__diagsMask__C                
c31378f4  ti_sysbios_timers_timer64_Timer_anyMaskHigh__C                      
c31378f8  ti_sysbios_timers_timer64_Timer_anyMask__C                          
c31378fc  ti_sysbios_timers_timer64_Timer_freqDivisor__C                      
c3137900  ti_sysbios_timers_timer64_Timer_numLocalTimers__C                   
c3137904  ti_sysbios_timers_timer64_Timer_numTimerDevices__C                  
c3137908  xdc_runtime_Assert_E_assertFailed__C                                
c313790c  xdc_runtime_Core_A_initializedParams__C                             
c3137910  xdc_runtime_Core_Module__diagsEnabled__C                            
c3137914  xdc_runtime_Core_Module__diagsIncluded__C                           
c3137918  xdc_runtime_Core_Module__diagsMask__C                               
c313791c  xdc_runtime_Error_E_memory__C                                       
c3137920  xdc_runtime_Error_Module__diagsEnabled__C                           
c3137924  xdc_runtime_Error_Module__diagsIncluded__C                          
c3137928  xdc_runtime_Error_Module__diagsMask__C                              
c313792c  xdc_runtime_Error_Module__loggerFxn8__C                             
c3137930  xdc_runtime_Error_Module__loggerObj__C                              
c3137934  xdc_runtime_Error_policyFxn__C                                      
c3137938  xdc_runtime_Error_policy__C                                         
c313793c  xdc_runtime_Error_raiseHook__C                                      
c3137940  xdc_runtime_IGateProvider_Interface__BASE__C                        
c3137944  xdc_runtime_IHeap_Interface__BASE__C                                
c3137948  xdc_runtime_IModule_Interface__BASE__C                              
c313794c  xdc_runtime_Log_L_error__C                                          
c3137950  xdc_runtime_Memory_defaultHeapInstance__C                           
c3137954  xdc_runtime_Startup_execImpl__C                                     
c3137958  xdc_runtime_Startup_maxPasses__C                                    
c313795c  xdc_runtime_Startup_sfxnRts__C                                      
c3137960  xdc_runtime_Startup_sfxnTab__C                                      
c3137964  xdc_runtime_System_Module__gateObj__C                               
c3137968  xdc_runtime_System_abortFxn__C                                      
c313796c  xdc_runtime_System_exitFxn__C                                       
c3137970  xdc_runtime_System_extendFxn__C                                     
c3137974  xdc_runtime_System_maxAtexitHandlers__C                             
c3137978  xdc_runtime_Text_charTab__C                                         
c313797c  xdc_runtime_Text_nameEmpty__C                                       
c3137980  xdc_runtime_Text_nameStatic__C                                      
c3137984  xdc_runtime_Text_nameUnknown__C                                     
c3137988  xdc_runtime_Text_nodeTab__C                                         
c313798c  xdc_runtime_Text_visitRopeFxn__C                                    
c3137990  ti_sysbios_family_c64p_Exception_Module__id__C                      
c3137992  ti_sysbios_family_c64p_Exception_useInternalBuffer__C               
c3137994  ti_sysbios_family_c64p_Hwi_Module__id__C                            
c3137996  ti_sysbios_family_c64p_Hwi_Module__loggerDefined__C                 
c3137998  ti_sysbios_gates_GateMutex_Module__id__C                            
c313799a  ti_sysbios_hal_Hwi_Module__id__C                                    
c313799c  ti_sysbios_heaps_HeapMem_Module__id__C                              
c313799e  ti_sysbios_knl_Clock_Module__id__C                                  
c31379a0  ti_sysbios_knl_Clock_Module__loggerDefined__C                       
c31379a2  ti_sysbios_knl_Semaphore_Module__id__C                              
c31379a4  ti_sysbios_knl_Semaphore_Module__loggerDefined__C                   
c31379a6  ti_sysbios_knl_Swi_Module__id__C                                    
c31379a8  ti_sysbios_knl_Swi_Module__loggerDefined__C                         
c31379aa  ti_sysbios_knl_Task_Module__id__C                                   
c31379ac  ti_sysbios_knl_Task_Module__loggerDefined__C                        
c31379ae  ti_sysbios_timers_timer64_Timer_Module__id__C                       
c31379b0  ti_sysbios_timers_timer64_Timer_startupNeeded__C                    
c31379b2  ti_sysbios_timers_timer64_Timer_useTimer64pRegMap__C                
c31379b4  xdc_runtime_Core_Module__id__C                                      
c31379b6  xdc_runtime_Error_Module__loggerDefined__C                          
c31379b8  xdc_runtime_Error_maxDepth__C                                       
c31379ba  xdc_runtime_Main_Module__id__C                                      
c31379bc  xdc_runtime_Memory_Module__id__C                                    
c31379be  xdc_runtime_Text_charCnt__C                                         
c31379c0  xdc_runtime_Text_isLoaded__C                                        
c31379c2  xdc_runtime_Text_registryModsLastId__C                              
c31379c4  xdc_runtime_Text_unnamedModsLastId__C                               
c31379c8  _stack                                                              
c31389c8  __CIOBUF_                                                           
c31389c8  __TI_STACK_END                                                      
c3138bc8  __TI_STATIC_BASE                                                    
c3138bc8  dsp_num                                                             
c3138bcc  gOsalSemAllocCnt                                                    
c3138bd0  gOsalSemPeak                                                        
c3138bd4  gOsalTimerAllocCnt                                                  
c3138bd8  gOsalTimerPeak                                                      
c3138bdc  gOsalHwiAllocCnt                                                    
c3138be0  gOsalHwiPeak                                                        
c3138c00  ti_sysbios_family_c64p_Hwi0                                         
c3138c00  ti_sysbios_family_c64p_Hwi_int0                                     
c3138c20  ti_sysbios_family_c64p_Hwi_int1                                     
c3138c40  ti_sysbios_family_c64p_Hwi_int2                                     
c3138c60  ti_sysbios_family_c64p_Hwi_int3                                     
c3138c80  ti_sysbios_family_c64p_Hwi_int4                                     
c3138ca0  ti_sysbios_family_c64p_Hwi_int5                                     
c3138cc0  ti_sysbios_family_c64p_Hwi_int6                                     
c3138ce0  ti_sysbios_family_c64p_Hwi_int7                                     
c3138d00  ti_sysbios_family_c64p_Hwi_int8                                     
c3138d20  ti_sysbios_family_c64p_Hwi_int9                                     
c3138d40  ti_sysbios_family_c64p_Hwi_int10                                    
c3138d60  ti_sysbios_family_c64p_Hwi_int11                                    
c3138d80  ti_sysbios_family_c64p_Hwi_int12                                    
c3138da0  ti_sysbios_family_c64p_Hwi_int13                                    
c3138dc0  ti_sysbios_family_c64p_Hwi_int14                                    
c3138de0  ti_sysbios_family_c64p_Hwi_int15                                    
c3139704  __TI_Handler_Table_Base                                             
c313970c  __TI_Handler_Table_Limit                                            
c3139710  __TI_CINIT_Base                                                     
c3139740  __TI_CINIT_Limit                                                    
ffffffff  __TI_pprof_out_hndl                                                 
ffffffff  __TI_prof_data_size                                                 
ffffffff  __TI_prof_data_start                                                
ffffffff  __binit__                                                           
ffffffff  __c_args__                                                          
ffffffff  binit                                                               
UNDEFED   __TI_INITARRAY_Base                                                 
UNDEFED   __TI_INITARRAY_Limit                                                
UNDEFED   __TI_TLS_INIT_Base                                                  
UNDEFED   __TI_TLS_INIT_Limit                                                 

[794 symbols]
